:020000040800F2
:10000000000004201D8F0008A1340008A53400085A
:10001000A9340008AD340008B13400080000000025
:10002000000000000000000000000000E14B01089B
:10003000B5340008000000006D4C0108C94C0108EF
:100040006D8F00086D8F00086D8F00086D8F0008A0
:100050006D8F00086D8F0008B9340008C1340008A6
:100060006D8F00086D8F000805110008E51E00085F
:100070000D1F0008351F00086D8F00085D1F000868
:10008000691F00086D8F00086D8F00086D8F0008D4
:100090006D8F00086D8F00086D8F0008953800087F
:1000A0006D8F00086D8F00086D8F00086D8F000840
:1000B0006D8F00086D8F00086D8F0008311E0008DD
:1000C0003D1E0008491E0008551E0008611E00085C
:1000D0006D1E00086D8F0008791E00086D8F0008E6
:1000E000C93400086D8F00086D8F0008493500087D
:1000F00061350008793500086D8F0008911F0008F0
:10010000000000006D8F00086D8F00086D8F0008E3
:1001100000000000000000006D8F00086D8F0008D7
:10012000B91F0008C51F0008F91F00088D35000819
:100130006D8F00086D8F00086D8F00086D8F0008AF
:100140006D8F00086D8F00086D8F00086D8F00089F
:100150006D8F00089935000805200008951E0008DD
:100160006D8F00086D8F0008000000000000000087
:10017000000000000000000000000000000000007F
:100180006D8F00086D8F0008000000000000000067
:100190006D8F00086D8F0008000000000000000057
:1001A000000000000000000000000000000000004F
:1001B0006D8F000800000000000000006D8F000837
:1001C0006D8F000810B5034B0360044614F0A6FAC7
:1001D000204610BD109A010810B5054B0360044677
:1001E00014F09CFA2046082115F0F2FF204610BDBD
:1001F000109A010890F8A6340A4A10B50446C0F8CF
:10020000982423B1D0F8A00408B115F0E3FF94F8C6
:100210008A3423B1D4F8840408B115F0DBFF2046FA
:1002200010BD00BF289E010810B5064A064B0260AB
:10023000044640F8783F14F071FA204614F0A8FB09
:10024000204610BD2C9A0108109A010810B5064AE4
:10025000064B0260044640F8783F14F05FFA2046EF
:1002600014F096FB204610BD2C9A0108109A010844
:1002700010B5094A094B0260044640F8783F14F073
:100280004DFA204614F084FB20464FF4C27115F05D
:100290009FFF204610BD00BF2C9A0108109A01084C
:1002A00010B5084A084B0260044640F8783F14F045
:1002B00035FA204614F06CFB2046842115F088FFA7
:1002C000204610BD2C9A0108109A010808B5274C49
:1002D0002368BFF35B8FD90712D5254C2368BFF382
:1002E0005B8FDA072FD5234C2368BFF35B8FDB07C7
:1002F00017D5214B01221A7015F08AFB04F00AFD74
:10030000204600F003FD0028E7D01C4800F0D8FB91
:100310001B4A1C49194800F005FD204600F0FCFC72
:10032000DBE7204600F0F2FC0028E2D01349164833
:1003300000F092F9124A1549134800F0F3FC2046E8
:1003400000F0EAFCD5E7204600F0E0FC0028CAD027
:100350000A490F4800F06AF8094A0E490C4800F0B3
:10036000E1FC204600F0D8FCBDE700BF10040020EF
:10037000880200200002002058D901201404002027
:100380004D0D0008F50100080402002029020008B4
:100390008C0200204D02000808B5044600212046CA
:1003A00014F096FB78B9204614F0A0FB06280ED175
:1003B000D4F88000032102F035FD0021204614F01E
:1003C00087FB0028EFD0022003F068FBE6E704F08B
:1003D000A1FC00BF70B5541A82B00F2C0E460194D8
:1003E000054611D8012C006808D10B780370019CD8
:1003F00028686C600023035502B070BD5CB900230F
:100400006C60035502B070BD002201A915F0F0FE2A
:10041000019B2860AB602246314618F011FC019C1C
:1004200028686C600023035502B070BD70B5114A96
:1004300086B002AE04460D466846A2F10A01009657
:10044000FFF7C8FF032369464FF48062204614F08B
:100450001DFB0098B04203D00299013115F0B8FE9F
:10046000054B2360C4F88051204614F057FA20460B
:1004700006B070BD429A0108E89C010870B5D0F83A
:100480008051284600F084FB421E18BF0122064618
:100490000321284602F0FAFC32460121284602F0E8
:1004A000F5FC05F5987003F0DBF90FF0DDFC4E4824
:1004B0000EF01EFE4D48082278210FF00BFB4C4831
:1004C000C82278210FF006FB4A48DC2278210FF081
:1004D00001FB49481E2278210FF0FCFA47480EF034
:1004E00007FE012E75D004200EF0E6FD4448502290
:1004F00078210FF0EFFA301E18BF012080000EF0B7
:10050000DBFD6E2278213F480FF0E4FA00200EF068
:10051000D3FD3D48962278210FF0DCFA012200211C
:10052000284602F0B3FC0021284602F0D3FD032840
:10053000044629D0042830D0012C02464FF0030194
:10054000284617D102F0A2FC00222146284602F0DC
:100550009DFC04200EF0B0FD5022782128480FF0B9
:10056000B9FA00200EF0A8FD26486E2278210FF07F
:10057000B1FA0026FA2004F005FC0021284602F01A
:10058000A9FD03280446D5D1FA2004F0FBFB284638
:10059000314600F001FB304670BD002203212846A1
:1005A00002F074FC01221146284602F06FFC002084
:1005B0000EF082FD5022782111480FF08BFA204670
:1005C0000EF07AFD0F486E2278210FF083FA012693
:1005D000D0E700200EF070FD0948502278210FF07E
:1005E00079FA04208BE700BFD8E90108449A010892
:1005F0005C9A0108649A0108789A0108C0D9010838
:10060000909A0108A89A0108C09A01080000000009
:1006100030B595B00446FFF731FF9FED0D7B062303
:1006200040220021054603A88DED007B029318F0BF
:1006300074FA684614F066FA6421204614F058FAF9
:10064000D4F88001294600F02BFB15B030BD00BF67
:10065000030000000200000070B5114A86B002AE2F
:1006600004460D466846A2F10E010096FFF7B2FE61
:10067000022369464FF40072204614F007FA0098EE
:10068000B04203D00299013115F0A2FD054B236061
:10069000C4F88050204614F041F9204606B070BDE1
:1006A000EE9A0108FC9C010802484FF4DC3110F07E
:1006B00031B800BFD01100204FF0C043C0B2188045
:1006C000704700BF4FF0C0435880704741B100EB06
:1006D00041014FF0C04230F8023B53808842FAD1CA
:1006E000704700BF41B100EB41014FF0C042538859
:1006F00020F8023B8842FAD1704700BF30B5002491
:10070000A1B02146682206A801940294039404949F
:10071000059418F002FA23462246144914480FF0B3
:1007200007FB05460DF0F8FAF022114620460DF0C1
:1007300075FAF022114620460DF058FA20460321A2
:100740000EF0D2FD01A928460DF0EFF9094A0A4B37
:100750000A4C1194CDE90E23094A1592094B0A4A15
:1007600006A928460DF0FFF921B030BDE0F70108D9
:100770002CF60108B9060008C5060008CD060008D9
:10078000E506000831D5000895CE00084FF0FF308F
:10079000704700BF30B58BB01E4B00220192196B21
:1007A00041F008011963196B01F0080101910199E9
:1007B0000292196B41F040011963196B01F040017D
:1007C000029102990392196B41F0200119631B6B8E
:1007D0004FF4006003F0200303930490012304A965
:1007E0000D4805930224CDE90624039D04F0C4FDC1
:1007F0000822002304A90948CDE9042304F0BCFD24
:1008000020220123064804A9CDE9042304F0B4FD05
:100810000BB030BD00380240000C0240001802400E
:1008200000140240837B054A10B5044602601BB1E8
:10083000806808B115F0CEFC204610BD289E010846
:10084000837B084A10B5044602601BB1806808B17A
:1008500015F0C0FC20464FF4967115F0B9FC204607
:1008600010BD00BF289E01082DE9F04F0646808983
:10087000B369B568D6F80490C0F1004203EB4202B8
:10088000AA4238BF02EB400283B01088328A0A4481
:10089000121A32829A1CB2611980B6F80C8005EBEC
:1008A00048018A4214BFB2692A46B261D9F80000F1
:1008B000F26901924FEA4807023F2F4414468646E8
:1008C000002133F902A9BEF902C0BEF900B09D4271
:1008D00094BF1A463A461FFA8CFC32F902399BB291
:1008E0004CEA0B4C43EA0A43954288BF3A462CFB3C
:1008F000031C32F902A9BEF90610BEF904B09542F4
:1009000094BF13463B4689B233F9022992B241EAB9
:100910000B4142EA0A429D4288BF3B4621FB02C18D
:10092000013C0EF1080ECCD1D6F820E07361C6F878
:100930002811BEF1000F20D0019A08F1004808F1FB
:10094000FF384FEAC20C05EB480802E0D9F8000076
:1009500053469F1EAF422CBFBA46C24630F90C2008
:10096000B3F90030C6F814A012FB03110134A645F8
:10097000C6F828110CF1020CE8D8B6F9243091FB26
:10098000F3F000B203B0BDE8F08F00BF012200F227
:10099000644408B5114605460523204600F01CFBBB
:1009A00005F27C46204600F057FB0221304600F05D
:1009B0000DFC05F59365204600F074FB204600F021
:1009C00079FB0121204600F099FB40F30F212846D6
:1009D000FFF74AFF47F6FF7382B20221304600F06C
:1009E0000BFCE8E780B5DFED308A9FED30AADFED44
:1009F00030AADFED309A9FED309A82B00746B0EE14
:100A000068BAB7EE008A002500F5936900F2C45871
:100A100068EE0A7AD7F83006FDEEE77A17EE903ADC
:100A200019B208F063FEBEEEC98A484618EE103AC5
:100A30001CB22146FFF718FFC0EB0011090144BFAB
:100A400001F57F41FF3106460914D7F8340608F056
:100A50004DFE2A46CDE9005618492346404618F077
:100A600021F801354146002004F0FCF8B5F5817FFE
:100A700009D178EE8B8A0025F4EEEA8AF1EE10FABD
:100A8000C8BFDFED098A0EF077FC68EEA97A87EE21
:100A9000890A07EE905AF8EEE77A20EE270A15F059
:100AA000E7FBB0EE408AB3E70000C84200007042A6
:100AB00000007A44DB0FC94000007A45F09A010833
:100AC00030B5602189B0044601F0B6FA2C4BC4F869
:100AD000843404F2BE4281200021A4F8880484F802
:100AE0008A14C4F89034C4F894340292ADF80C001F
:100AF0004FF400538DF80E100592069204F28441D3
:100B000002AA04F5936000F0B9F99DF80E301BB10C
:100B1000029808B115F05EFB00251A4BC4F8983412
:100B20002846C4F8C055C4F82856C4F82C5603F01B
:100B30009DFF2946204600F04BFC2946204600F048
:100B400061FC2946204600F067FC0F4B01951A6BAB
:100B50000E4842F001021A631B6B03F0010301937C
:100B60004FF480620123CDE9022302A9002202236F
:100B7000CDE90423019B04F0FFFB204609B030BD02
:100B80001C9D0108109D0108003802400000024031
:100B9000032102F0BFBA00BF0A46032102F0B0BA37
:100BA000F0B5D0F82C5685B004460E462DB1284637
:100BB00005B0BDE8F04009F08EBA09F065FD4FF4CC
:100BC0000873039302230193F0231A4600902946E9
:100BD0000295284609F042F92A46C4F82C066FF01F
:100BE0007F4109F08FF92C49D4F82C06012209F035
:100BF00089F903222949D4F82C0609F083F9D4F89D
:100C00002C06012109F09BF9334604F23C624FF4B3
:100C1000F0714FF47F0008F02FFD334604F6FC120C
:100C2000C4F830064FF4F0714FF4004008F024FD92
:100C3000D4F83076C4F8340606463946D4F82C0683
:100C400009F01CF938463C2108F06BFDD4F82C065D
:100C5000314609F013F93046B42108F062FD14233F
:100C600001221146184608F0FBFBB7EE000AC4F853
:100C7000380608F023FCD4F83816D4F82C0609F00E
:100C80001FF9D4F82C06009514212B462A4609F0AA
:100C90006EF905B0F0BD00BF80808000404040008C
:100CA00008B505460C46C0F82816B1B90FF0DCF8B7
:100CB0001149204603F0D6FF1049204603F0D2FF29
:100CC0000F48502278210EF005FF0E486E22782141
:100CD0000EF000FF2846FFF759FE4FF4F071FFF7C2
:100CE0005FFF0949002003F0BDFF0449002003F025
:100CF000B9FF2846FFF776FE089B0108289B0108EC
:100D00006C9B0108889B0108A89B01080078B0FA39
:100D100080F04009704700BF01230370704700BF97
:100D2000704700BF00207047704700BFFEE700001B
:100D3000044A05491368002B08BF0B46184410608D
:100D400018467047D0C9012078180220002070474B
:100D5000837B074A10B5044602601BB1806808B166
:100D600015F038FA2046282115F032FA204610BD39
:100D7000289E0108837B054A10B5044602601BB11A
:100D8000806808B115F026FA204610BD289E01089B
:100D90002DE9F84F06468089B369B468D6F81CB0CF
:100DA000C0F1004203EB4202A24238BF02EB400214
:100DB0001088328A0A44121A32829A1CB26119804F
:100DC000B6F80CC004EB4C018A4214BFB26922464B
:100DD000B26172684FEA4C0CD2F800A0ACF1020C80
:100DE000A4440AEBCB0E52460020002133F90289BD
:100DF000B2F90070B2F902509C4294BF9946E146A4
:100E0000C8FB870139F90239B2F904704C4594BF27
:100E1000C846E046C3FB850138F90299B2F906508D
:100E2000444594BF43466346C9FB870133F90279C1
:100E300008329C4288BF63469645C7FB8501D5D1E1
:100E4000326A73614FEA8B0B82B15A440AEB420A51
:100E50001A463EF9025B32F9027994428CBF63462E
:100E60001346F245C7FB8501F2D17361B6F9242020
:100E7000D31716F0D3FB00B2BDE8F88FF8B51546CE
:100E80001F46AB79134A026004460E4641607BB9A7
:100E9000AA8883732B688281836043618361B288EF
:100EA000A784930802F00302E36122622046F8BDA2
:100EB000A888400015F090F9AB79AA88A06060611D
:100EC000A061A373A281002BE9D02968520017F01A
:100ED000B7FEE4E7289E010810B5034B0360044603
:100EE00013F07CFC204610BD3C9E010810B5054B5C
:100EF0000360044613F072FC2046082115F068F9DF
:100F0000204610BD3C9E010830B5044689B040F82B
:100F10000C1B0223A36060600822002117F0FDFD76
:100F200000251D4B00951A6B257542F002021A63CD
:100F30001A6B1A4802F002020092009A01951A6B8D
:100F400042F004021A631B6B03F0040301930122B5
:100F50000123CDE9022302A9019B00220023CDE950
:100F6000042304F009FA0E4B0E481022CDE90223A7
:100F700002A902230122CDE9042304F0FDF92A4647
:100F800009210A2003F022FF01220448114604F03F
:100F90000DFB204609B030BD00380240000402407D
:100FA000000021100008024070B505460C461646A8
:100FB00022460021286800F0A7F90022286811467F
:100FC00000F0A2F980B204B970BDB0424FF00A003F
:100FD000FAD003F0D7FEEBE7F8B517460022044637
:100FE0000E46006811461D4600F08EF9002211469B
:100FF000206800F089F945F2065211462046FFF7B5
:10100000D3FF43F64B020021206800F07DF9760201
:1010100000221146206806F47E4600F075F9002192
:1010200006F14D02206800F06FF900221146206899
:1010300000F06AF905EB4712D2B2120200214E32DB
:10104000206800F061F900222068114600F05CF988
:1010500001232375F8BD00BF10B540F24F3204469E
:101060000021006800F050F900221146206800F0CD
:101070004BF94FF44C5211462046FFF795FF45F2CD
:10108000055211462046FFF78FFF044813F0D0FBAE
:10109000034B4FF480621A6010BD00BFD8C9012015
:1010A00000E100E002484FF0FF3113F0B3BB00BF96
:1010B000D8C9012010B5044688B005A90E48019092
:1010C000032303AA2068039101A90293049300F06B
:1010D00049F9039B2068596802F022F86268039B73
:1010E000000A10609968206802F01AF86368000A24
:1010F000586008B010BD00BF449E0108436853F813
:101100002100704700B5102083B004F05BFA0A4854
:1011100001A913F09BFB019B012B09D14FF0E023A8
:101120004FF08052C3F8042DBFF34F8FBFF36F8F82
:1011300003B05DF804FB00BFD8C9012030B589B009
:101140001E4B002500951A6B016042F002021A63E3
:101150001A6B02F002020092009A01951A6B42F09B
:1011600004021A631B6B03F004030193144B4FF446
:101170008042CDE902230446012202A9114802233C
:10118000CDE90423019B04F0F7F82A460921282021
:1011900003F01CFE01220123CDE9022302A9022350
:1011A00000220948CDE9042304F0E6F801220648AC
:1011B000114604F0FBF9204609B030BD003802406A
:1011C00000002110000402400008024010B5032373
:1011D00084B0C943194080228DF806208DF805108F
:1011E00000688DF8043001AC02AA0121CDE9024368
:1011F00000F0CCF804B010BD10B584B01344303109
:1012000003220292C3F3072C8DF80C1000688DF8AE
:101210000DC003AC01AA012101948DF80E3000F03D
:10122000B5F804B010BD00BF0160704708B50022DA
:101230000121054813F014FBBDE80840034A0449A6
:101240000148FFF76FBD00BFD8C901204D0D000850
:10125000D90E000870B5064C064EA4F1280544F8D6
:10126000086D204613F0BAFAAC42F8D170BD00BF49
:1012700050CF01203C9E010810B50648064C40F8AE
:10128000084F13F0ABFA03480460BDE8104013F0B8
:10129000A5BA00BF50CF01203C9E010810B50648FA
:1012A000064C40F8084F13F099FA03480460BDE873
:1012B000104013F093BA00BF60CF01203C9E01089C
:1012C00010B50648064C40F8084F13F087FA03485B
:1012D0000460BDE8104013F081BA00BF70CF012058
:1012E0003C9E010810B50648064C40F8084F13F024
:1012F00075FA03480460BDE8104013F06FBA00BFF0
:1013000080CF01203C9E010800B585B0019279B9DB
:1013100004230DEB030103AA0E4806F097FF4FF0DC
:10132000FF310D4813F076FA039805B05DF804FB21
:10133000022201A9094806F01BFF41F234234FF0B5
:10134000FF310748039313F065FA039805B05DF881
:1013500004FB00BFF8CF012098CF0120A0CF0120CF
:1013600090CF012008B54B681268096805489B00BA
:101370009BB206F06BFFBDE8084003484FF0FF3119
:1013800013F048BAF8CF012098CF012008B51368B0
:10139000928851B919460A4806F0EAFEBDE80840AD
:1013A00008484FF0FF3113F035BA1946064806F0E9
:1013B000DFFEBDE8084005484FF0FF3113F02ABAC0
:1013C000F8CF012098CF0120A0CF012090CF01209D
:1013D00010B50B460848094AC45C525C08484FF4F3
:1013E000806104F0E3F822460548BDE810404FF460
:1013F000005104F0DBB800BF509E0108549E010864
:10140000001402400A1E034818BF0122202104F0E4
:10141000CDB800BF001002400A1E034818BF0122C9
:10142000402104F0C3B800BF0010024000B58BB0EB
:10143000264B00220092196B41F008011963196BC9
:1014400001F00801009100990192196B41F010011F
:101450001963196B01F01001019101990292196B46
:1014600041F020011963196B01F0200102910299EA
:1014700003921A6B42F040021A631B6B4FF4405008
:10148000012103F040030022CDE90401039304A9E4
:101490000F480023CDE90623039B03F06DFF602373
:1014A00004A90C48049303F067FF42F20C4304A91B
:1014B0000948049303F060FF4FF4984307480493EE
:1014C00004A903F059FF0BB05DF804FB003802409B
:1014D000000C0240001002400014024000180240BC
:1014E0002DE9F04F91B04FF0000BBD4CCDF80CB092
:1014F000236BBC48BC4D43F001032363236B03F013
:1015000001030393039BCDF810B0636C43F4805345
:101510006364636C03F48053A022022604930AA937
:101520004FF003084FF00509049B0A920127CDE90B
:101530000C680B96CDF8389003F01EFF1022122392
:10154000A8480C970AA9CDE90A2303F015FF402308
:10155000A4480A930AA9CDF830B003F00DFFA34BBD
:101560002B604FF482736B604FF48023AB610823D0
:10157000EB6128460A23C5F808B0C5F80CB0C5F8D9
:1015800010B06F61C5F820B0C5F824B0C5F828B018
:10159000EB6206F0ABFD002840F01F810590236B45
:1015A000DFF86CA2924A43F480032363236BCAF8EA
:1015B0000C0003F480030593059BCAF81400402334
:1015C000CAF80830CAF81800CAF81C00CAF82C007B
:1015D000CAF83000CAF800204FF480634FF08062F0
:1015E0004FF400314FF0040B5046CAF80420CAF8FB
:1015F0002880CAF81030CAF82010CAF824B003F0C6
:10160000B7FC0246002840F0E880394601903A20B5
:1016100003F0DCFB3A2003F015FCC5F848A0CAF83B
:101620003850DFF8F0A1019ACAF80820CAF80C2057
:10163000CAF81420CAF81820CAF81C20CAF82C20AE
:10164000CAF830206B4ACAF800204FF0C0624FF44D
:101650008063CAF8042050464FF44032CAF824B0E0
:10166000CAF81030CAF82880CAF8202003F080FC9D
:101670008346002840F0B18002463946382003F006
:10168000A5FB382003F0DEFB5A4631462320C5F87F
:101690004CA0CAF8385003F099FB232003F0D2FB8A
:1016A000CDF818B0236B43F002032363236B03F0E0
:1016B00002030693069BCDF81CB0236B43F0040392
:1016C0002363236B03F004030793079BCDF820B03B
:1016D000236C43F480432364236C0B960AAD0820EB
:1016E00003F4804329460A9008934348089BCDF8A9
:1016F0003890CDE90C6803F03FFE4FF400532946C3
:101700003E480A93CDF830B0CDF8389003F034FE5F
:101710004FF4805212233948CDF838902946384D7D
:101720000C97CDE90A2303F027FE0820354BE8612A
:101730004FF482720A206A60E8624FF480222B60C4
:1017400028464FF40043AA61C5F80CB02E61C5F8D5
:1017500014B0C5F820B0C5F824B0C5F828B0AB6007
:1017600006F0C4FC002838D10990236B43F4001321
:101770002363236B244C03F400130993099B6060DB
:101780004FF48063402223614FF400311F4BE0602F
:101790006061A061E0616062E06220632046C4F89D
:1017A0002880A2602162236003F0E2FB8046A0B99A
:1017B000394602460F20AC64A56303F007FB0F20F7
:1017C00003F040FB42463146242003F0FFFA242078
:1017D00003F038FB11B0BDE8F08F03F09BFA00BFB7
:1017E0000038024000000240F8CF012000300140E4
:1017F00040640240106402400008024000040240BD
:10180000A0CF01200038004008CC012070600240C9
:10181000C8CD012068CD01202DE9F04F8FB0884C54
:101820008848894E002503950A95236C43F40013DC
:101830002364236C03F400130393039B0495236C2C
:1018400043F480032364236C03F480030493049B18
:101850000595236B43F002032363236B03F002031C
:101860000593C02212234FF0020A4FF0040908A981
:10187000CDE90823CDF82CA0059BCDF8309003F0DE
:101880007BFD724B724AB560C6E900236E274FF4A8
:10189000804330467561B561F5613562F76033614B
:1018A00004F02EF9002840F0C8800690226B6949A8
:1018B00042F400122263226B02F400120692069A8E
:1018C000654A4FF480659060D06050619061D0614E
:1018D000506211604FF480384FF000711046516033
:1018E0001561C2F8208003F043FB8346002840F0D6
:1018F000A480594AB26396630C2102460B2003F080
:1019000065FA5649564AC1F804B0C1F80CB0C1F89E
:1019100014B0C1F818B0C1F81CB0C1F820B0C1F8BB
:1019200024B008464FF0400B0A600D61C1F808B0C2
:1019300003F01EFB024600287FD1484971638E6385
:1019400001900D210C2003F041FA12233D48099328
:1019500008A90123CDF830900A93CDF82CA0089562
:1019600003F00AFD4FF40073DFF80C91354808933B
:1019700008A909230C9303F0FFFC344BC9F8043089
:101980004FF48043019AC9F810304846354BC9F8E6
:101990000C70C9F80820C9F81420C9F81820C9F833
:1019A0001C20C9F82020C9F8003004F0A9F800284C
:1019B00043D10790236B43F400132363236B2A4C1A
:1019C00003F400130793079B284BA060E06060615D
:1019D000A061E06160624FF060672046C4E90037B3
:1019E000C4F82080256103F0C3FA064628BBC9F875
:1019F0003840C4F838901E4C02460C210D2003F0EC
:101A0000E5F91C4B67602046C4F808B0E660256124
:101A10006661A661E66126626662236003F0A8FA49
:101A2000024650B90C212F20C9F83440C4F8389030
:101A300003F0CCF90FB0BDE8F08F03F06BF900BFF5
:101A4000003802400004024034CA0120801A060017
:101A5000005400401060024048CB0120A8CB012078
:101A6000286002400058004088CA012040600240BF
:101A7000E8CA0120B8600240E0C901202DE9F04128
:101A80008AB000253F4E0195336B3F4C43F0010374
:101A90003363336B03F001030193019B0295336CB5
:101AA00043F400333364336C03F4003302930C20AB
:101AB00002210723CDE90401029A34480893012248
:101AC000032304A9CDE9062303F056FC304AA560A0
:101AD0004FF4E133C4E9002320460C23E56025617F
:101AE0006361A561E56107F029F8002847D10390FB
:101AF000336B284D43F400133363336BA86003F456
:101B000000130393244BE8606861A861E8612862D0
:101B100068624FF0006828464FF48067C5E90038D6
:101B2000039A2F6103F024FA064640BB02460D21BA
:101B300010206563AC63194D03F048F9102003F0E1
:101B400081F94023AB602846154BC5F80480EE6050
:101B50002F616E61AE61EE612E626E622B6003F0EA
:101B600007FA024658B90D2111202563AC6303F032
:101B70002DF9112003F066F90AB0BDE8F08103F0F9
:101B8000C9F800BF0038024028CD01200000024003
:101B90000044004068CC012088600240C8CC01208D
:101BA000A06002402DE9F0478AB0604E0024009406
:101BB000336B43F004033363336B03F0040300938C
:101BC000009B0194336B43F040033363336B03F0AA
:101BD00040030193019B0294736C43F020037364F0
:101BE000736C4020022103F020030825CDE9040195
:101BF00002934F48029B089504A94FF001084FF04B
:101C00000309CDE9068903F0B7FB4FF40072022304
:101C10004848089504A9CDE90423CDE9068903F0D5
:101C2000ABFB4FF440520223CDE904234148089511
:101C30000022032304A9404DCDE9062303F09CFBB9
:101C40003E4A3F4BAC60C5E900234FF400434FF4DC
:101C50004072EB6128460C23AA61EC602C616B6139
:101C600006F06CFF00285FD10390336B354C43F4D2
:101C700080033363336BA06003F480030393324B20
:101C8000E0604FF02069C4E900396061A061E06163
:101C9000E06220634FF4003320464FF4806A4FF037
:101CA00004080227039AC4F810A02362C4F8248011
:101CB000A76203F05DF90646002835D102460621E9
:101CC00039206C63A563214C03F080F8392003F0C0
:101CD000B9F840231E4AA36020464FF48033E660E3
:101CE0006661A661E661E6622663C4F80490C4F802
:101CF00010A0C4F82480A7622260236203F038F9A0
:101D0000064688B90246062146202C63A56303F0E7
:101D10005DF8462003F096F832460A21472003F08A
:101D200055F80AB0BDE8F08702F0F4FF0038024031
:101D30000008024000180240E8CE012000140140D3
:101D400080841E0028CE01202864024088CE012015
:101D5000B864024030B5044683B001F0BDFD40F2E6
:101D60000E2204F5AA70C4F850210021C4F84C01D9
:101D7000012516F0D2FE02F0CBFF15490095802315
:101D800004F55972002002F08BFF002811DA20467A
:101D9000FFF74CFB2046FFF7A3FB2046FFF73CFD77
:101DA0002046FFF76BFE2046FFF7FCFE204603B0FF
:101DB00030BD08490095802304F57972284602F069
:101DC0006FFF0028E3DB0449002002F04BFFDEE751
:101DD000CC9B0108DC9B0108EC9B010802680849C8
:101DE0001368884223F04003136003D0054B9842E8
:101DF00003D07047044801F03DBB044801F03ABBF2
:101E0000F8CF0120A0CF012098CF012090CF012052
:101E1000054B984200D0704702680448136823F0CD
:101E20004003136001F026BBF8CF012098CF0120BA
:101E3000014804F055BA00BF34CA0120014804F03B
:101E4000EBBE00BF34CA0120014804F049BA00BF0C
:101E5000E0C90120014804F0DFBE00BFE0C9012055
:101E6000014806F097BB00BFF8CF0120014806F0FB
:101E700091BB00BFA0CF012008B5044806F0D2FEF8
:101E8000BDE80840024801F0F5BA00BF28CD0120A6
:101E900080CF012070B5104C94F83A5094F8393046
:101EA0002046EDB2DEB206F0BDFE222D0BD0212E73
:101EB00000D070BD94F83930202BFAD1BDE87040C5
:101EC000064801F0D7BA94F83A30202BF1D1BDE89A
:101ED0007040034801F0CEBAE8CE012078CF01204F
:101EE00070CF012010B5074C204603F06BF994F831
:101EF0003530012B00D010BDBDE81040024801F084
:101F0000B9BA00BF48CB012060CF012010B5074C03
:101F1000204603F057F994F83530012B00D010BD5E
:101F2000BDE81040024801F0A5BA00BFA8CB0120CF
:101F300068CF012010B5074C204603F043F994F810
:101F40003530012B00D010BDBDE81040024801F033
:101F500091BA00BF88CA012050CF0120014803F088
:101F600031B900BF08CC012010B5074C204603F062
:101F700029F994F83530012B00D010BDBDE8104090
:101F8000024801F077BA00BF68CC012080CF012061
:101F900010B5074C204603F015F994F83530012BA5
:101FA00000D010BDBDE81040024801F063BA00BF88
:101FB000E8CA012058CF0120014803F003B900BF4F
:101FC00068CD012010B5094C204603F0FBF894F8C9
:101FD0003530012B00D010BD054B06482022BDE84E
:101FE000104083F8392001F045BA00BF28CE012007
:101FF000E8CE012070CF0120014803F0E3B800BF14
:10200000C8CD012010B5094C204603F0DBF894F848
:102010003530012B00D010BD054B06482022BDE80D
:10202000104083F8392001F025BA00BF88CE012086
:10203000E8CE012078CF012010B50446FFF78AFED4
:10204000214604F26440FEF75FFF214604F27C4023
:10205000FFF774F8214604F59060FFF7E5F8204695
:1020600010BD00BF38B5002201213048304C12F0BD
:10207000F7FB304A30492D48FEF754FE002201217B
:102080002E4812F0EDFB2B4A2B492C48FEF74AFE56
:10209000002201212A4812F0E3FB002201212948F5
:1020A00012F0DEFB234A28490020FEF73BFE002207
:1020B0000121264812F0D4FB00220121244812F00D
:1020C000CFFB1C4A23490020FEF72CFE00220121F1
:1020D000214812F0C5FB00220121204812F0C0FB6C
:1020E000144A1F490020FEF71DFE002201211D4851
:1020F00012F0B6FB002201211B4812F0B1FB0D4A81
:102100001A490020FEF70EFE04F1280520460022A1
:102110000121083412F0A4FBAC42F7D1BDE83840ED
:10212000044A13490020FEF7FDBD00BF98CF0120EF
:1021300028CF01204D0D0008D90E000890CF0120B6
:1021400080CF012088CF0120E512000870CF012048
:1021500078CF0120C112000860CF012068CF012094
:102160009D12000850CF012058CF0120791200089D
:1021700055120008B420704710B4B328144C94BF13
:1021800084464FF0000CA4F800C0B329114C94BF52
:102190008C464FF0000CA4F800C01418B42CDCBF1F
:1021A00002F1FF32801803EB0102D4BF80B2B320EA
:1021B000B42ADCBF03F1FF33C918074C074B20805A
:1021C000D4BF89B2B3215DF8044B1980704700BFBA
:1021D00052D0012050D00120020000200000002039
:1021E00008B501F005FD4FF6FF7008BDB42070473B
:1021F00008B5292001F088FDBDE80840382001F02D
:1022000083BD00BF08B5282001F07EFD142001F039
:1022100087FD102001F078FDBDE80840962001F010
:102220007FBD00BF70B5C0B282B0002200F11E04B5
:10223000A0F12F032A208DF805400E468DF80420CA
:102240008DF806208DF8073001F05EFD01AC2546C3
:1022500015F8010B01F052FD02AB9D42F8D1F1B22D
:10226000A1F14D032B208DF805108DF8073001F0FA
:102270004BFD14F8010B01F041FD02AB9C42F8D17B
:1022800002B070BD38B5D50802F4784305F0FC05FE
:102290001D441446ADB2FFF7C5FF2C2001F034FDFC
:1022A000284601F02BFDE00200F47840BDE83840FC
:1022B00001F024BD2DE9F8430546C60A05F01F08C4
:1022C000F60008461F4606EBC826C5F3451311461F
:1022D0004FEAC80805F4784505EB830508EB832829
:1022E000FFF7A0FF2C20B6B2ADB21FFA88F801F0BC
:1022F0000BFD8FB107F1FF390024284601F0FEFCE9
:10230000304601F0FBFC4C45404601D001F0F6FCA4
:102310000234A4B2A742F0D8BDE8F88338B5044629
:102320000D46FFF77FFF29462046FFF77BFF2E2053
:1023300001F0EAFC01F0EEFC01F0ECFC044601F0D7
:10234000E9FCC4F38502C0F3C42303EB421304F495
:102350007844181980B238BD2DE9F04F044615466F
:1023600083B02C2025440F46994601F0CDFCA542B0
:1023700019DD274EDFF8A080DFF8A0A0254B4FF035
:10238000000B3288A2420AD8B8F80020BA4206D818
:10239000BAF80020A24202D31A88BA4206D2023406
:1023A000A4B2AC42EDDB03B0BDE8F08F39F81B10EE
:1023B000C80800F0FC0001F4784108444FEA4B02E1
:1023C00080B2019201F09AFC019A39F81B000232A6
:1023D000C00239F802100192C90A00EBC10080B2B4
:1023E00001F08CFC691EA1420A4B02D10BF1020BD9
:1023F000D5E7019A39F80220D000C0B2520900EBAB
:10240000822080B201F07AFC0BF1020B014BC6E78F
:1024100052D001200000002050D0012002000020F6
:10242000354B2DE9F04F354C1B882488558895880D
:1024300001331B1B324C1FFA83FE324BB4F800C031
:102440001B880CF1010CACEB030C5389948911FA35
:102450008CFC9BB28C4587B043EA044348D9D7181B
:10246000C3B203F11E0A2F3B0CF1FF39DBB25FFA56
:102470008AFA00931FFA89F64FEA4E0B4FF00008D4
:10248000CDF804E002900391009B8DF814802A207F
:102490008DF815A08DF816808DF8173001F034FCFA
:1024A00005AC254615F8010B01F028FC06ABAB4244
:1024B000F8D1F2B28DF815202B204D3A8DF8172067
:1024C00001F022FC14F8010B01F018FC06ABA3424A
:1024D000F8D13B463146019A0298FFF73DFF039B36
:1024E000013E9945B6B25F4402D909F1FF39CBE705
:1024F00007B0BDE8F08F00BF0200002052D00120DD
:102500000000002050D001202DE9F04F01EB030B1B
:10251000594587B0894641D2C3B203F11E0A2F3B09
:10252000DBB20093109E029053005FFA8AFA019387
:1025300000270392009B8DF814702A208DF815A0B7
:102540008DF816708DF8173001F0DEFB05AD1FFA1F
:1025500089F4A84618F8010B01F0D0FB06AB9845AA
:10256000F8D15FFA89F28DF815202B204D3A8DF8BD
:10257000172001F0C9FB15F8010B01F0BFFB06ABFA
:102580009D42F8D13346039A02982146FFF7E4FEB4
:1025900009F10109019BD9451E44CBD307B0BDE821
:1025A000F08F00BF2DE9F04F0C4685B0114606466E
:1025B00020469A461546FFF735FE2C2001F0A4FB75
:1025C000BAF1000F47D0F30806F4784203F0FC0399
:1025D0001344E4B2F6029BB204F11E0B4D3D00938E
:1025E0002F3CB3B20026EDB201935FFA8BFBE7B24A
:1025F000B0462A208DF80C808DF80DB08DF80E8035
:102600008DF80F7001F080FB03ACA14619F8010BA7
:1026100001F074FB04AB9945F8D105F14D032B2073
:102620008DF80D308DF80F5001F06EFB14F8010B92
:1026300001F064FB04ABA342F8D12C2001F064FB51
:10264000009801F05BFB0136019801F057FB013562
:102650005645EDB2CDD105B0BDE8F08F30B583B0B1
:1026600001F0C6FA352001F04FFB002001F046FBD7
:102670003A2001F049FB062001F040FBB02001F0B8
:1026800043FB012001F03AFBFE2001F037FBB120B3
:1026900001F03AFBDE2001F031FB212001F02EFB9E
:1026A000B72001F031FB052001F028FB332001F0B9
:1026B00025FBB82001F028FB052001F01FFB33208B
:1026C00001F01CFBC82001F01FFB042001F016FBE9
:1026D000032001F013FBC92001F016FB5E2001F07E
:1026E0000DFB082001F00AFBCA2001F00DFB0A20B7
:1026F00001F004FB0C2001F001FB022001F0FEFAC6
:10270000CC2001F001FB032001F0F8FA042001F0D5
:10271000F5FAD02001F0F8FA0C2001F0EFFAB3201E
:1027200001F0F2FA022001F0E9FAC02001F0ECFA1F
:10273000532001F0E3FAC52001F0E6FA002001F091
:10274000DDFA452001F0DAFAC22001F0DDFA0320BB
:1027500001F0D4FA122001F0D1FADD2001F0D4FA10
:10276000002001F0CBFAB42001F0CEFA112001F0E4
:10277000CBFA962001F0D4FA1C4B01932A2001F0E9
:10278000C3FA01AC254615F8010B01F0B7FA02AB0C
:10279000AB42F8D10022B3232B208DF805208DF811
:1027A000073001F0B1FA14F8010B01F0A7FA02ABFF
:1027B0009C42F8D1362001F0A7FA832001F09EFA5E
:1027C000292001F0A1FA382001F09EFA2C2001F016
:1027D0009BFA4BF6D854002001F090FA013CFAD154
:1027E000142003B0BDE8304001F09ABA001E00D1B9
:1027F000F020704710B4EF28144C94BF84464FF07B
:10280000000CA4F800C0EF29114C94BF8C464FF087
:10281000000CA4F800C01418F02CDCBF02F1FF3249
:10282000801803EB0102D4BF80B2EF20F02ADCBF96
:1028300003F1FF33C918074C074B2080D4BF89B27E
:10284000EF215DF8044B1980704700BF56D001207E
:1028500054D001203E0000203C000020F0207047B2
:1028600008B501F0C5F9042001F04EFA01F052FA62
:1028700001F050FAC0B208BD08B5292001F044FAB1
:10288000BDE80840112001F03FBA00BF08B5BD20E7
:1028900001F03AFAFE2001F031FA102001F034FA8A
:1028A000BDE808400A2001F03BBA00BF70B5C3B2D2
:1028B00082B00022A3F111042A208DF807400E46B1
:1028C0008DF804208DF805308DF8062001F01CFAF3
:1028D00001AC254615F8010B01F010FA02AB9D4240
:1028E000F8D1F1B2A1F111032B208DF805108DF86C
:1028F000073001F009FA14F8010B01F0FFF902ABFF
:102900009C42F8D102B070BD10B51446FFF7CEFF5F
:102910002C2001F0F9F92046BDE8104001F0EEB995
:1029200070B50C460646114620461D46FFF7BEFF11
:102930002C2001F0E9F935B100243046013401F0D2
:10294000DDF9A542F9D170BD2DE9F04F04461546D9
:1029500083B02C2025440F46994601F0D5F9A542B5
:1029600019D9124EDFF84880DFF848A0DFF848B0E8
:1029700000233288A2420BD8B8F80020BA4207D808
:10298000BAF80020A24203D3BBF80020BA4205D215
:102990000134A542EDD803B0BDE8F08F39F813003B
:1029A000019301F0ABF9019B0133F1E756D001200F
:1029B00054D001203E0000203C000020344B2DE983
:1029C000F04F344C1B8824885588958801331B1B95
:1029D000314C1FFA83FC314BB4F800B01B880BF16B
:1029E000010BABEB030B5389948911FA8BFB9BB260
:1029F0008B4587B043EA044347D95FFA80FAD7187A
:102A00000BF1FF3BAAF111094FEA4C035FFA89F978
:102A10001FFA8BF600934FF00008CDF804C0029027
:102A200003912A208DF814808DF815A08DF816805A
:102A30008DF8179001F068F905AC254615F8010BE3
:102A400001F05CF906ABAB42F8D1F2B28DF815207B
:102A50002B20113A8DF8172001F056F914F8010BCC
:102A600001F04CF906ABA342F8D13B463146019A3E
:102A70000298FFF769FF009B1F44039B013E9B45A3
:102A8000B6B202D90BF1FF3BCBE707B0BDE8F08F40
:102A90003E00002056D001203C00002054D00120F0
:102AA0002DE9F04F0E4619448E4287B03FD25FFAAF
:102AB00080FBABF1110A5300109F00935FFA8AFA72
:102AC0004FF000080191029003922A208DF81480A3
:102AD0008DF815B08DF816808DF817A001F014F957
:102AE0000DF11409B4B24D4615F8010B01F006F9C9
:102AF00006AB9D42F8D1F2B28DF815202B20113A89
:102B00008DF8172001F000F919F8010B01F0F6F823
:102B100006AB9945F8D13B46039A02982146FFF748
:102B200013FF009B1F44019B01369E42CDD307B08B
:102B3000BDE8F08F38B504460D46FFF7B7FE2946CD
:102B40002046FFF7B3FE2E2001F0DEF801F0E2F898
:102B500001F0E0F8044601F0DDF8C4F38502C0F3AB
:102B6000C42303EB421304F47844181980B238BD2F
:102B70002DE9F04F85B088460190114640469946B0
:102B80001446FFF793FE2C2001F0BEF8B9F1000FB8
:102B900038D05FFA88F8A8F1110B113C00265FFAD3
:102BA0008BFBE5B237462A208DF80C708DF80D802E
:102BB0008DF80E708DF80FB001F0A6F803ACA246A8
:102BC0001AF8010B01F09AF804AB5345F8D105F15E
:102BD00011032B208DF80D308DF80F5001F094F873
:102BE00014F8010B01F08AF804ABA342F8D12C20B1
:102BF00001F08AF80136019801F080F801354E4560
:102C0000EDB2D0D105B0BDE8F08F00BF70B584B093
:102C100000F0EEFF102001F077F80A2001F080F8B4
:102C2000012001F071F8C82001F07AF8112001F0BC
:102C30006BF8782001F074F8362001F065F8002078
:102C400001F05CF83A2001F05FF8052001F056F839
:102C5000212001F059F84FF06F432A20009301F032
:102C600053F86E4601AD6C4614F8010B01F046F8BE
:102C7000A542F9D12B2001F047F8344614F8010B96
:102C800001F03CF8AC42F9D1332340F60C42B220BB
:102C9000ADF800208DF803308DF8043001F034F8E1
:102CA000751D344614F8010B01F028F8A542F9D13E
:102CB000B72001F029F8352001F020F8BB2001F001
:102CC00023F81F2001F01AF8C02001F01DF82C2075
:102CD00001F014F8C22001F017F8012001F00EF8FD
:102CE000C32001F00BF8C42001F00EF8202001F001
:102CF00005F8C62001F008F80F2000F0FFFFD020F3
:102D000001F002F8A42000F0F9FF22482249234AEA
:102D10000292CDE9000142F62953E020ADF80C30D3
:102D200000F0F2FF0DF1FF340D36254615F8010FC6
:102D300000F0E4FFAE42F9D140F206631022ADF894
:102D4000043040F6513344218DF80220ADF80830AC
:102D5000162243F22F13E1208DF807108DF80A2078
:102D6000ADF80C3000F0D0FF14F8010F00F0C6FFF2
:102D7000A642F9D1292000F0C7FF112000F0C4FFBE
:102D8000352000F0C1FF002004B0BDE8704000F025
:102D9000B5BF00BFD00811080C15393350361314D5
:102DA00030B5012883B00BD002280BD06024362028
:102DB00000F0AAFF204603B0BDE8304000F09EBFFF
:102DC0000024F4E70D4A009200233320ADF80430CC
:102DD00000F09AFF6C460DF1060514F8010B00F0A7
:102DE0008DFFA542F9D1372000F08EFF002000F0C2
:102DF00085FF502000F082FFC024D8E7000001F0DA
:102E000070B5064C064EA4F1280544F8086D20461E
:102E100011F0E4FCAC42F8D170BD00BF40D10120FC
:102E20003C9E010810B539B301291AD0154A16483D
:102E300032F81110C16000234FF448624260036110
:102E4000836005F0E5FD0246D0B90E212C2001F08B
:102E5000BDFF0D4805F092FCBDE810402C2001F0AC
:102E6000F1BF032000F002FE2C2001F0F9FFBDE8C5
:102E70001040054805F092BC032000F003FEF3E784
:102E800001F048FF6C9E0108C4D10120032970B5F0
:102E900025DD274D012AA5F10C0411D0022A29D0E5
:102EA000002A42D1234EB05C00F0ECFDA54206D0D2
:102EB00054F8042BB05C00F0E5FDA542F8D170BDDC
:102EC00000231C4EF05C00F0D1FDA542F7D054F871
:102ED000043BF05C00F0CAFDA542F8D170BD012AA8
:102EE0001DD0022A15D002BB124BBDE87040585CC1
:102EF00000F0C8BD00220F4EB05C00F0CFFDA5422F
:102F0000DDD054F8042BB05C00F0C8FDA542F8D128
:102F100070BD084BBDE87040585C00F0BFBD054B6C
:102F2000BDE87040585C00F0A1BD01F0F3FE00BFA9
:102F3000689E0108689E01084FF06043F0B44FF0AE
:102F4000E02CD3F8004E154E154F012000FA02F286
:102F500024EA02052243DCF8FC4D124844F0807458
:102F6000CCF8FC4D013900244FF0020CC3F8B07FBF
:102F7000C3F8005E0C4FC3F8804E0C4DC0F8F0C093
:102F800001614FF48071C3F8404E3760C0F80413FC
:102F9000C3F8805EF0BCC3F8002E7047001000E05C
:102FA00055CEACC5000004E0FE0300400D0001005A
:102FB000F0B5A5B0364A374B00240194106C40F0B0
:102FC00080501064126C02F080520192019A0294B7
:102FD0001A6842F440421A601B68119103F440439E
:102FE0000D204FF4A021022401220425CDE908017F
:102FF00002934FF4800608A8CDE90E46CDE91245AC
:10300000029B0A920D921095149404F05DFD002825
:103010003BD14FF48053059007900F27032103A85D
:1030200006930397049404F013FB034668BB032242
:1030300018921D934FF48072229368231C9215936B
:103040004FF00062482315A8199416951F92179304
:1030500004F0E0FB0446C0B93146024604F06EFAC3
:1030600004F0BCFA04F08EFB0B4BA3FB003080098C
:1030700001F004FF284601F06FFF224639464FF069
:10308000FF3001F0A3FE25B0F0BD01F043FE00BF0C
:103090000038024000700040D34D621038B505463C
:1030A0002D200C4601F0DCFE002001F0DFFC44B9CD
:1030B00030BF2D2001F0C6FEBDE83840012001F0F0
:1030C000D5BC0121002003F077FE60212846FFF7E0
:1030D0006FFFEEE738B5FFF7E1FF084D012400214F
:1030E000284611F097FB30B90134052C05F108058D
:1030F000F5D1062038BD204638BD00BF20D10120C3
:10310000132908B501D9022008BD04F01DFF0020D5
:1031100008BD00BF132901D90020704704F01ABF71
:1031200008BA704730B589B0194C00250095236B5B
:1031300043F010032363236B03F0100300930F206D
:1031400001210122CDE90201009B124802A90023BE
:10315000CDE9042302F010F9284600F093FC012089
:1031600000F090FC022000F08DFC032000F08AFCAF
:103170000195236C084A094943F080032364236CBA
:10318000116003F080030193019B09B030BD00BFC3
:103190000038024000100240C4D10120001C004051
:1031A00010B584B001F086FE194B01244FF0005297
:1031B0006846CDE902340192ADF8004001F098FE76
:1031C00013234FF0006106228DF808306846002373
:1031D00001918DF80B208DF80C308DF8014001F035
:1031E00087FE1C234FF08041022268468DF808308C
:1031F000032301918DF801208DF80B308DF80C40E0
:1032000001F076FE042001F063FE04B010BD00BFA3
:10321000110000032DE9F0438BB03D4B00250095D4
:103220001A6B42F002021A631A6B02F00202009259
:10323000009A01951A6B42F020021A631A6B02F091
:1032400020020192019A02951A6B42F040021A6321
:103250001A6B02F040020292029A03959A6B42F0B6
:1032600002029A639B6B03F00203044600260327C5
:103270000393C022274802234FF0090904A9CDE98E
:1032800004234FF00A08039BCDF82090CDE9066790
:1032900002F072F84FF4407202231E48CDF82080ED
:1032A00004A9CDE90423CDE9066702F065F80422FC
:1032B00002231948CDF8209004A9CDE90423CDE9D3
:1032C000066702F059F8402202231448CDF8208006
:1032D00004A9CDE90423CDE9066702F04DF80423E3
:1032E0000F49A3631022172321636563E2632364FC
:1032F0006564A564E564256504F1300003F024FEEF
:1033000020B901F07BF90BB0BDE8F08301F002FDBC
:10331000003802400014024000040240001802403D
:10332000001000A000B583B00B4B002201925A6B35
:1033300042F040025A635B6B084A40F87C2F03F06E
:1033400040030193019B04F077FD10B903B05DF8D1
:1033500004FB01F0DFFC00BF00380240000806500B
:1033600030B589B00025184B02951A6C42F4807272
:103370001A641B6C03F480730C46029301A903A822
:10338000029B04F025FA04F003FA1049104A0A607F
:1033900040F2E732CA600F4A0D614300A2FB0323EB
:1033A0009B0C013B08464B608D6005F031FB04220D
:1033B00021462D2001F00AFD2D2001F043FD034898
:1033C00005F0DCF909B030BD0038024040D10120E1
:1033D0000020004083DE1B4338B504460D4601F053
:1033E00011FB214B1A6842F400721A601A6842F409
:1033F00080621A601A6842F480721A60032001F039
:10340000D3FC0F212046FFF7ABFF29462046FFF7EC
:10341000CFFD04F0E3F8002208212046FFF78CFDE1
:10342000012000F047FBFFF77DFE2046FFF7F2FE8C
:103430002046FFF777FF0D4A0D480121C2F83C1ED8
:1034400000237F21FF22C4E90003A160E260236121
:103450006361A361204604F00BFD18B9FFF7A0FEDD
:10346000204638BD01F056FC003C024000004742B7
:103470000028004000B583B001A911F0E7F958B168
:10348000019B4BB14FF0E0234FF08052C3F8042D65
:10349000BFF34F8FBFF36F8F03B05DF804FB00BF26
:1034A000FEE700BFFEE700BFFEE700BFFEE700BF8C
:1034B000FEE700BF704700BF012002F083B800BFE5
:1034C000022002F07FB800BF08B54FF4804002F040
:1034D00079F8BDE808404FF4004002F073B800BF2F
:1034E000102808B525D008D8012811D0022821D1EC
:1034F000BDE808401048FFF7BDBFB0F5804F13D0BE
:10350000B0F5004F16D1BDE808400C48FFF7B2BF38
:1035100000F058FB0A4B003818BF012003EBC00035
:10352000BDE80840FFF7A6BFBDE808400548FFF723
:10353000A1BF08BD01F0EEFB38D1012030D1012040
:1035400018D1012028D1012008B5034805F046F91B
:10355000024B01221A7008BD84D1012080D10120C4
:1035600008B5044805F03AF9BDE80840032000F02A
:1035700095BA00BFC4D1012008B5034805F02EF963
:10358000BDE8084001F0ECBB40D10120014801F04A
:1035900019BE00BF58D00120014801F013BE00BF82
:1035A000B8D0012038B5094C04F128052046002286
:1035B0000121083411F054F9A542F7D1BDE8384093
:1035C000034A04490020FDF7ADBB00BF18D101201C
:1035D0004D0D0008012E000810B54FF6FF7000F0E9
:1035E00097FD002000F082FC4FF6FF7000F084FC95
:1035F000084800F087FC084A01236421002000F0FD
:1036000001FDBDE81040054A01237821002000F0AB
:10361000F9BC00BF80000020349C0108409C0108D8
:1036200070B504460D46204601F0ACF850B9A5B976
:103630002378642043B301F0A5FB204601F0A2F8F3
:103640000028F5D0642001F09DFBECE701F09AFB27
:10365000204601F097F80028F4D1012D4FF06400C6
:10366000F4D12378013B012B4FF064000CD901F019
:1036700089FB204601F086F80028E3D12378013B3E
:10368000012B4FF06400F2D801F076FB86B22046A1
:1036900001F078F80028FAD1237845B153B96420B5
:1036A00001F070FBBDE87040642001F06BBB013B92
:1036B000012BF4D901F060FB6438B0424FF0640094
:1036C00003D9BDE8704001F05DBB01F05BFBDEE7B4
:1036D000F8B5174D35F81150044600201E46174620
:1036E00000F004FC29461422284600F0C3FD4FF6E2
:1036F000FF7000F0FBFB0A222946284600F0BAFDC5
:1037000020460121FFF78CFF63883B80E3883380EC
:1037100000212046FFF784FF4FF6FF7000F0E6FB24
:10372000294628461422BDE8F84000F0A3BD00BF9A
:10373000789E010838B500210446C068FFF7EAFC0E
:1037400000283ED0030C6082A382E068012101259D
:10375000FFF7E0FC00283BD12046FFF73DFF00F0DB
:10376000B5FB054600F0BAFB012281B2A8B200F019
:10377000DDFF0546002833D12346014603F8140B2C
:1037800004F112022046FFF7A3FF638AA28AE068D1
:1037900043EA02422946FFF7B3FC2346012103F81E
:1037A000185B04F116022046FFF792FFE38A228B92
:1037B000E068012143EA0242FFF7A2FC01202074E5
:1037C00038BD05460121E068FFF7A4FC0028C3D0FE
:1037D000030CE0822383002DBED00120207438BD6D
:1037E0004FF6FF7000F088FB4FF4784000F07EFB4E
:1037F000164A01239121002000F004FC144A012301
:10380000A021002000F0FEFB012D17D0022D0AD0D0
:1038100000F064FBA0F141010E4A012389B20020AF
:1038200000F0F0FBCAE700F059FBA0F141010A4AA1
:10383000012389B2002000F0E5FBBFE7074A2B46D1
:10384000AF21002000F0DEFBB8E700BF4C9C010870
:10385000549C0108A89C0108949C0108789C0108CC
:1038600038B505460CF03AFB022000F071FD00F07F
:103870002DFB044600F032FB022281B2A0B200F020
:1038800055FF00B138BD2846FFF754FFBDE838406A
:1038900001F01AB810B50E4B5C6982B0202001F01F
:1038A00091FEA30601D402B010BD0A4801A910F090
:1038B000CDFF019B012BF6D14FF0E0234FF080525A
:1038C000C3F8042DBFF34F8FBFF36F8F02B010BD4D
:1038D000003C014004D2012010B582B00446FFF73D
:1038E0007BFD00210B4B01911A6B84F8401142F4CF
:1038F0008052C4F83C411A631B6B03F4805301935C
:10390000019B10F0F3FE042006F096FC204602B066
:1039100010BD00BF0038024008B500220121054853
:1039200010F09EFFBDE80840034A04490148FDF736
:10393000F9B900BF04D201204D0D0008D90E0008CE
:1039400030B5474B474C83428BB04FF0000545D014
:103950000295236B444843F002032363236B03F077
:10396000020302934FF480621223CDE90423002264
:103970000223CDE9062304A90423029A089301F047
:10398000FBFC4FF40072092304A937480492089302
:1039900001F0F2FC0395236C43F480032364236C51
:1039A00003F480030393039B236A43F4800323629D
:1039B000236A23F4800323622A460F21212001F089
:1039C00005FA212001F03EFA2A460F21222001F0BB
:1039D000FDF9222001F036FA0BB030BD0095236BC3
:1039E000214843F002032363236B03F00203009397
:1039F00040221223CDE9042300220223CDE906232D
:103A000004A90423009A089301F0B6FC802304A9BA
:103A10001548049301F0B0FC0195236C43F40013A6
:103A20002364236C03F400130193019B236A43F482
:103A300000132362236A23F4001323622A460F2112
:103A40001F2001F0C3F91F2001F0FCF92A460F21C5
:103A5000202001F0BBF9202001F0F4F90BB030BDBB
:103A60000CD2012000380240000402400246034B01
:103A7000034833F82210002201F098BDA49E0108EB
:103A8000001002400246034B034833F82210012283
:103A900001F08CBDA49E0108001002400246034BB9
:103AA000034833F8221001F085BD00BFA49E010831
:103AB000001002402DE9F04300228DB00223DFF810
:103AC00000813B4D3B4FCDE9082306464446A4EB1D
:103AD0000803052B4ED8DFE803F040331C074D03E5
:103AE00000200DB0BDE8F083334B002204921A6B26
:103AF00042F020021A631B6B03F020030493049B23
:103B000037F8023B0693AEB1012E40D004350134A4
:103B1000DDE7294B002203921A6B42F020021A6360
:103B20001B6B03F020030393039B37F8023B0693C0
:103B3000002EE9D12868079606A901F01DFCE5E7EB
:103B40001D4B002202921A6B42F040021A631B6B5B
:103B500003F040030293029BD2E7174B002201922D
:103B60001A6B42F001021A631B6B03F0010301930D
:103B7000019BC5E7104B002205921A6B42F04002F0
:103B80001A631B6B03F040030593059BB8E70B4BCF
:103B90002868079306A901F0EFFB94F90090002232
:103BA00048460F2101F012F9484601F04BF9ADE704
:103BB000909E0108849E01080038024000002110F8
:103BC0007C9E010870B5084E084D002435F8021B94
:103BD00056F8040B01F0E4FC20B90134052CF5D1B2
:103BE000204670BDE0B270BD909E0108849E010821
:103BF00010B53D49AEB04FF020400124CDE91A0187
:103C00002421CDE90C140222022309201021CDE940
:103C10000E23CDE91623CDE90A04344A1F9107206B
:103C20004FF480410023149026914FF480504FF4BC
:103C30000011CDE91C33CDE92033CDE922331093B7
:103C4000159318931E932593279328932B932993C9
:103C500001932490CDE912442A91916B2143916301
:103C6000916B2140019101990293116B41F0080180
:103C70001163116B01F00801029102990393116B1A
:103C800041F010011163116B01F0100103910399D0
:103C90000493136B43F020031363136B0794022107
:103CA00003F020030493069103210C220498089149
:103CB0004CF2B37305A90E480992059301F05CFB21
:103CC0004FF6807305A90B48059301F055FB05A934
:103CD0000948059401F050FB12AA0AA91AA804F099
:103CE0001FFD2EB010BD00BF040100A0003802402F
:103CF000000C024000100240001402404FF0C0438C
:103D00005880BFF34F8F70474FF0C0431880BFF308
:103D10004F8F70474FF0C043588880B2704700BF44
:103D200001F030B810B50E4C204603F041F80346C0
:103D3000A0B90C480C49A360C4E900014FF48042CB
:103D40002046E36022616361A361E3612362FFF7C0
:103D5000F7FD2046BDE8104001F0D2BE10BD00BF07
:103D60000CD2012000540040A086010010B586B09E
:103D70004FF47A73944602930A46012301460DF1EB
:103D800017000090019313488DF817C001F098FFB9
:103D900008B906B010BD0F4801F078FF0D4803F0D8
:103DA00007F803460028F4D10A4C0B490B48A360DE
:103DB000C4E900014FF480422046E3602261636160
:103DC000A361E3612362FFF7BBFD204601F098FE8B
:103DD00006B010BD0CD20120A086010000540040A6
:103DE00010B586B00A46002101234FF47A748DF88D
:103DF000171001460DF1170000900294144801932A
:103E000002F008F818B99DF8170006B010BD104868
:103E100001F03CFF0E4802F0CBFF03460028F2D130
:103E20000B4C0C490C48A360C4E900014FF48042DC
:103E30002046E36022616361A361E3612362FFF7CF
:103E40007FFD204601F05CFE9DF8170006B010BD16
:103E50000CD20120A08601000054004010B584B0AF
:103E60004FF47A74CDE9002302940A4601230146F7
:103E7000134801F0CFFF044610B9204604B010BD2E
:103E80000F4801F003FF0E4802F092FF034600289E
:103E9000F3D10B480B4A0C4942604FF48042016059
:103EA0008360C360026143618361C3610362FFF7A2
:103EB00047FD034801F024FE204604B010BD00BFBA
:103EC0000CD20120A08601000054004008B5024B2E
:103ED0001B689B6A984708BD60D2012008B5024B59
:103EE0001B68DB6A984708BD60D20120014B18604F
:103EF000704700BF68D20120014B5860704700BF77
:103F000068D20120014B9860704700BF68D2012041
:103F10002DE9F04F394B9C6887B0B4F804900491B8
:103F2000A2F12003E188256809F107028446D01038
:103F300001FB03F3C9EBC00200FB03F3D2B200297B
:103F400045D01D4409F1FF38DFF8B4A00591904435
:103F50002B4600224D460146E14604981E7800EBB0
:103F6000020B01291FFA8BFB07D0022932D11E78E0
:103F7000587846EA002676BAB6B2002401270191A5
:103F80000293039206E013B11C4A12889847013449
:103F9000A54214D9A8EB0402DAF8003007FA02F2BD
:103FA00009EB040032425B6980B25946EBD1002B29
:103FB000EDD0124A013492889847A542EAD8039A74
:103FC00005980199029B013290420B44C5D107B07C
:103FD000BDE8F08F35B15878360446EA0026987867
:103FE0000643CAE70598013290420B44EFD004988B
:103FF0001E7800EB020B1FFA8BFBB6E768D201209C
:1040000060D201202DE9F047174612F8014B064611
:1040100088461D461CB1104614F020FE441CDFF8F3
:104020009090DFF890A0D9F800309B6A9847DAF8B2
:104030000830012D9B88B0FBF3F031D0022D29D040
:1040400033B2002B07F1FF37D8BF0126002409E067
:104050003A78FFF75DFFDAF808309B880134334483
:10406000A4B29EB2D9F8003017F8015F9B6A003DF8
:1040700018BF01259847DAF808209288034602FB0A
:1040800014339BB293424146304601D3002DDFD119
:10409000BDE8F087001B10FB03F39B1B9EB2CFE72C
:1040A000001B00FB03F306EB53039EB2C8E700BFFF
:1040B00060D2012068D201202DE9F047DFF84CA042
:1040C000DAF800502C6A07468846164644B10E4A74
:1040D00033461088A4460A463946BDE8F047604793
:1040E0007AB1DFF8249001E0DAF800506B693819F2
:1040F000414680B213B1B9F8002098470134A64276
:10410000F2D1BDE8F08700BF68D2012060D2012063
:104110002DE9F041DFF838800C4ED8F800303768D0
:10412000DB6A30609847054660B10024D8F800305B
:104130009B6A9847A1B2024601340020FFF7BCFFFA
:10414000AC42F3D1BFB23760BDE8F08168D2012044
:1041500060D201202DE9F04F530087B0C3F1030373
:10416000CDE90001404F414E029392464FF00009C5
:104170000CE0029BA9EB0A020A330AF1FF3A09F1AB
:10418000010903EB8203CA4502936AD33B685B696A
:10419000002B59D0009A01991FFA89F41FFA8AF569
:1041A00002EB040BA1EB05081FFA8BFB1FFA88F842
:1041B00032885846414698473B68009A5B69121B13
:1041C00090B23288002B3FD0414603909847009A26
:1041D0003B68AA1891B2084601995B693288091BAD
:1041E00089B2002B30D00591049098473B68009A23
:1041F0005B69A2EB05081FFA88F8328823B305999A
:10420000404698473B6801995B6932880D44ADB2DE
:10421000D3B15846294698473B6832885B699BB1C1
:104220002946039898473B6801995B6932880C449A
:10423000A4B24BB10498214698473B6832885B6929
:1042400013B1214640469847094BB360029B002BAF
:104250008FDA063303EB890309F10109CA4502939A
:1042600094D207B0BDE8F08F60D2012068D201205F
:10427000780000202DE9F04FDFF8CC9083B0B9F83A
:104280000030C9F80030550082468846C5F1030564
:10429000164600240192CEB9A4BB002D05F10603F9
:1042A0004EDBA31B0A3505EB8305013E0134A64214
:1042B000F1D2019FB9F80030C9F800303A464146C2
:1042C000504603B0BDE8F04FFFF744BF1FFA86FB2E
:1042D000A3B2AAEB0B004FEA4B0B03EB080187B22A
:1042E0001FFA8BFB5A4689B238460093FFF7E4FE6B
:1042F000009BA8EB03015A4689B23846FFF7DCFE63
:10430000002CCAD01FFA84FBB3B2AAEB0B004FEA11
:104310004B0BA8EB030187B21FFA8BFB5A4689B2FD
:1043200038460093FFF7C8FE009B03EB08015A468E
:1043300089B23846FFF7C0FE002D05F10603B0DA5A
:1043400003EB8405B2E700BF68D201200000000043
:104350009FED2B7B70B52C4D2C4BAB6085ED007B1E
:104360000446FCF717FA2A482A4E0122202101F0C0
:104370001DF900224FF40061274801F017F90520CC
:1043800000F000FD01224FF40061234801F00EF916
:104390000A2000F0F7FC00224FF400611E4801F0F3
:1043A00005F9142000F0EEFC01224FF400611A48D8
:1043B00001F0FCF80A2000F0E5FC736898478528B6
:1043C00010D0164C636898474FF6FF73984201D09F
:1043D000012070BD124A236814609847114BAB60EE
:1043E000002070BD0E4A3368166098470CB1022C4D
:1043F000F4D12046FEF7D4FCF0E700BFAFF3008015
:1044000000000000FFFF000068D2012088000020AB
:104410000014024040000020000C02400400002074
:1044200060D201207800002030B595B09FED127B5E
:104430000521002203460124069110204FF08071CF
:10444000CDE90E21CDE91222CDE902040D920B92A5
:10445000119200924FF480756A4606A908480C959F
:104460008DED047B019402F061FE003818BF01203D
:1044700015B030BDAFF30080000000000000400028
:1044800074D201200000000010B594B04FF4807089
:10449000062100230C90069119480D9341F28832B1
:1044A00006A9CDE90E33CDE912330B93119302F037
:1044B000CFFD10B1012014B010BD9FED0F7B012284
:1044C0000392022310200522CDE9003302900692C8
:1044D00006A94FF0807441F288336A4608480F9469
:1044E0008DED047B02F022FE003818BF012014B0CD
:1044F00010BD00BFAFF300800000000000004000CE
:1045000074D2012070B58AB0384B39480024009429
:104510009A6B42F002029A639A6B02F002020092D6
:10452000009A9A6942F002029A619A6922F00202A4
:104530009A6101941A6B42F040021A631A6B02F0FE
:1045400040020192019A02941A6B42F002021A632D
:104550001A6B02F002020292029A03941A6B42F062
:1045600020021A631B6B03F02003039340220223F3
:10457000CDE904230A26012204A90323CDE9062359
:104580000925039B089600F0F7FE042304A91948A7
:1045900004930694089500F0EFFE4FF4807304A98D
:1045A00015480493089600F0E7FE04A94FF4007341
:1045B00011480493089600F0DFFE802304A90E48FA
:1045C0000493089500F0D8FE402304A90A480493F8
:1045D000089500F0D1FE22460F215C2000F0F6FB8A
:1045E0005C2000F02FFC0AB070BD00BF0038024014
:1045F00000180240000402400014024070B5494C0B
:10460000494B90B02046236002F00EFD054610B1E4
:10461000012010B070BD01462046FFF773FF042251
:104620001023A260E36065604FF0807696FAA6F3EF
:10463000B3FA83F3013B4FF4806220462361626149
:10464000A561E561256202F07FFC0028E0D1CDE99B
:104650000A00CDE90E004FF480756623099007909B
:104660000D9041F2883202A920460895029302F08B
:10467000EFFC10B1042010B070BD992341F28832D4
:1046800002A92046029302F0E3FC0028F2D141F295
:104690008830FFF7C9FE0028ECD18523CDE90A0652
:1046A000CDE90E0002930990012307900D9041F28D
:1046B000883202A9204608950C9302F0C9FC002814
:1046C000D8D141F288320DF10701204602F0A2FE56
:1046D0000028CFD1FFF7D8FE0028CBD18123029349
:1046E000F02292FAA2F29DF807300A20B2FA82F282
:1046F00000FA02F203F00F03134302A941F28832D9
:1047000020468DF8073002F0A3FC0028B2D141F218
:1047100088320DF10701204602F0F0FD00283FF439
:1047200078AFA7E774D20120001000A070B5114C3B
:10473000114E236830781546984763687020984773
:10474000CD2801D0032070BD8DB1022D0CBF0821F2
:104750000C210A4A0A4DA3681170702030702C6039
:1047600098472B683078DB689847002070BD062199
:10477000EFE700BF94000020D0D20120900000207D
:10478000D4D201202DE9F04FDFF8E0B0344ADBF855
:10479000003005461B69107883B0984728700028C0
:1047A00059D001AADFF8C8802E4F6E46AA464FF0B6
:1047B00000091446DBF80030294A5B69107831465D
:1047C00022469847284B34F8020B1A7836F8023BF9
:1047D000110706D5194626F8020C24F8023C0346B8
:1047E0000846910704D5C3F1EF039BB226F8023CBB
:1047F000520704D5C0F1EF0080B224F8020CD8F8BB
:104800000020D7F800E093421FFA82FC1FFA8EF1D5
:104810008CBFA3EB0C02ACEB030270458CBFA0EB8A
:10482000010EA1EB000E92B21FFA8EFE7244052A11
:1048300004DDC8F80030386001469C462AF802CFF3
:10484000AAF804102B7809F101094B4508F1040876
:1048500007F10407AED8002003B0BDE8F08F00BF19
:10486000D0D20120C0D2012090000020D4D201205B
:10487000C8D201200000000000B589B0104B1148DB
:10488000002201921A6B42F040021A631B6B9FEDEB
:104890000A7B03F0400301930122022302A9CDE920
:1048A00004238DED027B019B00F066FD09B05DF8ED
:1048B00004FB00BFAFF300802000000000002110C7
:1048C000003802400018024008B5FFF7D5FF0F215D
:1048D0000022172000F07AFA172000F0B3FA044BF8
:1048E000044A1B6810789B699847002008BD00BFE8
:1048F000D4D20120D0D20120704700BF00207047E1
:1049000010B50446FFF70EFAA821E0B2FFF768FAE7
:1049100010BD00BF10B582B000240221C0B28DF8D6
:104920000740FFF75DFA8DF807009DF8073003F0A8
:104930000F038DF807309DF80730022B88BF8DF8E4
:1049400007409DF80710044B9DF80700597000229E
:104950009A7002B010BD00BFD8D2012070B5164CBD
:104960001546A37862789A4282B00E461FD903B3E7
:10497000012B0CBF0921002104230DEB0302C0B25F
:10498000FFF76CFA9DF804309DF805209DF807109C
:104990001B0203F470631A439DF8063032801B0239
:1049A000A27803F470631943531C2980A37002B0EA
:1049B00070BD0321E0E700BFD8D201200122A4216D
:1049C000C0B2FFF7D3B900BF0022A421C0B2FFF7E5
:1049D000CDB900BF064A1378834204D0517888428B
:1049E00001D013B101B170470123D054FFF79AB938
:1049F000DCD20120704700BF0022A421C0B2FFF723
:104A0000B5B900BF10B4174A116885B04FF0E02364
:104A1000490400910099D3F8244D2143C3F8241D83
:104A20001168890401910199D3F8244D2143C3F8F9
:104A3000241D12680C4912010292029AD3F8144DF7
:104A40002243C3F8142D0A686FEAC2020392039A44
:104A5000D3F8141D0A40C3F8142D05B05DF8044BBB
:104A6000704700BFBCCC0108B8CC0108012882B057
:104A70000BD00B4B1B684FF0E022DB430093009BF5
:104A800011690B40136102B07047064B4FF0E022F2
:104A90001B680193019B11690B43136102B07047BE
:104AA000B8CC0108BCCC01082DE9F041C468876886
:104AB0000546164600202B699C4223D2013B1A1B57
:104AC0003B1BB34228BF3346934228BF13461844CA
:104AD0006A68F61A03EB04085BB1013C02EB040CB4
:104AE0000B4411F801EB0CF801EF8B42F9D1AF68E0
:104AF0001946B84514BF44460024EC60002EDAD1B4
:104B0000BDE8F0815A1E3A44121BD9E7F0B4C368DD
:104B100086684468F71A974203EB020523440BD9D1
:104B20003AB1013B0A4411F8014B03F8014F91429D
:104B3000F9D1C560F0BC704747B1013BCC1911F801
:104B4000012B03F8012FA142F9D14468AD1BF0D02D
:104B5000631E4C1911F8012B03F8012FA142F9D162
:104B6000C560F0BC704700BF10B5154A154C16481B
:104B70001649C4E906209FED107B4FF48060206247
:104B800010200023C4E91821A0661149A362042261
:104B9000E01D6362E3622367E366636784ED047B81
:104BA00014F04EF80B4B93E803002022A271206012
:104BB000A18010BDAFF300800300000003000000DF
:104BC000C09C0108F0D60120F0D20120E0D20120E3
:104BD000CC9C0108D09C010838B5214B00EB400467
:104BE00003EBC40E0130DEF82C4000EB4000012C3A
:104BF0008C46154603EBC00015D0022C0FD034BBF9
:104C0000DEF82830DEF8242093429CBFDEF8201026
:104C10005B18013B9A1A95421CD9204638BDBDE865
:104C20003840FFF741BFDEF82830DEF82440A342C9
:104C30009CBFDEF820105B18013B1C1B944228BF70
:104C4000144622466146FFF761FF204638BD002426
:104C5000204638BD2A466146FFF758FF2C46DCE760
:104C6000F0D60120F8B5054608460C4613F0F6FFCD
:104C70000A4B1B7806466BB1EFF311874FF020010A
:104C800081F31188324621462846FFF7A5FF87F3B6
:104C90001188F8BDFFF768FFEEE700BFF0D60120EE
:104CA0002DE9F041194D1E462B78044688461746DB
:104CB00033B32B69A34226D9EFF3118C4FF02001B7
:104CC00081F3118854B92246131905EBC305069BDD
:104CD000EB628CF311880020BDE8F081601C00EBD2
:104CE0004000C00004EB440305EBC30345F800801B
:104CF00028440021476062001E6299625962E3E71E
:104D0000FFF732FFD5E74FF0FF30E5E7F0D601209F
:104D1000FFF72ABFFEE700BF38B50E4A0E4B1278E8
:104D2000054618684FF47A73B3FBF2F3B0FBF3F067
:104D300000F0A4F8044608B90F2D01D9012038BDB0
:104D4000024629464FF0FF3000F040F8034B204662
:104D50001D6038BDBC000020C4000020C000002041
:104D6000034A044B11681B780B441360704700BF63
:104D700098D70120BC000020014B1868704700BF85
:104D800098D7012038B50446FFF7F6FF631C0546A7
:104D900002D0044B1B781C44FFF7EEFF401BA042DF
:104DA000FAD338BDBC0000200749CA6803024FF699
:104DB000FF0003F4E0630240134343F0BF6343F496
:104DC0000033CB60704700BF00ED00E01B4BDB6899
:104DD000C3F3022300B5C3F1070EBEF1040F03F1C4
:104DE000040C28BF4FF0040EBCF1060F1CD9A3F130
:104DF000030C4FF0FF3303FA0CF322EA03024FF0E7
:104E0000FF3303FA0EF321EA030303FA0CF313430F
:104E10001B010028DBB20ADB00F1604000F56140B5
:104E200080F800335DF804FB00229446E7E7044A6B
:104E300000F00F00024413765DF804FB00ED00E083
:104E4000FCEC00E0002807DD4109044A00F01F00E7
:104E50000123834042F82130704700BF00E100E0A9
:104E6000002808DD4309044900F01F000122203317
:104E7000824041F82320704700E100E00138B0F1A2
:104E8000807F10B403D301205DF8044B70474FF0CE
:104E9000E023074C58614FF0F00C84F823C0002247
:104EA000072110469A615DF8044B1961704700BFF5
:104EB00000ED00E0BFF35F8F044B5A6A002122F43B
:104EC00080325A62C3F89410704700BF00ED00E0D2
:104ED000064B40F00100C3F894005A6A42F4803255
:104EE0005A62BFF34F8FBFF36F8F704700ED00E042
:104EF0001849437800B5C1F8983002781AB343686E
:104F0000C1F89C30C37A90F80CC090F80FE01B06F3
:104F100043EA0C7390F80AC0134343EACC4390F879
:104F20000DC0827B43EA8C4343EA424390F809C0B8
:104F3000027A43EA0E4343EA0C2343EA4203C1F8F0
:104F4000A0305DF804FBC1F89C20C1F8A0205DF8FA
:104F500004FB00BF00ED00E04FF0E02204281369DD
:104F60000CBF43F0040323F004031361704700BF38
:104F700038B50446FFF700FF0546002C6AD02368C9
:104F8000022284F835201A68002122F0010284F8F8
:104F900034101A6005E0FFF7EFFE431B052B37D8EE
:104FA00023681A68D107F6D4A0686268E1682569A9
:104FB00002430A436169A0692A430A43E1691D6803
:104FC00002430A4331492940256A2A430A43616A58
:104FD000042924D01A605A6922F007021143D8B27A
:104FE0002B4A59611038A2FB0052120929496FF36C
:104FF0000903895CE1655F2888BF04333F228A404A
:10500000A36500209A600123606584F8353038BDBF
:10501000032320226265184684F8353038BDE56ADE
:10502000216B2943114319605969A26A21F00701D4
:10503000114341F00401002DD1D068B9012A21D0DB
:1050400032F00202CBD1EA01C9D5402201236265C8
:1050500084F83530012038BDB0F5005F04D0022A55
:10506000F3D9032AEFD0BAE7032AB8D801A050F841
:1050700022F000BF4B500008475000084B5000087A
:1050800085500008B5F1C07FA9D1DEE73F8010F060
:10509000ABAAAAAAC0CC010870B490F83440856DC0
:1050A000012C0AD090F835404FF0010C644580F88F
:1050B00034C005D0002380F83430022070BC704723
:1050C000022680F83560046800264665266826F4C6
:1050D0008026266063608368402B0EBFA260A160BB
:1050E000E260C26D08BFE1603F239340AB6023687C
:1050F000026C43F0160323601AB1236843F00803DF
:105100002360236843F001030020236070BC7047D4
:1051100070B50446866DFFF72FFE94F83530022BEC
:10512000054606D080220023626584F834300120D1
:1051300070BD23681A6822F016021A605A6922F0BC
:1051400080025A61226C32B31A6822F008021A6097
:105150001A6822F001021A6005E0FFF70DFE431BFA
:10516000052B0FD823681B6813F00103F5D1E16DFF
:105170003F228A400121B260184684F8343084F816
:10518000351070BD032020220023626584F834307E
:1051900084F8350070BDA26C002AD5D1D8E700BFD5
:1051A00090F83530022B03D08023436501207047EF
:1051B0000268052380F83530136823F001030020CE
:1051C00013607047F0B583B0674A876D1668002397
:1051D0000193C36D3D6808229A402A42044603D0D9
:1051E00001680868400778D401229A402A4203D017
:1051F0002168496908066AD404229A402A4203D0E9
:105200002168096889075CD410229A402A4203D099
:1052100021680868000741D420229A402A4214D00D
:1052200021680868C00610D5BA6094F83520052AB0
:1052300063D00B6813F4802F0B687ED0190340F104
:105240008980E36B0BB120469847636D23B3636D90
:10525000DA071AD522684549052384F835301368E2
:10526000A1FB061623F00103B60A136002E01368DF
:10527000DB0704D5019B0133B3420193F7D9002228
:10528000012384F8342084F83530E36C23B12046C0
:1052900003B0BDE8F040184703B0F0BDBA600A683B
:1052A00012F4802F0A6822D1D20503D40A6822F0B2
:1052B00008020A60226C002AAED020469047E36DB7
:1052C000AAE7BA60626D42F0040262659CE7BA60C8
:1052D000626D42F0020262658EE7086820F0040009
:1052E0000860BA60626D42F0010262657CE71103FA
:1052F000E0D5A26C002AE0D18EE70A6822F01602FF
:105300000A604A6922F080024A61226C3AB30A6854
:1053100022F008020A603F2202FA03F3216DBB600B
:105320000022012384F8342084F835300029B3D0DA
:10533000204603B0BDE8F040084713F4807380D1E5
:105340000A6822F010020A60012284F8343084F8DE
:10535000352076E7636C002B7FF475AF75E7A26CA0
:10536000002AD4D1D7E700BFC4000020B5814E1B6E
:1053700090F83500704700BF2DE9F04F00230D680D
:1053800083B04FF0010803E00133102B00F094804C
:1053900008FA03F232EA050402EA050AF4D14C687D
:1053A0008E684FEA430E24F0100C06FA0EF90CF149
:1053B000FF3B032606FA0EF6BBF1010F6FEA060665
:1053C0007DD9C268324042EA0902C26002681640D2
:1053D00004F0030202FA0EF232430260E200D3D577
:1053E000674E00220192726C42F480427264726CC9
:1053F00002F480420192019A23F0030202F18042FA
:1054000003F0030C0F2702F59C324FEA8C0C07FACD
:105410000CFE5C4F9668B84226EA0E0623D007F5CC
:105420008067B84200F08B80574FB84200F08C8004
:10543000DFF85CE1704500F08E80DFF858E17045E0
:1054400000F08F80DFF850E1704500F09180DFF8C8
:105450004CE170450CBF4FF0060E4FF0070E0EFAF0
:105460000CFC46EA0C069660484A1268E7036FEAAD
:105470000A06464F54BF32404AEA02023A607A684E
:10548000A703424F54BF32404AEA02027A60BA6828
:10549000E7023E4F54BF32404AEA0202BA60FA685D
:1054A000A40203F10103394C54BF32404AEA02021C
:1054B000102BE2607FF46CAF03B0BDE8F08FD0F842
:1054C00008B0CF680BEA060B07FA0EFA4AEA0B0A95
:1054D000C0F808A0D0F804A02AEA020A22099A40DB
:1054E00042EA0A024260C268324042EA0902BCF162
:1054F000020FC26008D004F00302046802FA0EF240
:105500003440224302603FE70CFA0EFC4FEAD30E10
:1055100000EB8E0E0C69DEF8209003F0070292007B
:105520000F27944007FA02F229EA02021443CEF848
:105530002040026832404CEA0202026024E708FA86
:105540000CFC46EA0C068EE74FF0020E0EFA0CFC3D
:1055500046EA0C0687E7032707FA0CFC46EA0C0626
:1055600081E74FF0040E0EFA0CFC46EA0C067AE7CF
:105570004FF0050E0EFA0CFC46EA0C0673E700BF6E
:10558000003802400000024000080240003C014098
:10559000000C0240001002400014024000180240BB
:1055A00000690840003818BF0120704702B909049B
:1055B00081617047436931EA030308BF09048161CF
:1055C000704700BF044A5169014208B500D108BDC7
:1055D0005061FDF785FF08BD003C01402DE9F8430F
:1055E0000F46804616461D464FEA1149B9F1010F94
:1055F000D8F8003002D111E0691C19D19C696FEA1A
:10560000040CCCF3400C8CF0010C5FFA8CFC66456A
:10561000F2D00020BDE8F8836A1C09D15C6927EA52
:105620000404A4B2B4FA84F46409B442F4D0F0E7F8
:10563000FFF7A2FB089BC01AA84201D8002DD5D1C4
:1056400000222023C8F8302088F83D3088F83E201A
:10565000D8F8403088F83C2043F02003C8F84030A8
:105660000120D7E72DE9F84307460E4690469946B4
:105670003D686C6926EA0404A4B2002C3ED06B6934
:105680005B050FD4B8F1FF3F03D023E06B695A05E7
:1056900008D46B6926EA03039BB2002BF6D11846A7
:1056A000BDE8F8832B6843F400732B6000222023AD
:1056B0006FF4806169613A6387F83D3087F83E2076
:1056C0003B6C43F004033B64002387F83C3001202B
:1056D000BDE8F883FFF750FBA0EB0900404502D876
:1056E000B8F1000FC4D1002320223B6387F83D208E
:1056F00087F83E303B6C13433B64E5E72046CFE739
:1057000070B504460D4616462068436913F0400301
:1057100018D14269D20617D4FFF72EFB801BA8428E
:1057200001D8002DF0D100232022236384F83D20EE
:1057300084F83E30236C13432364002384F83C3008
:10574000012070BD002070BD6FF01001202241616A
:10575000236384F83D2084F83E30236C2364ECE717
:10576000036D5BB9C36C0268012B836C15D0C3F366
:1057700007231361036D013303657047036D012B2C
:1057800003D0036D022B0ED07047836C0268DBB22E
:105790001361036D013303657047DBB21361036D61
:1057A00002330365704790F83D30222B0ED090F8FD
:1057B0003D30212BE8D1426A036812F8011B1961C0
:1057C000438D4262013B9BB24385DDE7026813686B
:1057D00043F480731360704770B504460D46164657
:1057E00023685A6910062FD45A69510519D46A1CC6
:1057F00011D0FFF7C1FA801BA84201D8002DEFD1CC
:1058000000232022236384F83D2084F83E30236C5B
:105810001343236413E05A69150615D45A695605D3
:10582000F9D500226FF4806020215861226384F84A
:105830003D1084F83E20236C43F0040323640023CE
:1058400084F83C30012070BD002070BD70B5044666
:105850000D46164623685A6950072FD45A695105D8
:1058600019D46A1C11D0FFF787FA801BA84201D80F
:10587000002DEFD100232022236384F83D2084F8FB
:105880003E30236C1343236413E05A69550715D443
:105890005A695605F9D500226FF4806020215861BD
:1058A000226384F83D1084F83E20236C43F0040307
:1058B0002364002384F83C30012070BD002070BDBB
:1058C0002DE9F0479946036890461A6842F48072C1
:1058D00082B01A605A690A9E0B9FD20705468A4613
:1058E00010D4711C0BD0FFF747FAC01B86422B68FF
:1058F00033D3002E31D05A69D00703D4F3E75C6963
:10590000E207FCD50AF0FE021A612A493B463246FC
:105910002846FFF7A7FED8B92B6801905969019175
:105920009B6901933A4631462846019BFFF754FF95
:10593000044650B9B9F1010F2B6826D15FFA88F2FD
:1059400020461A6102B0BDE8F0872B6C042B2BD0E7
:105950000124204602B0BDE8F087002120222963FF
:1059600085F83D2085F83E102A6C85F83C1042F001
:1059700020022A641B68DC0502D54FF400732B64F7
:105980000324204602B0BDE8F0874FEA18201861D2
:105990003A4631462846FFF71FFF0028D5D12A682E
:1059A0005FFA88F31361D4E72A68136843F400733D
:1059B0001360CDE7020001002DE9F0470468994625
:1059C000236843F4806384B0236023680C9E0D9F9A
:1059D00043F4807323606369DB0705468A4690467B
:1059E00010D4711C0BD0FFF7C7F9C01B86422C687E
:1059F00052D3002E50D06369D80703D4F3E763690C
:105A0000DA07FCD50AF0FE0323613B493B463246E8
:105A100028465FFA8AFAFFF725FE002838D12B685E
:105A20000390596903919B6903933A46314628468E
:105A3000039BFFF7D1FE40BBB9F1010F2B6842D1A8
:105A40005FFA88F21A613A4631462846FFF7C4FEEB
:105A5000D8B902462868016841F480710160334674
:105A600000974FF001112846FFF7B8FD2A6800287B
:105A70003ED14AF001032049136128463B46324695
:105A800004B0BDE8F047FFF7EDBD2B6C042B29D027
:105A9000012004B0BDE8F087002220232A6385F8A6
:105AA0003D3085F83E202B6C85F83C2043F02003E8
:105AB0002B642368DC0502D54FF400732B640320AC
:105AC00004B0BDE8F0874FEA18221A6131463A4621
:105AD0002846FFF781FE0028D7D12A685FFA88F3AD
:105AE0001361B0E72A68136843F400731360CFE7CB
:105AF0001368DB05E3D5DFE702000100704700BF54
:105B000070B50446002800F09B8090F83D3003F00B
:105B1000FF02002B00F096802368242284F83D20A9
:105B20001A6822F001021A601A6842F400421A60F0
:105B30001A6822F400421A6001F02AFE4D4B616897
:105B400099424DD84C4B98427AD922684B4D490026
:105B5000A5FB0035431EB3FBF1F3516821F03F0173
:105B600041EA95415160116AAE0C013621F03F01C6
:105B700031431162D06940F6FC7C013320F44F4080
:105B800013EA0C0F20F0FF0061D104230343D3611B
:105B90001168206AE36921F0C00103430B431360DD
:105BA0009168E068236921F40341034321F0FF0178
:105BB0000B439360D168A069636921F0FF0103433F
:105BC0000B43D3601168002341F0010120201160D4
:105BD000236484F83D002363184684F83E3070BD8A
:105BE000274B98422CD92268244B5668A3FB003CD3
:105BF00026F03F0646EA9C4656604FEA9C45431E07
:105C00004FF496761F4806FB05F5A0FB0505106AC4
:105C1000AD0920F03F00013505431562D069A56844
:105C200020F44F4020F0FF00A5B901EB4101B3FB88
:105C3000F1F30133C3F30B03CBB143F40043A5E706
:105C4000012070BD80F83C20FFF758FF64E7C3F3E4
:105C50000B039BE701EB810101EB8101B3FBF1F346
:105C60000133C3F30B0313B143F440438EE7012325
:105C70008CE700BFA08601007F841E0083DE1B43EB
:105C8000FF083D00D34D6210704700BF10B50446B9
:105C9000A0B10268242380F83D30136823F001038B
:105CA0001360FFF7F1FF00232364184684F83D30AA
:105CB00084F83C30236384F83E3010BD012010BDD1
:105CC0002DE9F04F044683B09946BDF834A00E9EEE
:105CD0000F469046FFF750F894F83D30202B0546CC
:105CE00008D0022003B0BDE8F08FFFF745F8401B55
:105CF00019287BD8206883696FEA030C1CF0020B1B
:105D0000F3D094F83C30012BEBD003680122DB0781
:105D100084F83C2078D53946076827F40067076087
:105D20000C98606221200195009684F83D00402087
:105D300084F83E0000202064A4F82AA0608D20850D
:105D40003348E0624B4642462046FFF7B9FD002843
:105D500048D1238D5BB32A4631462046FFF73CFDF0
:105D6000002837D1676A2068B4F828C039460CF19A
:105D7000FF3211F8013B0361638D013B9BB26385E8
:105D8000D0F814E0616293B21EF0040F2385E1D0D5
:105D90006BB17A780261628DACF1020C013A1FFAA4
:105DA0008CF3023792B2676223856285D2E72A4676
:105DB00031462046FFF74AFD60B92268136820216A
:105DC00043F40073136084F83D1084F83C0084F8B9
:105DD0003E0087E7236C042B04D12268136843F448
:105DE00000731360012003B0BDE8F08F2023C4F8D6
:105DF00030B084F83D3084F83EB0236C84F83CB079
:105E000043F0200323646CE703681343036082E7D5
:105E10000000FFFF2DE9F04F044687B09946BDF81A
:105E200044A0129E0F469046FEF7A6FF94F83D3020
:105E3000202B054609D00227384607B0BDE8F08F71
:105E4000FEF79AFF401B192849D8206883696FEA3A
:105E5000030C1CF0020BF3D094F83C30012BEAD079
:105E600003680122D90784F83C2046D539460768E3
:105E700027F4006707601098606222200195009661
:105E800084F83D00402084F83E0000202064A4F8FF
:105E90002AA0608D20858248E0624B46424620461B
:105EA000FFF78AFD0746A8B9238D22684BBB0290F5
:105EB0005369029393690293029B136843F400733E
:105EC00013600023202284F83D2084F83C3084F8BD
:105ED0003E30B1E70127384607B0BDE8F08F2023F8
:105EE000C4F830B084F83D3084F83EB0236C84F8B8
:105EF0003CB043F0200323649DE703681343036031
:105F0000B4E7012B00F0BC80022B00F082800590EA
:105F10005169059192690592059A032B4DD8012B81
:105F200000F0A180022B5F49009533464FF000023C
:105F300020467DD0FFF752FB02460028CAD12368D5
:105F4000196821F4806119601969636A1970616ABE
:105F5000638D01316162013B218D9BB263854B1ED4
:105F600023855049009533462046FFF737FB00282C
:105F7000B0D12368616A1A6842F400721A601B6922
:105F80000B70638D626A2168013B9BB26385531C71
:105F900009696362238D013B23855170238D628DD6
:105FA000616A013B013A01319BB292B26162238581
:105FB0006285002B85D0032BB1D92A463146204675
:105FC000FFF79EFB002885D12268636A12691A7068
:105FD000628D2068238D616A013A92B262854269BE
:105FE000013B9BB201F1010C52072385C4F824C088
:105FF000DFD503694B70628D238D013A92B26285C1
:10600000626A013B9BB2013223856262002BD2D1CE
:1060100057E7116821F480611160116841F4006153
:10602000116004905169049192690492049A74E792
:10603000FFF7D4FA00287FF44DAF2368616A1A682D
:1060400042F400721A601B690B70638D626A013B37
:106050009BB26385238D013B23852368511C1B69FB
:1060600061625370C7E72A4631462046FFF748FB76
:1060700000287FF42FAF23681A69636A1A70BAE7A1
:10608000116821F480611160039051690391916955
:1060900003910399116841F4007111603DE700BF5D
:1060A0000000FFFF04000100704700BF704700BF01
:1060B000704700BF704700BF704700BF704700BF08
:1060C000704700BF704700BF704700BF704700BFF8
:1060D000806B38B5416B90F83D400368826B5FFA86
:1060E00084FC39B30024CC63EAB11D68D46325F481
:1060F00080651D6044850C65002111651A6822F0D9
:1061000001021A6090F83D20602A28D00CF0280483
:10611000282C17D02022002380F83D2080F83E3024
:10612000FFF7D2FF38BD1C6824F480641C604285F0
:106130000A65E3E7EAB11C68D16324F480641C605B
:106140004185D9E71A6842F001021A601A680021F5
:1061500042F480621A60016380F83D40E0E700236A
:10616000202280F83D2080F83E300364FFF7AEFF28
:1061700038BD196821F4806119604285BEE700BF0F
:1061800090F83D2090F83E100368102910B5D2B267
:1061900004464AD002F02801282941D05968080550
:1061A00038D50022226384F83E205A6812F4006237
:1061B0001FD05A68606B22F400625A6090F8353044
:1061C000012B52D0444B0365FEF7EAFF002869D14A
:1061D000236C190704D02268536823F4E0635360EA
:1061E00094F83D30226C5207DBB201D5282B65D0E4
:1061F00010BD94F83D10602921D05A69500605D58C
:10620000626A1B691370636A013363622046FFF799
:106210005BFFDDE7602AC4D0202284F83D20C0E780
:106220000022226384F83D10BFE7222AB2D11A6807
:1062300022F400621A605A681205B2D4ECE72021F9
:1062400084F83D1022645A69520606D5626A1B69B9
:106250001370626A2368013262621A6822F00102D6
:1062600020461A60FFF732FFB2E7A06B1A4B0365B6
:10627000FEF796FF0028ABD023685A69510606D571
:10628000626A1B691370626A2368013262621A686B
:10629000A06B22F0010220211A60036D84F83D10EA
:1062A000984795E72268606B1368202123F001036B
:1062B0001360036D84F83D10984789E70023074970
:1062C000E16220222363204684F83D2084F83E309A
:1062D000FFF7F4FE10BD00BFD16000080000FFFF13
:1062E00070B5036804465868E56A94F83E1094F85F
:1062F0003D2010298CB0D2B25FFA81FC21D0BCF1D4
:10630000400F1ED0216C002900F0CB805969002578
:1063100011F0020600F08B80860540F18A80226C25
:1063200002B19D6994F83D2002F02802282A00F06D
:1063300027826FF002010022596184F83C200CB0E2
:1063400070BD99695A69D6071AD4B5F52A0FF6D0E7
:10635000B5F12A4FF3D012F0080538D0850539D5AC
:10636000626C616BD2B21A61002900F0F981CA6BCC
:10637000002A00F076825A6842F400625A60DEE732
:10638000860527D5E26AB2F52A0F00F0EE81E26AAF
:10639000B2F12A4F04BF0822E26294F83E20402A5C
:1063A00000F0E6812269B2F5804F00F0FE81226D97
:1063B000002A00F06081226D012AC0D1626CC2F314
:1063C000C81202F0060242F0F1021A61B7E796071E
:1063D00000F13D8111F0040F596865D00905AED474
:1063E000160602F0040140F14F81450540F14C8151
:1063F000002940F04C8194F83D20208D94F83E1007
:10640000E56AD2B2C9B2002840F09A82212A00F08F
:106410008583402993D1222A91D1628D92B2002A9C
:1064200040F0A7835A6822F480625A6087E7CD065D
:1064300063D402F0F702212A01F0040500F0B980CC
:106440004E0640F1F580410540F1F280002D40F00C
:10645000F28094F83D10628D92B2C9B2002A3FF4E6
:106460006EAF626A1B691370638D626A013B9BB2F7
:106470006385638D01329BB26262002B7FF45FAF54
:106480002A297FF45CAF226853682225282123F44F
:10649000806353602046256384F83D10FFF70AFEB1
:1064A0004DE79D69596933E709053FF548AF560641
:1064B00002F0040100F1FF8000293FF440AF8205A3
:1064C0007FF53DAFE06A628D616A92B2042A00F006
:1064D0000E82628D92B2032A00F04482628D92B2E3
:1064E000022A00F08D821B690B70638D626A013B8A
:1064F00001329BB26262638521E7850599D594F8E4
:106500003D505A6822F4E0625A600B965A690B9229
:106510001A6842F001021A600B9A1A6822F480622B
:106520001A605A681005EDB200F1EA80638D9BB2E3
:1065300013B323685A6951070AD5626A1B6913703D
:10654000628D636A013A591C92B223686162628566
:106550005A69520609D5626A1B691370638D626AB3
:10656000013B01329BB262626385638D9BB21BB1BA
:10657000236C43F004032364236C002B40F0EA8077
:106580002A2D00F07D8194F83D30282B00F06B819E
:10659000236B222B02D0222D7FF4D1AE00232022A8
:1065A0002363204684F83D2084F83E30FFF782FDC7
:1065B000C5E60E0627D5410525D53DBB94F83D001F
:1065C000618D89B2C0B200293FF4B9AE616A11F899
:1065D000015B1D616162618D013989B26185618DE7
:1065E00089B200297FF4ABAE29287FF4A8AE5968A0
:1065F000282521F4806159602046226384F83D50AB
:10660000FFF756FD9BE6002D3FF499AE82057FF51E
:1066100096AE628D92B2002A3FF491AE626A12F891
:10662000011B1961638D6262013B9BB2638586E643
:10663000002D3FF484AE82057FF581AE628D92B26B
:10664000002A3FF47CAE626A1B6913704DE7860531
:106650007FF5C0AE94F83E20E06A266B94F83D10BA
:106660002229D2B200F0E2800A955A690A929B6907
:106670000A930A9B63E6626CC2F3C81202F0060238
:1066800042F0F0021A615AE600293FF458AE800544
:106690007FF555AEE16A94F83D20212A00F02E8165
:1066A00094F83E30402B7FF44AAE20460CB0BDE853
:1066B0007040FFF755B845057FF5FEAE00297FF421
:1066C000FEAE94F83D20222A7FF439AE628D92B25C
:1066D000032A40F2FB81626A1B691370638D626A50
:1066E000013B9BB26385638D9BB20132032B6262D7
:1066F0007FF425AE2268536823F4806353601EE65E
:1067000005F0F702222A70D0606B0268526892B2DC
:106710006285628D92B21AB1226C42F00402226448
:106720005A6822F400625A60FEF722FE012808D05F
:10673000606B944B0365FEF733FD10B1606B036D26
:106740009847638D9BB2002B7FF4F3AE236C002B34
:106750003FF419AF20460CB0BDE87040FFF710BD04
:10676000A26B002A7FF403AEE9E50122E26214E69F
:10677000226D002A33D1626C02F0FE021A61DEE55E
:106780005A682E0622F480625A60C5F3800154BF15
:10679000E268A269002381F00101C9B284F83C30AB
:1067A00092B22046FFF788FCC9E594F83D20212AE3
:1067B000626C16BF42F0010202F0FE02D2B21A6110
:1067C000626B1AB1D26B002A7FF4D5ADA26B002A9E
:1067D0003FF4B5ADD26B002A7FF4CDADAFE5626C6E
:1067E00042F00102D2B21A61A9E5A06B02685268B8
:1067F00092B26285628D92B21AB1226C42F00402AA
:1068000022645A6822F400625A60FEF7B1FD012842
:106810003FF48CAEA06B5B4B0365FEF7C1FC002818
:106820003FF484AEA06B036D98477FE6216D09B9F4
:10683000402A7ED0226D22B92169B1F5404F00F087
:106840008380628D92B25ABB03925A6903929A690D
:106850000392039A1A6842F400721A6000232365B7
:106860006DE5A26BB6E700234749E162202223636E
:10687000204684F83D2084F83E30FFF71FFC5EE59B
:1068800028222363204684F83D20FFF713FC94F868
:106890003D30282BE7D0236B222B7FF450AD7DE6D3
:1068A000628D92B2012A73D0628D92B2022A00F0F8
:1068B000EA801A6842F480621A605A6815050ED59B
:1068C000202800F28881072840F281812F4A083869
:1068D000C240D00703D55A6842F480525A60002261
:1068E00009925A6909929B690993099BB6E75A680C
:1068F00022F480625A601B690B70F6E5628D92B2D9
:10690000002A7FF48BAE082963D0202961D011F5CD
:10691000803F5ED0596821F4E06159601120202346
:10692000206384F83E20204684F83D30FFF7BCFB0E
:1069300005E501915A6901929B690193019BFEE46F
:10694000212A7FF466AD68E502925A6902929A693B
:106950000292029A1A6842F480721A60236D01331F
:106960002365ECE45A68042822F480625A603FF4FC
:10697000BAAD02283FF4B7AD1A6822F480621A60FB
:10698000B1E500BFD16000080000FFFF0101000178
:1069900010F5803F00F0F380082800F0DA8020280E
:1069A00000F0D780122E00F02A81102800F22981F1
:1069B000964A0241D60700F124811A6842F48062A7
:1069C0001A60002206925A6906929B690693069BFA
:1069D00044E7596821F4E0615960196800222020D9
:1069E00041F400711960226384F83D0094F83E3050
:1069F00084F83E20402B204698D1FFF761FB9EE4AF
:106A000001380F2809D8DFE800F0393408340808C5
:106A1000080808080808080808391A6842F40072CB
:106A20001A601B690B70638D626A2168013B9BB21F
:106A300063850B69511C61625370638D2168626AC2
:106A4000013B9BB263854B68013223F440732020E5
:106A500062624B6084F83D0094F83E30402B55D084
:106A60000022122384F83E2020462363FFF71EFBFA
:106A700065E41A6842F480621A60D2E71A6822F468
:106A800080621A60CDE7102800F28D80604AC24013
:106A9000D50740F188801A6842F480621A605A680B
:106AA00012050BD5072840F2A6805A4A0838C24082
:106AB000D60703D55A6842F480525A6000220892E1
:106AC0005A6908929B690893089BC7E6E16A022904
:106AD0003FF435AC012A3FF632AC1A68606A22F402
:106AE00080621A605A6822F4E0625A601B6903707F
:106AF000638D626A013B9BB22021638584F83D105F
:106B000094F83E300132402B6262A9D1002384F810
:106B10003E3020462363FFF7D5FA10E4082D3FF4FA
:106B200058AF202D3FF455AF15F5803F3FF451AFDE
:106B30005A6822F4E0625A60112000212023206369
:106B400084F83E10204684F83D30FFF7ADFAFFF799
:106B5000F6BB1A68002122F480621A6007915A6914
:106B600007929A690792079A1A6842F400721A60AB
:106B700074E694F83E20402A7FF450AD95E51A68FB
:106B800022F480621A605A6812F4006228D01A68EF
:106B9000002122F480621A6004915A6904929B6970
:106BA0000493049B5AE61A6822F480621A601A68F9
:106BB00042F400621A605A6811057FF57FAF202801
:106BC0007FF670AF10F5803F7FF478AF72E7012851
:106BD0007FF485AE7FE610F5803F7FF480AE7AE6E5
:106BE00005925A6905929A690592059A1A6842F4C3
:106BF00000721A6032E601287FF460AF5AE701287C
:106C0000A7D11A6822F480621A60DAE6EBFFFEFF71
:106C10001400010001010001F0B503685C695968C6
:106C200090F83E20E60583B0D2B204F400750CD58E
:106C3000CF0504F480660BD56FF480715961002D87
:106C40003FD1002E6DD0012508E01DB1C9051BD430
:106C500003B0F0BD66052ED5C905F9D5418D90F874
:106C60003D60076B202A89B2F6B237D06FF480619D
:106C7000102A596145F0040127D0402A25D0270564
:106C800021D541F008050BE0022504F480666FF47D
:106C900000715961002EE1D1270504D545F00805A2
:106CA0006FF400625A61036C2B43036403B0BDE8C8
:106CB000F040FFF765BA2405CAD5CA05C8D508252E
:106CC000EEE70325E3E70D46EDE71A68260542F4F3
:106CD00000721A60F7D545F00C05E1E7D9B906F066
:106CE000F702212A03D0282E15D1212F13D190F895
:106CF0003D20C16A0829D2B219D0202917D0212AF3
:106D000004F4006434D06FF480625A61002CC5D161
:106D1000002DC8D19CE76FF480625A6145F00401F0
:106D2000ADE7250501D50925BAE70125BBE7282AE6
:106D3000E5D11E4AC2625A68019022F4E0625A60AC
:106D40006FF480625A611A6822F480621A6000232C
:106D50002022036380F83D2080F83E30FFF7AEF933
:106D600014F4006F0198D3D0036845F0080597E745
:106D70000E49C1620263202280F83D20002280F883
:106D80003E205A68019022F4E0625A606FF48062FB
:106D90005A611A6822F480621A60FFF789F9019833
:106DA000002CE1D1002D7FF47EAF51E70000FFFF02
:106DB00090F83D00704700BF10B40D4C0D4A236899
:106DC00023F00303034323601369012943F0040301
:106DD00013610AD040BF20BF20BF064A5DF8044BB4
:106DE000136923F004031361704730BFF5E700BF58
:106DF0000070004000ED00E04B6A2DE9F04133B136
:106E0000B2F1406F03D08C6A0568013C2C618C693B
:106E10000E6AD1F81C804CB343EA040C4B6900683D
:106E2000CF6A0D6B4C6B4FEA834E4CEA020C0B6839
:106E3000002E4CD04CEA060C8E68C6610E69B8F183
:106E4000000F4DD043EA08033B432B432343334316
:106E5000CC68234343EA0E0343EA0C03B2F1406FCC
:106E6000436146D04B688361BDE8F081F6B14C695F
:106E70000068CF6A4D6B43EA060C8B68C3610E6BEA
:106E80000B694CEA020CA404B8F1000F3DD043EAB0
:106E900008033B4333432B43CD682B43234343EA4F
:106EA0000C03B2F1406F4361DCD122E0B8F1000F76
:106EB00034D1F3B1CC6A006823430C6B13432343F2
:106EC0004C6B4A69234343EA8243436111E0B8F1C2
:106ED000000F10D043EA08033B432B432343B7E79B
:106EE0003B432B432343334343EA0E0343EA0C0360
:106EF0004361BDE8F0813B432B43234343EA0E0348
:106F000043EA0C034361BDE8F0813B4333432B4329
:106F1000234343EA0C034361BDE8F081CC6A006877
:106F200043EA0803134323430C6B23434C6B234373
:106F3000CC6823434C69B2F1406F43EA8443436118
:106F400090D1D6E7704700BF70B50446FDF714FF37
:106F50000546002C59D094F8413003F0FF02002B75
:106F600049D0A66C2268A1681368013923F4F8534C
:106F700043EA0123136093689B060CD5711C33D040
:106F8000FDF7FAFE401BB04241D8002E3FD02268E8
:106F900093689806F4D4E569E368116860682B4348
:106FA000256A21F07F412B4343EA006321F0D001A1
:106FB0000B431360A5696369506819492B43256920
:106FC000014043EA05430B4353601368002143F03B
:106FD00001034FF0010C13600846616484F841C05E
:106FE000002384F8403070BD93689B06D3D5936826
:106FF0009B06F9D4CFE784F840202046FFF7A2FF94
:1070000041F288331E46A364ACE7012070BD04231F
:1070100084F84130636C012003436364E0E700BF00
:10702000FEF8E0FF704700BF10B5044670B102687B
:10703000136823F001031360FFF7F4FF0023636478
:10704000184684F8413084F8403010BD012010BD4E
:107050002DE9F84304460D461746FDF78DFE94F8DA
:107060004030012B804638D0012384F8403094F81A
:107070004130012B5FFA83F907D04FF0020900235A
:1070800084F840304846BDE8F883002363642668EE
:10709000022384F84130B368980611D57A1C0CD0CD
:1070A000FDF76AFEA0EB0800874237D3002F35D0EA
:1070B0002668B3689906F3D402E0B3689B06FCD453
:1070C000002229462046FFF797FE6B6A53B1012341
:1070D00084F841304FF00009D1E74FF002094846EB
:1070E000BDE8F883B368990710D47A1C0BD0FDF77C
:1070F00043FEA0EB08039F4210D37FB12668B3681C
:10710000980703D4F3E7B3689B07FCD50222012359
:10711000F2604FF0000984F84130B0E7042384F8AE
:107120004130636C43F001036364A8E72DE9F84F35
:1071300081461E468A469346FDF71EFE99F840306A
:10714000012B074666D0012389F8403099F8413079
:10715000012B5FFA83F807D04FF00208002389F86B
:1071600040304046BDE8F88F0023C9F84430D9F8D4
:107170000040422389F84130A368990611D5731C59
:107180000CD0FDF7F9FDC01B864248D3002E46D037
:10719000D9F80040A3689A06F3D402E0A3689D06DC
:1071A000FCD4DBF80030A362DBF804306362DBF868
:1071B0000830E3622568DBF8103025F4400C4CEA17
:1071C000030C4CF48002DBF80C3022604846CAF80D
:1071D00028304FF000625146FFF70EFEA3681807F3
:1071E00010D4721C0BD0FDF7C7FDC01B864216D30E
:1071F000AEB1D9F80040A368190703D4F3E7A36838
:107200001B07FCD508220123E2604FF0000889F833
:107210004130A3E74FF002084046BDE8F88F042351
:1072200089F84130D9F8443043F00103C9F84430BB
:1072300094E700BF70B50446FDF79EFD94F8413019
:107240009907054638D50022236884F840201A683B
:1072500052073AD41A6842F002021A609A689607F6
:107260000DD4A66C711C29D0FDF786FD401B86420B
:107270003AD3002E38D023689A689007F4D50222BA
:10728000DA609A68920610D5A66C711C0AD0FDF7D8
:1072900073FD401B864227D336B323689A68900655
:1072A000F5D402E09A689206FCD45A69012122F0D2
:1072B00040625A6184F84110002070BD9A689607B8
:1072C000DDD49A689607DAD4F8E71A68E06B22F002
:1072D00004021A60FDF71CFF23680028BAD0626C14
:1072E00042F004026264B5E7042384F84130636C21
:1072F00043F001036364012070BD00BF2DE9F84332
:10730000044689461546FDF737FD94F84030D4F819
:107310000080012B064664D0012384F8403094F8A5
:107320004130012BDFB206D00227002384F8403021
:107330003846BDE8F88300236364B9F1000F5CD0E0
:10734000122384F84130D8F810300133E362D8F8C2
:107350001030C4F824900133A362D8F8143023F01D
:107360004063C8F81430E36A42460BB393685B0786
:1073700010D4681C0BD0FDF7FFFC801B854234D372
:10738000002D32D023689B685A0703D4F3E7936833
:107390005907FCD5636A1B7888F82030E16A636A74
:1073A00022680139E162E16A013363620029DDD1BB
:1073B000936898070BD4691C24D0FDF7DDFC831B70
:1073C0009D4212D38DB1226893689B07F5D50223A5
:1073D000D3602046FFF72EFF0746012384F8413093
:1073E000A3E702273846BDE8F883042384F8413038
:1073F000636C43F001036364EFE7636C43F00803DD
:10740000636492E793689B07E1D493689B07F9D57F
:10741000DDE700BF2DE9F843044615468946FDF730
:10742000ABFCD4F80080D8F8182094F84030012B39
:1074300006466BD0012384F8403094F84130012B8C
:10744000DFB206D00227002384F840303846BDE87A
:10745000F88300236364B9F1000F63D0222384F81A
:107460004130D8F810300133A363D8F81030C4F895
:10747000309001336363D8F8143023F0406343F055
:107480008063C8F81430C8F81820A36B424623B3B1
:10749000936813F0060F12D1691C0CD0FDF76CFC39
:1074A000801B854236D3002D34D023689B6813F0AF
:1074B000060F04D1F2E7936813F0060FFBD0236B9D
:1074C00098F820201A70A16B236B22680139A16300
:1074D000A16B013323630029DAD1936898070BD499
:1074E000691C24D0FDF748FC831B9D4212D38DB14B
:1074F000226893689B07F5D50223D3602046FFF7E7
:1075000099FE0746012384F841309CE7022738465C
:10751000BDE8F883042384F84130636C43F0010331
:107520006364EFE7636C43F0080363648BE793687D
:107530009B07E1D493689B07F9D5DDE770B5244E2E
:1075400088B00D461446F8B90090336B43F0010340
:107550003363336B069003F0010300934FF48072A2
:107560000223CDE902231B480022032302A9CDE90F
:107570000423009BFDF700FFB36823F0EC632B436B
:107580002343B36008B070BD00220192336B1248F0
:1075900043F004033363336B069203F00403019357
:1075A0004FF400720223CDE9022302A90022032333
:1075B000CDE90423019BFDF7DFFEB36823F0784398
:1075C00043EA050141EAC401B16008B070BD00BFE3
:1075D000003802400000024000080240014B012236
:1075E000DA64704700004742164908B58B6803F01B
:1075F0000C03042B1BD0082B01D0134808BD4A688C
:107600004B68496813F4800302F03F0211D10E4821
:10761000C1F38811A1FB000110F050F8094B5B6821
:10762000C3F3014301335B00B0FBF3F008BD07482F
:1076300008BD0648C1F388110023A1FB000110F02A
:107640003DF8EBE7003802400024F40000127A0015
:107650002DE9F0410D46044660B1454A136803F038
:107660000F038B4209D2CBB21370136803F00F03E0
:107670008B4202D00120BDE8F0812368980714D521
:10768000590704D53B498A6842F4E0528A601A07D8
:1076900004D538498A6842F460428A603549A06856
:1076A0008A6822F0F00202438A60DF0721D562680F
:1076B000012A55D0931E012B2E4B1B684DD99907DB
:1076C000D8D52C4EB36823F003031343B360FDF702
:1076D00053FB41F28838074604E0FDF74DFBC01B21
:1076E000404542D8B368626803F00C03B3EB820FE5
:1076F000F3D11F4A136803F00F03AB4206D9EBB274
:107700001370136803F00F03AB42B3D123685A0719
:1077100006D51849E0688A6822F4E05202438A607C
:107720001B0707D5134A2169936823F4604343EA92
:10773000C1039360FFF758FF0E4A0F4C92680F4940
:10774000C2F303120346A25C0D48D34000680B60ED
:10775000FDF7E2FA0020BDE8F0819801B1D489E795
:10776000044B1B689E03ACD484E7032083E700BF6F
:10777000003C024000380240D0CC0108C400002088
:10778000C0000020014B1868704700BFC4000020F3
:10779000044B05499B68054A0868C3F38223D35C00
:1077A000D840704700380240C4000020C8CC01080F
:1077B000044B05499B68054A0868C3F34233D35C10
:1077C000D840704700380240C4000020C8CC0108EF
:1077D0000E4B0F2210B402609A680D4C02F00302A7
:1077E00042609A6802F0F00282609A6802F4E05205
:1077F000C2609B68DB0803F4E053036123685DF813
:10780000044B03F00F030B60704700BF00380240C9
:10781000003C02402DE9F041036813F0010582B0FD
:1078200004460BD0A4494569D1F88C2022F0C062EF
:107830002A43B5FA85F5C1F88C206D099E070CD551
:107840009D48A169D0F88C2022F0C0520A43C0F8AC
:107850008C20002908BF45F00105180700F19F8022
:107860005F0705D5954B94F83820C3F8E0212368CD
:10787000DE0608D59049606AD1F8942022F44002CF
:107880000243C1F89420980603F0400134D58A4899
:10789000A66AD0F8942022F000623243B6F1006F5D
:1078A000C0F8942000F0E180002900F0C0808249F7
:1078B000206AD1F8942022F080520243012DC1F8B1
:1078C00094201FD0DA0508D57B49E06AD1F88C20D6
:1078D00022F000420243C1F88C209B0508D5764A6D
:1078E000216BD2F88C3023F400430B43C2F88C3068
:1078F000002002B0BDE8F0810029D8D1012D01D0CF
:10790000802BDFD16E4B6C4E00229A66FDF734FA65
:10791000054604E0FDF730FA431B022B3BD83368E1
:107920001A01F7D4654B626BC3F8D8202268D307DD
:1079300040F181806369002B7DD1E368A0686168B4
:107940001B0643EA801320690B435B4943EA00733B
:10795000C1F8843010060CD5E368A068626821691C
:107960001B0643EA80131343534A43EA0173C2F8E8
:107970008430534B504E01229A66FDF7FDF90546BF
:1079800004E0FDF7F9F9401B022804D83368190117
:10799000F7D5236896E7032002B0BDE8F081464B97
:1079A000484E002201921A6C42F080521A641B6CFD
:1079B00003F080530193019B336843F48073336079
:1079C000FDF7DAF9074604E0FDF7D6F9C31B022BF1
:1079D000E1D83368D905F7D5374EE369326F12F431
:1079E000407203F4407112D08A4210D0336F344A8F
:1079F0000121C2F8401E23F440730021C2F8401E4A
:107A00003367336FDA0747D4E36903F44071B1F5A4
:107A1000407F36D028498A6822F4F8128A60264AC4
:107A2000116FC3F30B030B431367236818E7012D92
:107A30007FF448AF66E7970703D5A369002B3FF4AF
:107A40007CAF960604D5A36AB3F1006F3FF475AF1F
:107A500055067FF57FAF236A002B7FF47BAFA36AC7
:107A6000B3F1006F7FF476AF67E700293FF44AAFC8
:107A7000D0F89430226A23F080531343C0F8943036
:107A800040E70D48826823F0704122F4F81221F497
:107A900040710A438260C2E7FDF76EF941F288380F
:107AA000074605E0FDF768F9C01B40453FF673AF98
:107AB000336F9B07F6D5A7E7003802400010474216
:107AC00000004742007000402DE9F0410368DD07E7
:107AD00082B004462FD59F498A6802F00C02042A1E
:107AE00000F0C2808A6802F00C02082A00F0B88018
:107AF0006368B3F5803F00F0F980B3F5A02F00F084
:107B00004C81944D2A6822F480322A602A6822F43B
:107B100080222A60002B40F0EE80FDF72DF906460A
:107B200005E0FDF729F9801B642800F202812B682B
:107B30009B03F6D423689F0728D5864A916811F0E5
:107B40000C0F00F09F80916801F00C01082900F0F3
:107B50009580E368002B00F00F817F4B7D4E012262
:107B60001A60FDF709F9054605E0FDF705F9401B28
:107B7000022800F2DE8033689807F6D53368226960
:107B800023F0F80343EAC203336023681A0716D5CB
:107B90006369002B00F081806F4B6E4E0122C3F8A9
:107BA000802EFDF7E9F8054605E0FDF7E5F8401BF6
:107BB000022800F2BE80736F9B07F6D52368580732
:107BC0002FD5644A136C13F0805377D00025634E91
:107BD0003368D90540F19D80A368012B00F0AD808A
:107BE000052B00F019815B4E326F22F001023267E3
:107BF000326F22F004023267002B40F0A380FDF7C1
:107C0000BBF841F28838074605E0FDF7B5F8C01B20
:107C1000404500F28E80336F9807F6D4002D40F077
:107C2000C680A369C3B14B4DAA6802F00C02082AB2
:107C30002FD0022B484B4FF000021A6600F0BD8097
:107C4000FDF79AF8044604E0FDF796F8001B0228B9
:107C50006FD82B689B01F7D4002002B0BDE8F081FB
:107C60004A6850027FF544AF3A4A126891037FF5A3
:107C700062AF6268002A7FF45EAF0AE05268560283
:107C80003FF567AF334A1268950723D5E268012AAA
:107C900020D0012002B0BDE8F0812F4A2D4EC2F85D
:107CA000803EFDF769F8054604E0FDF765F8401BE6
:107CB00002283ED8736F9F07F7D47FE70193136CB8
:107CC00043F080531364136C03F080530193019BC2
:107CD00001257CE71F4920690A6822F0F80242EA80
:107CE000C0020A601A077FF56AAF51E7194A1368A4
:107CF00043F480331360FDF73FF8164E054604E069
:107D0000FDF73AF8401B642813D833689A03F7D577
:107D100010E7336843F480733360FDF72DF80746AE
:107D20003368DA053FF558AFFDF726F8C01B022887
:107D3000F6D9032002B0BDE8F081064A136F43F084
:107D400001031367FDF718F8024F064641F2883821
:107D50000BE000BF003802400000474200700040C6
:107D6000FDF70AF8801B4045E3D83B6F9B07F7D52A
:107D7000002D3FF456AF1AE02C4A2D4E1360FCF74D
:107D8000FBFF054604E0FCF7F7FF401B0228D0D8B4
:107D900033689907F7D42368F8E6254B1A6842F44C
:107DA00080221A601A6842F480321A60A3E7204ADF
:107DB000136C23F08053136433E7FCF7DDFF0646B2
:107DC00004E0FCF7D9FF801B0228B2D82B68990188
:107DD000F7D4216AE369626AE06A0B4343EA8213DB
:107DE000A26A216B43EA0063520843EA0173013A35
:107DF0000E4943EA024301226B600A66FCF7BCFFAE
:107E00000B4D044604E0FCF7B7FF001B022890D896
:107E10002B689A01F7D51FE7054B1A6F42F0040251
:107E20001A671A6F42F001021A678BE70000474297
:107E300000380240704700BF10B50446A0B1437936
:107E400003F0FF0263B12168022363710B68002213
:107E500043F0040301200B6060711046A26010BD66
:107E60000271FFF7E7FFEEE7012010BD704700BF8A
:107E700038B50446002860D0437F03F0FF02002B92
:107E80005DD0236853220220CA21607759625A626A
:107E9000DA6855063CD599686268256921F4E001E5
:107EA00021F040019960616998682A430A430243BE
:107EB000E1689A6019611A69A16842EA01421A618F
:107EC000DA6822F08002DA609A6891060DD51A6CA1
:107ED000A06922F480221A641A6C02431A64FF21FA
:107EE000012259620020627738BDDA6822F0A002D0
:107EF000DA60FCF741FF054605E0FCF73DFF401B5B
:107F0000B0F57A7F14D82368DA689206F5D5DEE7F3
:107F10004FF0FF32DA60FCF72FFF05462368DA687E
:107F20005006B8D4FCF728FF401BB0F57A7FF5D98E
:107F30002268FF21042351626377012038BD027754
:107F4000FFF794FF9DE700BF0368503343F82120FB
:107F5000704700BF0368503353F82100704700BFDB
:107F60002DE9F04106689846B36831EA03030CBF77
:107F700001230023934207460C4615460AD0B8F168
:107F8000FF3F12D1B36834EA03030CBF012300237F
:107F9000AB42F7D10020BDE8F0819B6834EA0303CF
:107FA0000CBF01230023AB42F4D0FCF7E5FE069B97
:107FB000C01A40453B68F0D379685A68B1F5827FB2
:107FC00022F0E0025A6013D0BA6AB2F5005F07D11E
:107FD0001A6822F400521A601A6842F400521A60B9
:107FE0000122002387F8512087F850300320D2E780
:107FF000BA68B2F5004F02D0B2F5806FE4D11A68CA
:1080000022F040021A60DFE730B5174B174D1B68AE
:10801000A5FB035C85B04FEA5C5C4FF47A7303FB0D
:108020000CF303934368B3F5827F044607D10CE059
:10803000039B2268013B039393681B0602D5039BB5
:10804000002BF5D1002005B030BD00920B46002278
:108050008021FFF785FF0028F4D0636D43F02003F3
:1080600003206365EFE700BFC4000020819F5E1618
:1080700030B50B4611464268B2F5827F83B00446A4
:1080800008D0009100220121FFF76AFF88B9002083
:1080900003B030BD8268B2F5004F1ED0B2F5806FDC
:1080A0000ED00091002280212046FFF759FF0028C2
:1080B000EDD0636D032043F02003636503B030BD52
:1080C00005682A6822F040022A60009100220121FE
:1080D000FFF746FF0028DAD0EBE70068026822F0DD
:1080E00040020260DDE700BF704700BF70B5044684
:1080F00000283BD090F8513003F0FF02002B30D025
:1081000004F1080007C86368666A03430B436169AA
:10811000E06913430B432268216A022584F8515019
:1081200003430B431168A069A56A21F04001116067
:108130002B43010C00F400700343136001F00403AF
:108140003343B5F5005F536004BFE36A1361D3693D
:10815000002023F400630121D361606584F851108D
:1081600070BD80F85020FFF7BFFFC9E7012070BD48
:1081700090F85030012B70B504465ED090F8513025
:108180000120834284F85000DDB205D0022500238F
:1081900084F85030284670BD0029F8D0002AF6D067
:1081A000032384F8513000236365A363E28663648C
:1081B0002364A387E387A368A286B3F5004F2268F0
:1081C000216335D0A36AB3F5005F28D0A06C1C4EA4
:1081D000E38E06641B4EC6631B4EC66400260C323B
:1081E0009BB20665FCF758FF88B923681A685206E7
:1081F00003D41A6842F040021A605A6842F0200222
:108200005A605A6842F0020200255A60BFE7636D67
:10821000012243F01003636584F85120B7E7136827
:1082200023F400531360136843F400531360CDE745
:10823000136843F480431360C4E70225284670BDE9
:1082400079830008CD830008A983000838B5044667
:1082500090F8500001287ED0012084F8500094F856
:10826000510001285FFA80FC0ED06068B0F5827F73
:1082700004D00220002384F8503038BDA0680028C4
:10828000F7D1BCF1040FF4D1002962D0002A60D0EC
:10829000002B5ED094F85100A38604281CBF052053
:1082A00084F8510000206065A387E386E387A36A12
:1082B0002163B3F5005F2168A2632064606407D185
:1082C0000B6823F400530B600B6843F400530B60FE
:1082D00094F85130E06C042B14BF204B204BC36347
:1082E000204BC3644FF000030365E38F14BF1E4DA2
:1082F0001E4D05640C319BB2FCF7CEFE014608BB57
:108300002268A06C536843F001035360E38E01645C
:10831000C163C16401659BB2216B0C32FCF7BCFEEA
:1083200080B923681A68520603D41A6842F04002E2
:108330001A605A6842F020025A605A6842F00202FB
:108340005A6097E7636D012243F01003636584F878
:10835000512001208EE7022038BD00BFF1840008C3
:108360003D840008A98300089983000889830008D8
:10837000704700BF704700BF08B5806BFFF7FAFF7A
:1083800008BD00BF704700BF08B5806BFFF7FAFF5C
:1083900008BD00BF704700BF08B5806BFFF7FAFF4C
:1083A00008BD00BF704700BF806B026808B5536806
:1083B00023F003035360436D012143F01003436531
:1083C00080F85110FFF7EEFF08BD00BF30B505463D
:1083D00083B0846BFCF7D0FC2B681B68DB0502467E
:1083E00021D42368586820F020005860586820F095
:1083F0000200586064212046FFF706FE18B1636D45
:1084000043F020036365A36833B922680193D368FE
:10841000019393680193019B01230022E28684F873
:108420005130636D23B92046F9F7D8FC03B030BD55
:108430002046FFF7B7FF03B030BD00BF70B505465B
:1084400082B0846BFCF798FC2B681B68D905064644
:1084500021D42368A16A5A68B1F5005F22F0200296
:108460005A6035D0A26852B35A6822F001025A60AD
:10847000324664212046FFF7FBFD08B120236365E7
:10848000012223680021E18784F851209A68D206EE
:1084900006D4636D73B92046FFF76AFF02B070BD62
:1084A000626D4FF6EF7142F0020262659960636D92
:1084B000002BF0D02046FFF775FF02B070BD626858
:1084C000B2F5827FD0D15A6822F003025A60CFE71A
:1084D00001220090642311462046FFF741FD18B1A8
:1084E000636D43F0020363652368DA68BAE700BF8F
:1084F00070B5054682B0846BFCF73EFC2B681B68A8
:10850000D905064622D42168A26A4B68B2F5005FFD
:1085100023F020034B602DD0324664212046FFF724
:1085200073FD18B1636D43F02003636523685A68D7
:10853000002122F0030201205A60E186E18784F8DD
:1085400051009A68D20606D4636D73B92046F9F7D4
:108550005FFC02B070BD626D4FF6EF7142F0020237
:1085600062659960636D002BF0D02046FFF71AFF1B
:1085700002B070BD01220090642311462046FFF72F
:10858000EFFC18B1636D43F0020363652368DB6899
:10859000C2E700BF30B502685168936813F0400F1E
:1085A00085B00446C3F3801519D113F0010F2FD104
:1085B000980745D49D0600F19180DB050DD58D0609
:1085C0000BD5636D002043F0080363650390936847
:1085D0000393039B636D002B5AD105B030BD13F09C
:1085E00002001AD008067CD413F020002CD18D068E
:1085F000F3D594F85150032D79D0656D45F00405FD
:1086000065650090D06800909068009000983AE00E
:1086100011F0400FCCD0036C65E08D06DDD594F8E9
:108620005150032D63D0656D45F0040565650090DC
:10863000D0680090906800900098980623D515E0C7
:1086400008064ED49806B8D58806C6D575B194F8F4
:10865000510003284BD0606D40F00400606500209D
:108660000090D0680090906800900098606D40F095
:10867000010060650020029090680290106820F070
:10868000400010600298DB059BD4636D002BA4D0E2
:108690005368012023F0E0038D07536084F85100F4
:1086A0002DD05368E06C23F00303536040B1164BA8
:1086B0000365FCF775FD18B1636D43F04003636516
:1086C000A06C002889D0104B0365FCF769FD0028D9
:1086D00083D0636D43F0400363657EE78806C5D4AD
:1086E0007BE7636C204605B0BDE8304018470023A7
:1086F0000193D368019393680193019B6DE7204632
:10870000FFF750FE69E700BF0D87000808B5806BD2
:108710000023C387C386FFF745FE08BD704700BF2F
:1087200070B50E461546044618B390F8493003F06C
:10873000FF02CBB1214651F8080B00F053FBA268B1
:108740002068314600F08CFB236BA26860682946E4
:1087500000F0B2FB2268A16852F8213043F0010317
:1087600042F82130002070BD80F84820FFF7D6FF86
:10877000E0E7012070BD00BF704700BF0368DA6802
:1087800042F00102DA609A6802F00702062A03D07A
:108790001A6842F001021A60002070470368DA6824
:1087A00022F00102DA601A6A41F211110A4208D17C
:1087B000196A40F24442114203D11A6822F00102C0
:1087C0001A600020704700BF704700BF704700BFAD
:1087D000704700BF704700BF704700BF03681A6949
:1087E000910710B5044602D5DA6892075FD41A697A
:1087F000500702D5DA68510746D41A69120702D524
:10880000DA6810072ED41A69D20602D5DA68D006C3
:1088100018D41A69D10702D5DA68D2075DD41A696B
:10882000100602D5DA6811065FD41A69520602D51D
:10883000DA68500661D41A69910602D5DA689206A0
:1088400043D410BD6FF010021A61DB69082213F4E3
:10885000407F2277204664D0FFF7BAFF00222368CA
:108860002277D6E76FF008021A61DB6904229907C4
:108870002277204652D1FFF7A9FF2046FFF7AAFF33
:10888000002223682277BEE76FF004021A619B6919
:10889000022213F4407F227720463CD1FFF796FF57
:1088A0002046FFF797FF002223682277A5E76FF0A5
:1088B00002021A619B6901229B07027725D0FFF70C
:1088C00087FF00222368227791E76FF0200220467D
:1088D0001A61BDE8104000F0B7B86FF001021A61EC
:1088E0002046FFF771FF236899E76FF080021A6155
:1088F000204600F0ABF8236897E76FF040021A615A
:108900002046FFF769FF236895E7FFF75FFF2046E2
:10891000FFF760FFD5E7FFF75BFFC4E7FFF758FFFE
:10892000AEE7FFF753FF2046FFF754FF96E700BF7F
:10893000354A0368904210B44DD0B0F1804F34D026
:10894000A2F57C42904230D002F5806290422CD059
:1089500002F58062904228D002F5784290423AD0E7
:108960002A4A904225D002F58062904221D002F539
:10897000806290421DD0A2F59832904219D002F543
:108980008062904215D002F58062904211D08C68CE
:108990000A68496923F080030B4303600123C46222
:1089A00082625DF8044B436170474A6823F07003AC
:1089B0001343CC684A6923F44073234323F08003B4
:1089C00013438C680A6803600123C46282625DF805
:1089D000044B436170474C68CA6823F0700323431B
:1089E00023F4407313434A695DF8044B23F080037A
:1089F000134303608B68C3620B6883620B69036374
:108A000001234361704700BF000001400040014066
:108A100010B50446B0B190F83D3003F0FF0263B1E9
:108A20002146022351F8040B84F83D30FFF780FF04
:108A30000123002084F83D3010BD80F83C20FFF772
:108A40009BFEEDE7012010BD704700BF704700BFDF
:108A50000268116938B50446C068A368256921F425
:108A6000405101431161D168E0692B43656921F4EC
:108A700016412B4321F00C0103430B43D360536990
:108A8000A16923F440730B43B0F5004F5361284BA9
:108A900023D09A421ED003F580639A421AD0FEF783
:108AA00077FE636819219A00A0FB01019B0F0EF06D
:108AB00005FE204AA2FB00135B092168642404FB25
:108AC000130000013230A2FB00201B0103EB501306
:108AD0008B6038BDFEF76CFEE3E79A4225D003F5C4
:108AE00080639A4221D0FEF753FE626819219218E2
:108AF0004FF000035B41A0FB01010EF0DFFD0D4ACA
:108B00002468A2FB00314909642303FB1103DB0045
:108B10003233A2FB0323C3F342121B0902EB0112FF
:108B200003F4F8731344A36038BDFEF741FEDCE79D
:108B3000001001401F85EB51704700BF38B5044657
:108B400050B390F8393003F0FF0203B322682423B6
:108B500084F83930D36823F400532046D360FFF7FC
:108B600077FF23681A6922F490421A615A6922F049
:108B70002A025A61DA680025202142F40052DA60A4
:108B80002846E56384F8391084F83A1038BD80F837
:108B90003820FFF7D1FFD9E7012038BD704700BF6B
:108BA000704700BF90F83A30222B10B522D181686F
:108BB00002690468836AB1F5805F1CD0591C12BB3E
:108BC000626881621A70C38D013B9BB2C3858BB909
:108BD0000368DA6822F02002DA60DA6822F4807230
:108BE000DA605A69202122F001025A6180F83A10B5
:108BF000FFF7D6FF10BD62B96268C2F3080223F81E
:108C0000022B8362DFE76268816202F07F021A70E2
:108C1000D9E76268D2B223F8012B8362D3E700BFA1
:108C2000704700BF03681A6870B51607DD68596998
:108C300004460CD1960601D5A90671D4160601D5B5
:108C4000280646D4510601D56A065ED470BD11F0DF
:108C5000010129D115F4907FF0D0D60709D5E80598
:108C600040F1A180E06B40F00100E063500764D563
:108C7000F1B9960766D5100700F19280E16B0029E3
:108C8000E4D0900602D5A90600F191805A69E16B03
:108C900002F0400201F0080152EA01055CD12046D1
:108CA000FFF7BEFFE56370BDD60742D450073BD542
:108CB000E16B41F00201E163910737D5E16B41F0CF
:108CC0000401E1631107D9D5E16B41F00801E163CB
:108CD000D4E794F83920212AB8D1A168226AB1F5E5
:108CE000805F69D0511C216212785A60E28C013A8F
:108CF00092B2E284002AA9D1DA6822F08002DA6016
:108D0000DA6842F04002DA6070BDDA68202122F0B1
:108D10004002DA60204684F83910FFF73FFF70BD4B
:108D2000BDE87040FFF73EBF9007C7D41107CBD412
:108D3000A4E7E80596D45607BAD4960702D50029C9
:108D400099D0BBE7160799D505F020000843BBD1A1
:108D5000E26B002A9AD170BDDA6822F49072DA6070
:108D60005A69202122F001025A6184F83A105A69A6
:108D7000520611D55A69606B22F040025A6158B10F
:108D8000134B0365FCF70CFA00283FF45FAF606BF0
:108D9000BDE87040036D18472046FFF741FF70BDE6
:108DA000A90691D4D4E756073FF563AFC5E720463F
:108DB000FFF7F8FE236869E711882069C1F308010D
:108DC000596010B90232226290E7013222628DE7C7
:108DD000D58D000808B5806B0023C385C384FFF7D9
:108DE0001FFF08BD0A68F0B450F822301B4D8C6894
:108DF000CE68CF6B1D404B68234333430E6933432A
:108E00004E693343CE6933430E6A33434E6A33436C
:108E10008E6A3343CE6A33430E6B33434E6B896B9A
:108E200033433B430B432B43082C08BF43F0400321
:108E3000B6F5801F40F8223006D012B103681943FE
:108E400001600020F0BC7047002AFAD0036843F4A8
:108E500080130360036819430160F2E78004C0FFD8
:108E60000B6900EB820203F1FF3C536810B58C697B
:108E700003F0404E0B6823434C6843EA04138C68AC
:108E800043EA0423CC68496943EA044343EA0C53A8
:108E9000023943EA016343EA0E0353600368DB02CD
:108EA0004FEA0C5C05D5436823F470034CEA0303D6
:108EB0004360002010BD00BFB3F5804F30B406D032
:108EC0006FF0704340F8223030BC0020704750F8FB
:108ED00022300A4C8D691C400B682B434D6843EAD5
:108EE00005138D68C96843EA052343EA0143234318
:108EF00040F8223030BC0020704700BF0000F0CFA7
:108F0000054BD3F888204FF0006142F47002C3F89B
:108F100088209960704700BF00ED00E0DFF834D092
:108F2000002103E00C4B5B58435004310B480C4BC1
:108F300042189A42F6D30B4A02E0002342F8043B5F
:108F4000094B9A42F9D3FFF7DBFF0FF0FFFDF7F76C
:108F5000BDF9704700000420681D020800000020D1
:108F6000000200200002002078180220FEE737B53A
:108F70000D4600F108010246C36A03C91C688DE86A
:108F800003001046694601F08AF8B5F90020BDF9E2
:108F9000003022449A4217DCB5F90420BDF90430B0
:108FA000121B9A4210DBB5F90220BDF902302244AF
:108FB0009A4209DCB5F90600BDF90630041B9C4253
:108FC000ACBF0020012000E0012003B030BDB0F9AB
:108FD000003070B5B0F904601588D0889488528844
:108FE0004D80F31A9BB2181A9B1A08808B80CC8094
:108FF00070BD438E1B0713B50C460FD5684601F0B4
:1090000061FBBDF802302380BDF80630A380BDF8B7
:1090100000306380BDF80430E38002E0084601F0D0
:1090200051FB02B010BD38B504460D4601F0F9FF02
:10903000E36A284629461A68BDE8384005F0DCBADC
:1090400037B50C46054607F03FFB428E019094422F
:1090500003D04486284602F02CF801A807F042FB12
:1090600003B030BD37B50C46054678B107F02CFB90
:10907000428E019004EA02018C4204D014434486DB
:10908000284602F016F801A807F02CFB03B030BD0B
:1090900037B50D46044670B107F016FB428E0190BD
:1090A00022EA05018A4203D04186204602F001F8F7
:1090B00001A807F017FB03B030BD0000024B428649
:1090C0001B68C36201867047C8000020F0B50D46DA
:1090D00085B00646002800F0938007F0F5FA2B686B
:1090E0000290162B52D00CDC112B33D002DC0D2B4E
:1090F0003ED07EE0142B77D0152B7AD1B0F93030EA
:1091000070E01F2B6BD002DC1E2B42D071E0312BA4
:109110001ED0B3F5407F6CD1C36A1968EB68C36297
:109120001B6802A8CD1A07F0DDFA304607F0CCFA2A
:1091300004AC694244F8040D0A462B46009500F041
:1091400034FF204607F0CEFA304601F0B2FF4EE081
:1091500000243FE0438ED9064BD5EB681B7A002BE9
:1091600047D002A807F0BEFA304601F017F840E0F9
:10917000EB68DB68002B3CD01B7A002B39D002A8AF
:1091800007F0B0FA304601F0BDFA30E0EB68038634
:109190002DE0EB68418E012B08D1CA060DD5304673
:1091A00041F00101FFF74CFF082708E021F0010121
:1091B0003046FFF745FF092701E04FF0FF3702A8CF
:1091C00007F090FA7B1C4FF0000405D0304639467A
:1091D00001F0B7F8EC600DE00123EB600AE0438E8C
:1091E000C3F30013EB6002E0E968FFF71CFF002403
:1091F00000E00124029B23B102A807F073FA00E00B
:109200000124204605B0F0BD70B50D46FE2116467E
:10921000044601F035FA294600F0B3FF2046FF214D
:1092200001F02EFA3146BDE8704000F0AABFF8B553
:109230001C46438E069F1B070D4616460AD5002C7A
:1092400007DB2846311BA21906F018FB013C3D4400
:10925000F5E7F8BD002C07DB2846311BA21906F004
:1092600095F8013C3D44F5E7F8BD37B505460C4699
:1092700019B9684601F026FA6C466B8E1B0705D5B6
:10928000224628466946FFF7A2FE6C46284621463C
:10929000FFF76DFE18B1EB6A20461B69984703B0D3
:1092A00030BD2DE9F04F2DED028B85B00D4607F056
:1092B0000BFA0090006905F01BFF009BD86805F0D1
:1092C00045FF022005F0F8FE009CA68CE36916F02D
:1092D00001061AD0002B77D0A06807F0F5F90190AD
:1092E000C26A636917681F4401F01EF9A369384414
:1092F00033B1012B70D1B5F9003083426CDD1CE035
:10930000B5F90430834218DB66E0002B5CD0A0681E
:1093100007F0DAF90190C36AD3F8008006F010F87C
:1093200063690746C8EB030901F006F9B5F90210B5
:10933000EA88484407448F4203DA01A807F0D2F9CB
:1093400042E012B29042F8DCA06802A901F0FCF8F9
:10935000019BBDF90CB0DA6DD3F854A0BDF90870CB
:10936000256AC2EB0B0BB3F87820D207574458BFDD
:10937000D3F88C603D443544BD4222DDE369ED1AEB
:10938000FAE7BD421BDDA06905F0A0FE236AD4ED1B
:109390000A7AEB1ACAEB0303C8EB03039B1B08EE24
:1093A000103AB8EEC88A284628EE278A494605F0C2
:1093B000ABFFB0EE480A94F82C0005F0A5FCE36979
:1093C0001D445D45DDDDB8E7684607F08BF905B063
:1093D000BDEC028BBDE8F08FA06802A901F0B4F8E3
:1093E000019B1D6ED3F8588005F0AAFFBDF90E60F1
:1093F000019BBDF80AA0D3F88030761B256A751B47
:109400001D44B54201DAE369FAE74FF0020990FB27
:10941000F9F908FA8AF39D428FDBB5421CDCA0699A
:1094200005F054FE236AD4ED0A7A711BC91A019B18
:10943000D3F880208A1808EE102AB8EEC88A384679
:1094400028EE278AC9EB050105F05EFFB0EE480A59
:1094500094F82C0005F058FCE369ED1AD9E70000F8
:109460002DE9F34781463020884617461E4607F00F
:10947000FDFB8246D0B107F027F902AD0D4A45F851
:10948000040D4FF07E538362C0F81490C0F818802A
:109490008784C66100F10C03044692E8030083E868
:1094A0000300054B2360284607F01CF9504602B024
:1094B000BDE8F087CC000020A392000800B52DED98
:1094C000028BF0EE408A83B090B107F0FDF890ED8A
:1094D0000A8A0190B4EE688AF1EE10FA04D0C0ED69
:1094E0000A8A806801F0E5FD01A807F0FBF801E0B9
:1094F0009FED048AB0EE480A03B0BDEC028B5DF824
:1095000004FB00BF0000000013B5044607F0DCF8C0
:109510000190406A20B107F011F9019B00225A62C4
:1095200001A807F0DFF8204607F008F902B010BDE7
:109530002DE9F0438BB007F0C7F80790406A002888
:1095400060D007F0C1F8079B05900646986807F0C1
:10955000BBF8079BD0F85480056E876DC46D0690EC
:1095600008A9986800F0F0FFBDF82230079A069825
:10957000BDF82010D2F820901F44ADF82270BDF83D
:109580002430BDF826701C1B7F1B1369D0F88C504B
:109590005D1B92F82830414489B2A4B2BFB2012BBE
:1095A000ADF82010ADF82440ADF82670D0F88080DA
:1095B00009B208D024B2641B0134A14204DD0C1BA3
:1095C00006EB44062D1B0C46002D15DD906905F0B9
:1095D000BDFD4FF0FF3201238DE80C00079A3FB22A
:1095E00092F829300293C9EB0709304629462246F2
:1095F00009EB080306F066F906A807F073F805A85A
:1096000007F070F807A807F06DF80BB0BDE8F0831D
:109610001FB590F82830012B0446806827D102A995
:1096200000F092FFA06807F04FF8BDF80A20836DA4
:1096300001901344ADF80A30BDF80E20036ED31A22
:10964000ADF80E30426DBDF8083013442269134462
:109650009BB29A1E01A8013BADF80820ADF80C3072
:1096600007F040F8A06802A901F0E7FC01E000F073
:109670005FFB04B010BD00002DE9F74380462C20AD
:109680000E4617461D4607F0F1FA044618B370005F
:1096900007F0ECFA814658B157B14DB107F014F814
:1096A00039466A0001900FF0CBFA01A807F01AF8CA
:1096B000204607F009F80A4B0190C360094B03608C
:1096C000094BC0F82490C0F81880466105614360DA
:1096D00001A807F007F8204603B0BDE8F08300BFFB
:1096E0001196000831950008099500081FB5ADF8DE
:1096F000061006F0E9FF029068B1406A06F0E4FF48
:109700000DF10602014603900223029800F03FFB90
:1097100003A806F0E7FF02A806F0E4FF05B05DF835
:1097200004FB13B50C4660B106F0CEFF036A01904E
:10973000A34203D00462806801F0BBFC01A806F0DC
:10974000D1FF02B010BDF0B58BB002A9044600F005
:10975000FBFE204606F0B8FFBDF90A20BDF90E60F9
:109760000190B61A826D456DC76DB61A026EB61AB3
:10977000B0F87820510707D4416FB1422046D4BFDA
:109780000021012100F0FBFC019BBDF90C105A6F78
:10979000DA67BDF90820C3F884608A1A551BB3F84C
:1097A00078209207C7EB050507D4196FA942204618
:1097B000D4BF0021012100F0E0FC0198036FC0F844
:1097C0008830C0F890507C3000F08AFF01988830D3
:1097D00000F086FF019B03F17C0207CA883307AEC5
:1097E00086E8070093E8070004AD85E8070001A8B4
:1097F00006F078FF204631462A46FFF705FD0BB0FC
:10980000F0BD73B50C46064606F05EFF019020469B
:1098100007F066FB0546204600F0F6FE019BFE2899
:109820000CBFC3F88050C3F88C50304601F041FCA7
:1098300001A806F057FF02B070BD2DE9F04F446853
:109840000668054697B020462946FFF73FFCB6F567
:10985000407F074602D12046FFF775FF002F00F03A
:1098600064822B680B2B00F0008206DC052B40F095
:1098700059822046FFF767FF54E20F2B03D0262BB7
:1098800000F03D824EE2ED680295204606F01CFF96
:10989000C36AC16D1B68D0F85490D0F858B0D0F8A6
:1098A00060A00D900EAD28460393019100F00AFFD1
:1098B0000D982946FFF7D9FC95E8030012AB83E821
:1098C00003000398BDF84A1082B25944BDF84E0017
:1098D0001144ADF84A1002EB0A01411AADF84E10DE
:1098E000BDF8481011444944ADF8481001990A44A4
:1098F000BDF84C108A1AADF84C2093E8030010AA6A
:1099000082E80300104600F0FBFB0D9B586B05F04E
:109910001BFC06F0A9FA0D9BD3F8943013B1204636
:10992000002198470D9D95F86C30002B00F08D803C
:10993000204614A900F008FEEB6ABDF856001B682B
:10994000BDF85420BDF8521004930790BDF8503074
:10995000286C0592069308916E6CAF6C05F0F6FBCF
:1099600005F0E8FC099016B9002F4BD146E0EB6CEE
:1099700006EB030CB5F87830DB0754BFD5F88C3014
:1099800000230CEB0308B04502DBC6EB0808FAE73E
:1099900095F87A0005F0A4FB0598019A03B20698A1
:1099A0004A4401B2C2F101025B1A13449845DBDA62
:1099B0000498BDF95210BDF9563095F87A20484404
:1099C00040445944CAEB03031AB1024605F038FF7C
:1099D00002E01A4605F0DAFCB044DDE795F87B00BA
:1099E00005F07EFB079908980BB20BEB0A0201B257
:1099F000C2F101025B1A13449E420CDB099805F088
:109A00006FFB22E02E6DD5F880303E44F61ABE4240
:109A1000E4DBF61BFBE70198BDF95420BDF95610B5
:109A2000BDF95030121A95F87B00CAEB0101891B71
:109A30004B4420B118460B4605F002FF03E00846F0
:109A4000194605F01BFF3E44CCE7039A12A80EA965
:109A500004F0D2FD12A800F053FB0D9B93F83B20BD
:109A6000FF2A00F0A380B9F1000F08D1BBF1000F6D
:109A700005D1019919B9BAF1000F00F09780DA6A9F
:109A800014A920461568009300F05EFD00F04CFD1F
:109A9000049000F051FDBDF95220009BBDF95460C7
:109AA00005905A440392019A986BBDF95070BDF924
:109AB0005680B61A05F048FB009BD86B4F44CAEBA2
:109AC000080805F043FBB9F1000F1BD00298049978
:109AD000B0F9003009F1FF322A445B1A934211DCDD
:109AE000BDF95630BDF95000CAEB030305EB0B017D
:109AF000013306F087F9039A781E511E08F101021E
:109B000005F044FCBBF1000F17D002980599B0F99D
:109B100002200BF1FF332B44521A9A420DDCBDF99F
:109B20005000BDF95210BDF9542006F06BF9039AAC
:109B3000791E501E721C05F0A1FE019BD3B1029943
:109B4000BDF95420D01AB1F90430049901305B1AE0
:109B500083420FDBBDF95630CAEB030305EB0B0163
:109B6000013306F04FF9039A701C511E08F10102EF
:109B700005F00CFCBAF1000F18D00298BDF9563070
:109B8000B0F906200598CAEB03010131C0EB020AC7
:109B90008A450BDBBDF95000BDF9542006F032F9BF
:109BA00008F10100791E721C05F068FE0D9BD3F8C8
:109BB000943013B120460121984710A800F0A0FA74
:109BC0000D9B586E07F098FC00250746BD421AD041
:109BD0000D9B2946586E07F011FD06F075FD149097
:109BE00078B10668304606F06FFD0C9030B103681E
:109BF0000299304698470CA806F074FD14A806F0A8
:109C000071FD0135E2E712A800F07AFA0D9B986E1B
:109C100007F072FC00250746BD421AD00D9B29466D
:109C2000986E07F0EBFC06F04FFD149078B10668D3
:109C3000304606F049FD0B9030B10368029930467A
:109C400098470BA806F04EFD14A806F04BFD013511
:109C5000E2E7002000F054FA0D9BD3F8943013B1E2
:109C60002046022198470DA846E0204606F02CFD2C
:109C70001290406E07F040FC00240646B442129B4E
:109C800018DA586E214607F0B9FC06F01DFD149055
:109C900070B10568284606F017FD109028B1476896
:109CA00010A806F01FFD2846B84714A806F01AFDB4
:109CB0000134E3E7986E07F01FFC00240546AC4230
:109CC000129B0FDA986E214607F098FC06F0FCFC18
:109CD000149028B1006806F031FD14A806F002FDCA
:109CE0000134ECE716AC586E07F05FFC54F8103DF9
:109CF000986E07F05AFC204606F0F4FC15E0EB687D
:109D0000052B0FD12046AE6800F0F0FB864205D04F
:109D10002046AE6800F0E5FB864203D16868A9687A
:109D2000FFF76FFD284601F0EFFD17B0BDE8F08F9B
:109D30002DE9FF41044606F0C7FC034604A8D3F80A
:109D4000548040F80C3D9F6DDE6D1D6E06F0CAFC20
:109D5000204602A900F0F8FBBDF808309844BDF891
:109D60000A30ADF808801F44BDF80C30ADF80A7019
:109D70009E1BBDF80E30ADF80C605D1B204602A99D
:109D8000ADF80E5001F059F904B0BDE8F081F8B516
:109D90001D46836804460E46174623B3006963696F
:109DA00098420ED1421E6A43084629440EF09CFE9A
:109DB0002069013800FB056039462A460EF094FE02
:109DC0000CE0431C236100FB051011462A460EF0EF
:109DD0008BFEE36813B120469847F8BDA068BDE844
:109DE000F840FFF7A5BFF8BDF0B587B00C9C009414
:109DF0000D9C0194174C0294109C6C34039401F058
:109E000099F9064618B307F00CFC054607F009FC63
:109E10000446304606F058FC45660F4D84660F999F
:109E200005900022FFF74AF906AF0FCD57F804ED71
:109E30000EF134040FC40FCD0FC495E80F0084E871
:109E40000F000E9BAEF87830384606F04BFC3046DB
:109E500007B0F0BD3B980008D400002010B586B0D4
:109E6000089C0094099C01940A9C02940B9C039406
:109E700000240494FFF7B8FF06B010BD30B585B0DC
:109E800004460191D0B106F01FFC04AB456E43F8C7
:109E9000040D184606F026FC019806F015FC024653
:109EA00004A8946040F8082D06F01CFC284601A97F
:109EB000042207F030FB204601F0FBF805B030BD6E
:109EC00030B585B004460191D0B106F0FDFB04AB7E
:109ED000856E43F8040D184606F004FC019806F060
:109EE000F3FB024604A8946040F8082D06F0FAFB44
:109EF000284601A9042207F00EFB204601F0D9F8FC
:109F000005B030BD73B50D461446064698B106F04F
:109F1000DBFB032C019009D800EB8400446BAC42BE
:109F200005D04563304601F0C4F800E0002401A8E4
:109F300006F0D8FB00E00446204602B070BD73B5C1
:109F40000E46054678B106F0BFFB90F86C400190D4
:109F5000B44204D080F86C60284601F0AAF801A849
:109F600006F0C0FB00E00446204602B070BD2DE9BB
:109F7000F3410F4690461D46064698B106F0A4FBF5
:109F8000044602A8089B236640F8044D6765C4F8A0
:109F90005880E56506F0A6FB3046FFF7D4FB304657
:109FA00001F087F802B0BDE8F0812DE9F04F87B0ED
:109FB000C46903938A469346002C6DD0204606F070
:109FC00083FB816A059001F42073802BB0F8008038
:109FD00042888688C58808D0B3F5207F08D108EB71
:109FE0000A091FFA89F9039B08E0039883B201E08C
:109FF0001FFA8AF303EB08091FFA89F901F4A0613B
:10A000003344B1F5807F9BB208D0B1F5A06F08D181
:10A0100002EB0B0C1FFA8CFC109F08E010998FB21A
:10A0200001E01FFA8BF707EB020C1FFA8CFC0FFA0A
:10A0300089F90FFA88F812B22F440FFA8CFCB9EBA9
:10A0400008010292BFB2C2EB0C0200D142B120461D
:10A050000193CDF800C000F008FADDF800C0019BC4
:10A060001BB2C9EB030936B2029BC6EB08083FB22C
:10A070002DB2CCEB070C5D1B19EB08010CEB0502B4
:10A0800000D112B1204600F0E1F806A850F8043DD6
:10A090001C6A06F027FB8FE707B0BDE8F08FB0F928
:10A0A0000030B0F9022008465242594205F0E0B8AB
:10A0B00010B5044670B100F0FCFF204600F0BBFA7A
:10A0C00004463CB12046FFF7F3FF204606F0F2FAC3
:10A0D000046AF6E710BD13B5044670B106F0F4FA51
:10A0E000826A0190930705D442F002028262204600
:10A0F000FFF7DEFF01A806F0F5FA02B010BD000080
:10A10000044B10B51B685C6C586400F02BFE2046B5
:10A1100010BD00BF1C010020F7B50D4611460646D4
:10A120001F4600F0ADFA0446A5B120B930463946C5
:10A1300006F0E5FE14E006F0C7FA02AB826A43F8C7
:10A14000040D22F4004242F002028262184606F038
:10A15000C9FA05E020B100F08CF9204601F006FBB9
:10A16000201C18BF012003B0F0BDFE220823FFF71A
:10A17000D3BFFF220023FFF7CFBFFFF7FABFFFF7E0
:10A18000F4BF1FB530B129B1242303916946009370
:10A1900000F038FF05B05DF804FB0000F0B587B0B3
:10A1A0000446002102A810220EF0B7FC002C3AD081
:10A1B0001F4B204A196852F82100844216461F4658
:10A1C00031D01E238DE81100029310B102A907F0CF
:10A1D0003FFA0123204602A9059307F039FA059DAD
:10A1E00015BB3B6846F82340204600F084F904463E
:10A1F00038B12023029302A900AB059307F028FA97
:10A20000F2E7009C204600F032F968B1204600F0E9
:10A2100072F9044640B12023029302A900AB0593D2
:10A2200007F016FAF2E70125284607B0F0BD00BF97
:10A230001817022008170220024B1A6818601046EF
:10A24000704700BF2017022007F0EEB92DE9F0415A
:10A2500051EA02038AB080460E4617466ED00028A7
:10A260006CD006F031FA0346039003C804AD06AC87
:10A2700085E8030084E803007EB19A6A02F4207244
:10A28000802A05D1BDF81820961BADF8186004E0AF
:10A29000BDF81C201644ADF81C6087B19A6A02F420
:10A2A000A062B2F5807F05D1BDF81A20D71BADF8AA
:10A2B0001A7004E0BDF81E201744ADF81E709B6AAA
:10A2C000DA0302D5404600F081FD94E80300039BC9
:10A2D00083E803009B6A9B070AD508A82946224603
:10A2E00004F0D6FF039B08A899691A6A00F072FE71
:10A2F000BDF91C40BDF91430BDF91E70BDF9160042
:10A30000BDF91860BDF91010BDF91A50BDF9122041
:10A31000E31A381A0AACAA1A0090711A0398FFF7C8
:10A3200044FE54F81C1D01F1080004F021FA4046D7
:10A33000052100F06BFE204606F0D4F90AB0BDE816
:10A34000F0811FB5262303916946009307F0A6FA12
:10A3500005B05DF804FB2DE9F04188B006460C46D7
:10A36000154604A8002110220EF0D7FB36B3304664
:10A3700006F0AAF921462A46019004F079FF0198D7
:10A38000214608302A4604F073FF08A850F81C2D17
:10A39000D2F81C80176A06F0A5F9404621462A46E5
:10A3A000FFF7D9FF03230493304602AB04A90793B8
:10A3B000029403953E4607F04BF9D7E708B0BDE895
:10A3C000F0812DE9F0438BB006460D46144606A8F1
:10A3D000002110220EF0A1FB002E43D00DB9002C5D
:10A3E00040D0304606F070F90346019003C80DF1E5
:10A3F000080888E8030022461846294604F038FF7A
:10A4000001980AAF29462246083004F031FF57F878
:10A41000243DD3F81C90384606F064F9224648469D
:10A420002946FFF798FF304606F04EF9826A019000
:10A4300092070AD5816941B1026A00F0B6FD019B1D
:10A44000404699691A6A00F0B0FD384606F04AF9AC
:10A4500003230693304604AB06A90993049505949B
:10A4600007F0F6F80BB0BDE8F083FFF7AABF00F0E5
:10A470009DBC13B588B106F027F9826A02AC91073A
:10A4800044F8040D06D522F0020282628169026A54
:10A4900000F0A0FD204606F025F902B010BD70B511
:10A4A00006460D4606F006F9C4694CB1204600F098
:10A4B000ABF8A842204613D006F0FCF8046AF4E793
:10A4C000304606F0F7F8C469204644B12946FFF744
:10A4D000E6FF28B9204606F0EDF8046AF4E770BDFF
:10A4E00070BD10B1FF21FFF7DABF704710B1FE2138
:10A4F000FFF7D5BF704708B5034610B106F0DAF88C
:10A500008369184608BD08B520B106F0D3F8B0F944
:10A51000000008BD08BD08B520B106F0CBF8B0F9C1
:10A52000020008BD08BD0000024B1B68986CFFF7D5
:10A53000EABF00BF1C010020024B1B68986CFFF7AC
:10A54000EABF00BF1C010020F0B50C4687B00646EC
:10A5500000284BD0002949D0FF2100F091F8FE21BE
:10A560000546304600F08CF869460746304607F04D
:10A57000BDF9304602A900F03BF8C7B1384604A93E
:10A5800007F0B4F9BDF90010BDF9022004A8494252
:10A59000524204F06DFE384600F046F800F08200AA
:10A5A000822804D1BDF81030013BADF80C30CDB19C
:10A5B000284604A907F09AF9BDF90010BDF9022058
:10A5C00004A84942524204F053FE284600F02CF8F9
:10A5D00000F48170B0F5817F04D1BDF81230013BE9
:10A5E000ADF80E3002AB03CB2060616007B0F0BD68
:10A5F0001FB5039104A9142341F8103D694600F0EA
:10A6000001FD05B05DF804FB1FB504461022684645
:10A6100000210EF082FA152320466946009300F0CF
:10A62000F1FC039804B010BD08B518B106F042F86B
:10A63000008D08BD08BD08B5034610B106F03AF814
:10A64000C369184608BD37B50D4606F03DF802ABA4
:10A65000C46943F8040D184606F044F820466CB16E
:10A66000FFF7D2FFA842204608D02946FFF7EBFFAC
:10A6700020B9204606F01EF8046AEFE703B030BDAB
:10A6800008B1FFF7E0BF7047034B1B685A7C034BD0
:10A6900053F82200704700BF1C010020F81602206A
:10A6A00037B50D4658B151B106F00EF802AC294647
:10A6B00044F8040D00F0B5FC204606F013F803B092
:10A6C00030BD0000044B0146186810B9034B1B68ED
:10A6D000986CFFF7E5BF00BFF41602201C010020B4
:10A6E00002688368D31A4268002ABCBF0022426015
:10A6F000426823EAE3739A42C8BF4360704700F0A0
:10A70000D8BC000073B50546002832D005F0DCFF48
:10A7100002AC034644F8080D006A08B968460EE02A
:10A720009B6A1A0711D405F0CFFF836A02AE1B079C
:10A7300046F8040D06D5684605F0D4FF304605F00E
:10A74000D1FF16E0304605F0CDFF009B68469E69BC
:10A7500005F0C8FF284600F0B7FA3146284600F059
:10A7600061FA284600F0A5FC28460349002207F0BC
:10A77000DCF802B070BD00BFFFA600080A4A0B4912
:10A78000002313700A4A0B6013600A4A4B6013607F
:10A79000094A13605360094A1360094A1360094A61
:10A7A0001360094A13607047C4D7012008170220BC
:10A7B0009CD701202C1702203417022040170220BA
:10A7C000F4160220201702203017022010B504468C
:10A7D00005F070FF836A044A13F4803F034B204660
:10A7E00008BF1346984710BD31B600081DBC0008CD
:10A7F000F0B5054685B00C461646002D4CD02846CF
:10A8000005F062FF876A0190BB0701463DD502ADA6
:10A8100026B12846324603F079FF02E003C885E8F6
:10A8200003002046294604F0D9FC70B317F0010F4D
:10A83000019B1ED13EB1B3F90220B6F902309A4213
:10A84000A8BF134601E0B3F90230B4F902209342E5
:10A85000B4F9062006DDBDF80A3019B28A4214DBCD
:10A86000013B04E0BDF80E3019B28A420DDDE380F1
:10A870000BE0DF694FB1384621462A46FFF7B8FFA3
:10A88000384605F017FF076AF4E704A850F80C3DB6
:10A890001D6A05F027FFB0E705B0F0BD2DE9FF41C7
:10A8A00004460F4690460025002C37D0204605F080
:10A8B0000BFF866A0190B207014628D502ACB8F1B9
:10A8C000000F04D02046424603F020FF02E003C8F8
:10A8D00084E803003846214604F080FCB8B1F30751
:10A8E00005D4BDF80C3001333B8001250FE0019BFE
:10A8F000DE6966B1304639462246FFF7CFFF0028B1
:10A90000304618BF012505F0D5FE066AF1E704A818
:10A9100050F80C3D1C6A05F0E5FEC5E7284604B07A
:10A92000BDE8F081F0B5044685B00E461746002C10
:10A9300031D0204605F0C8FE856A0190AA0701467D
:10A9400022D502AC27B120463A4603F0DFFE02E0F2
:10A9500003C884E803003046214604F03FFC98B168
:10A96000EB0704D4BDF80830013BB3800CE0019B39
:10A97000DD694DB1284631462246FFF7D3FF284610
:10A9800005F098FE056AF4E704A850F80C3D1C6A2F
:10A9900005F0A8FECBE705B0F0BD00002DE9F341BE
:10A9A000214D2B680646986C05F08EFE00903046CF
:10A9B00005F08AFE02AC0146019054F8080D0830FB
:10A9C00004F00CFC074628B30199009A2B68174C39
:10A9D0001F6DD3F84C8001F10800083203F096FE99
:10A9E000684605F07FFE019A2B68B2F90010B2F9B3
:10A9F0000220D9641A6501A8266005F073FE30466E
:10AA0000FFF7E4FE002323602B681F65C3F84C802A
:10AA1000012705E0684605F065FE01A805F062FE25
:10AA2000384602B0BDE8F0811C010020F416022077
:10AA30002DE9F347064605F047FE836A01909B0720
:10AA400005D401A805F04EFE02B0BDE8F087C46948
:10AA5000002CF6D0204605F037FE836A02AD03F0E5
:10AA60000303032B45F8080D37D10199083104F091
:10AA7000B5FB002831D002A850F8043DB3F8089087
:10AA8000B3F80A809F89B3F80EA005F02BFE684644
:10AA900005F028FE2046FFF781FF70B1204605F043
:10AAA00009FE00902046FFF7C3FF204605F002FE96
:10AAB0000090304605F0FEFD0190304605F004FEA2
:10AAC0000190204605F000FE019B0090A3F808903D
:10AAD000A3F80A809F81A3F80EA0009B68461C6A19
:10AAE00005F000FEB4E7000037B5044605F0ECFDC4
:10AAF000826A019040F601031340012B05D001A8A2
:10AB000005F0F0FD2046FFF761FE144B1B6813B300
:10AB10002046FFF78DFF204605F0CCFD8569046ACD
:10AB2000CDB194B1204605F0C5FD836A03F003035F
:10AB3000032B02D12046FFF731FF2046FFF778FFB5
:10AB4000204605F0B7FD046AEBE7284605F0B2FDA4
:10AB5000046A8569E4E703B030BD00BF40170220F6
:10AB60002DE9F347174D2B680646986C05F0ACFDB0
:10AB70002A68B0F808A0B0F80A90B0F80C80C7892D
:10AB800002AC083244F8040D00F1080392E8030017
:10AB900083E80300204605F0A5FD3068FFF7A4FF19
:10ABA0002B68986C05F090FD0190A0F808A0A0F823
:10ABB0000A90A0F80C80C781204605F093FD02B0F2
:10ABC000BDE8F0871C010020F7B507460D46284672
:10ABD00005F07AFD836A02AC13F00206014644F8E0
:10ABE000040D04D1204605F07DFD304616E03846C0
:10ABF00003F0BEFD019B9E69204656B905F072FD2B
:10AC0000074B1A68954208D058682B1A5842584189
:10AC100004E005F067FD3546D9E7012003B0F0BD3B
:10AC2000F8160220F0B5044685B00D46002949D03B
:10AC300005F04AFD0023036285610190284605F076
:10AC400043FD019BC56902909F6A2DB9C46101A8AB
:10AC500005F048FD02A833E0284605F035FD04AEB6
:10AC600007F0080746F8040D77B9836A1A070BD571
:10AC7000019B1D62029B01A8DC6105F033FD02A867
:10AC800005F030FD30461BE002A805F02BFD3046F4
:10AC900005F028FD284605F00DFD0390039B1D6A75
:10ACA0000DB91C620BE0284605F004FD002FF4D11D
:10ACB000836A1B07F1D5039B1C62019B1D6201A8DF
:10ACC00005F010FD05B0F0BD70B5044605F0F2FCCE
:10ACD00005468069A8B105F0EDFCC369A3420646AC
:10ACE00005D1184605F0E6FC036AF36170BD43B177
:10ACF000184605F0DFFC036AA342F8D12B6A036211
:10AD000070BD70BD03460846B3F90220B3F90010C8
:10AD100004F0AEBA114B30B51C68626C85B00546C4
:10AD2000BAB11068516802AB03C30D4B186800B983
:10AD3000A06C05F0C9FC04AC02A944F80C0DFFF7A7
:10AD4000E1FF204605F0CEFC02A8294603F010FDE5
:10AD500002A802F033FF05B030BD00BF1C01002087
:10AD6000F41602201FB50E4B1B6893F854200AB14D
:10AD70000C4811E0986C05F0A7FC019003C802ACE8
:10AD800084E8030001A805F0ADFC074B196811B178
:10AD90002046FFF719FF2046FFF7BCFF04B010BDA7
:10ADA0001C010020A8D70120F4160220064B10B584
:10ADB0000446186828B1A04204D005F07BFC406925
:10ADC000F8E710BD012010BD1417022013B504468A
:10ADD00000B305F079FC826A0190930717D5406AA9
:10ADE00040B10D4B1B68A34204D001F0DFFD019B75
:10ADF00000225A622046FFF71EFC04463CB1204662
:10AE0000FFF7E4FF204605F055FC046AF6E701A8C9
:10AE100005F068FC02B010BD3C170220B0F900201C
:10AE2000B0F904309A4208DCB0F90220B0F90630DB
:10AE30009A42CCBF002001207047002070470000DC
:10AE4000F0B585B006460D46174605F033FC846A1A
:10AE50000190A30734D52846FFF7E0FF00282FD044
:10AE600040F601032340012B2AD0304605F02CFC8C
:10AE700002AC024601902946204603F047FC2046DA
:10AE8000FFF7CCFFC8B1019B9E6A44F2200131401C
:10AE900003F1080529B128462946224604F0F8F9AD
:10AEA0000BE094E803003E4385E803009E62054BF7
:10AEB0001A8801321A8003F021FE01A805F012FC65
:10AEC00005B0F0BD101702202022FFF7B9BFF0B582
:10AED0000F4685B01546064648B305F0F5FB836A74
:10AEE00004AC9B07024644F80C0D03D4204605F041
:10AEF000F9FB1CE002A8394603F008FC0028F5D055
:10AF0000204605F0EFFB304602A92A46FFF798FFDE
:10AF10003046FFF790FB04464CB1204602A92A4672
:10AF2000FFF7D5FF204605F0C5FB046AF4E705B03E
:10AF3000F0BD2DE9FF41804617461D460C4600290D
:10AF400030D0084605F0C0FB866A0190B307024680
:10AF500025D502A8414603F0D9FB00B340F6010312
:10AF60003340012B07D1019B02A899691A6A2B462D
:10AF7000FFF7DFFF04E0204602A92A46FFF760FF43
:10AF8000019BDC695CB1BC4209D0204602A92A467B
:10AF9000FFF79DFF204605F08DFB046AF2E701A84C
:10AFA00005F0A0FB04B0BDE8F08170B50546084689
:10AFB0000C46164605F07EFB836A13F4803F284654
:10AFC000214632460CBF20234FF48043BDE8704039
:10AFD000FFF7AFBF2023FFF7ACBF13B5044605F062
:10AFE00073FB8169019041B1026AFFF7F3FF2046CC
:10AFF000FFF76AFE019B00229A6101A805F072FB2F
:10B0000002B010BD08B106F023BB70471FB504ABFA
:10B01000019043F8101D694606F01AFB05B05DF873
:10B0200004FB00230B8082884B800388D31A8B801B
:10B03000C2884388D31ACB807047F0B50F4687B0DB
:10B040000546002833D005F03FFB866A0190B20721
:10B050002AD503C804ACF30384E8030002D52846CC
:10B06000FFF7B4FE5FB13868796802AB03C301989B
:10B0700002A9FFF747FE204602A903F079FB20460C
:10B080002946FFF7A1FD78B140F601033340012BBB
:10B0900006D1019B204699691A6AFFF79BFF03E0DE
:10B0A00028462146FFF710FF01A805F01BFB07B05B
:10B0B000F0BD0021FFF7C1BF10B5044605F0FAFA54
:10B0C00080690028F9D1054B1A68944205D0586868
:10B0D000844214BF4FF0FF30012010BDF81602204B
:10B0E00008B5FFF7E9FF002803DBBDE8084004F0DE
:10B0F00041B808BD0D4A136870B59D6C04461646EC
:10B1000008B90B4A14689C642046FFF7E9FF03F076
:10B1100059F9204605F0CEFA3368B0F90010B0F9BD
:10B120000220D9641A65284670BD00BF1C010020AA
:10B13000141702202DE9F74F0C9D9B464B4B0746F9
:10B14000884692461E6865BB494B1B8863B3494BD2
:10B150001B685A7C484B53F822305A1C24D01BB32E
:10B160001D46284605F0B0FAB0F90020B0F90230CB
:10B17000019017449844BAF1000F05D1B0F904A02A
:10B18000C2EB0A0A0AF1010ABBF1000F05D1B0F9BE
:10B1900006B0C3EB0B0B0BF1010B01A805F0A2FAF3
:10B1A00002E06B1CDDD100250F982C3005F05EFD10
:10B1B0000446002856D00D9B1E432D4B1A880132A1
:10B1C0001A8005F081FA0E9B03610DF108092B4BE3
:10B1D000826A49F8080D33400780A0F8028057447E
:10B1E000D8441343013F08F1FF3883628780A0F8F9
:10B1F0000680684605F076FA214B186848B105F0DC
:10B2000059FA0746204605F055FA7B6943617C618F
:10B2100000E01C6029462046FFF704FDB50602D574
:10B220002046FFF767FFF00703D5164B1A68013277
:10B230001A60710602D5204606F082FBB2070DD5D2
:10B24000204605F041FA836A009043F002038362CE
:10B25000684605F047FA2046FFF72BFF20460121FC
:10B26000FFF7D4FE204603B0BDE8F08F2017022080
:10B27000F01602201C010020F81602209F3F3F001C
:10B28000141702204017022073B5044600286ED020
:10B29000FFF78CFD00286AD02046FFF70DFF0B2139
:10B2A00005462046FFF7B2FE204606F034FA204657
:10B2B00005F00AFA0190406A08B101F077FB2D4BC6
:10B2C0002D4A002119602D4B1B6852F82300A04223
:10B2D00008BF42F823102A4A52F82310A14204BFA3
:10B2E000002142F82310274B1B682BB15A68A24259
:10B2F00004BF00225A60F7E720460721FFF721F834
:10B30000019EF069FFF7C0FFF369002BF9D12046D9
:10B31000FFF763FE1C4B186850B105F0CBF90646E9
:10B320004069A042F8D1204605F0C4F94369736131
:10B33000019B9B6ADA0703D5144A11680139116031
:10B340009B0603D5124B1A88013A1A8001A805F012
:10B35000C9F9104B1A882046013A1A8005F0EEF917
:10B36000002D04DB0C4B53F82500FFF7C3FE02B0A1
:10B3700070BD00BFB8D7012008170220181702209F
:10B38000341702202C170220141702204017022025
:10B3900010170220F0160220F81602202DE9FF41B6
:10B3A0005D4F3B6893F85400002800F0B2805B4B7F
:10B3B0005A69012A1C4603DD013A5A610020A8E0BF
:10B3C00004F108061B6996E80300013302AD23610E
:10B3D00085E8030023B92388ADF80830638811E0BD
:10B3E000A3896289ADF80A2001339BB2B4F9042025
:10B3F000ADF808301BB29A4206DA2388ADF808305F
:10B40000E3890133ADF80A30BDF90A20B4F90630FA
:10B41000DFF808819A4204DD6369013B0020636123
:10B4200077E03B68986C05F04FF9BDF90820B8F952
:10B43000003001909A421CD1B8F80630ADF80E30B9
:10B44000B8F80430ADF80C30334B1B689A6C5AB125
:10B45000104605F02FF980460022006A2946FFF7C2
:10B46000C7F9D8F81820F2E7019B2946D869FFF7F9
:10B47000BFF9BDF80830ADF80C303B689A6C6AB182
:10B48000104605F017F9294680460022006AFFF7AA
:10B4900005FA0028EDD1D8F81820F0E7019B2946DD
:10B4A000D869FFF7FBF90028E3D1A388BDF908208C
:10B4B000ADF80C301BB29A4207DD95E8030086E830
:10B4C000030001A805F00EF997E73B689A6C52B1AA
:10B4D000104605F0EFF807460022006A2946FFF7FC
:10B4E00021FABA69F3E704AF294657F80C3DD86949
:10B4F000FFF718FA384605F0F5F8236944F620629C
:10B50000934289DC95E8030086E80300FFF72AFCF4
:10B51000012004B0BDE8F0811C010020A0D701206B
:10B520002DE9F041394F3B6893F8542086B0064628
:10B5300012B9FFF717FC64E0354D6A690132012A40
:10B540006A612C465DDC986C05F0BEF84FF0FF3266
:10B550002A61304A009012782AB100F1080302AA49
:10B5600093E8030005E0826A12F002080AD003C8DB
:10B5700002AA82E8030002AD66B12846314603F014
:10B58000F7F807E06B696846013B6B6105F0AAF8C4
:10B59000404637E03B68204E5A6CC2B1009B1068B1
:10B5A0005168019304AB03C3336833B101A805F0BC
:10B5B00099F8306805F088F80190019804A9FFF720
:10B5C000A1FB284604A903F0D3F801A800E06846CF
:10B5D00005F088F8316819B12846FFF7F5FA28B167
:10B5E0003B682846996CFFF7EFFA18B96369013B8D
:10B5F000636107E095E8030084E80300FFF7CEFEEF
:10B6000000E0012006B0BDE8F08100BF1C01002071
:10B61000A0D701201D170220F416022008B503F060
:10B6200073FD024B1B6800225A6408BD1C010020F8
:10B63000F0B589B0044605F047F80769866A0190BD
:10B64000083003C802AD85E8030001A805F04AF8F8
:10B65000002F31D0B3072FD520462E21FEF7F4FD61
:10B66000164B1A7816F4805F02F101021A701E461A
:10B670000AD00F23059404930795FFF7CFFF2046C8
:10B6800004A905F0E5FF10E02846FFF749FF60B187
:10B690000F23049305940795FFF7C0FF204604A9E4
:10B6A00005F0D6FFFFF77AFEF1E733782046013B3D
:10B6B0002F213370FEF7C8FD09B0F0BD1D17022021
:10B6C000F0B589B006AC039004F0FEFF00F108026B
:10B6D0000346059092E803009D6A9E691F6984E80D
:10B6E000030005A804F0FEFF44F220032B40002BCA
:10B6F00034D0BFB120460399FFF766FA90B10398A2
:10B70000FFF7F8FC69070FD526B105F0010585F0B4
:10B71000010500E0012500952046124903AA0023F7
:10B7200000F0DAFA002403E00398FFF7DDF90124C2
:10B73000039804F0C9FF826A059022F4804323F045
:10B740002003920448BF43F00403836205A804F079
:10B75000C9FF054B1A88013A1A8000E01C462046B2
:10B7600009B0F0BD61AB00081017022008B504F065
:10B77000A1FF836A43F400438362024B01221A60F3
:10B7800008BD00BF9CD701202DE9F04F4C4B1B6832
:10B790009FB003B1984700264A4D2B68DBB14A4B56
:10B7A0001C68BCB1204604F08FFF826A47691EAB5B
:10B7B00012F4004F43F8700D07D0184604F092FFC2
:10B7C0002046FFF761FD3C46EBE718463C4604F097
:10B7D00089FFE6E72C603D4B1B6803B198473C4B63
:10B7E0001B682BB93B4F3B6893F8543043B103E0DF
:10B7F00098470028F6D058E003F01EFD002854D1E9
:10B800003B6893F854504DB1334B1D8835B1334BE1
:10B810001B68002B4BD01B68984701253B6893F8A9
:10B82000543013B9002D37D145E0DFF8AC80B8F8BB
:10B830000030002BF6D0DFF8A890D9F800400CB902
:10B84000214B1C6802A803F0B5FC3B68D3F830B06C
:10B85000D3F834A014B900240DE063B92046FFF7F3
:10B860002FFF03462046019304F024FF4469019B07
:10B87000002CF2D1EFE75846C9F8004003F066FC0F
:10B88000504603F061FC02A803F09EFCB8F80030BB
:10B89000002BC7D00126C1E7104B186810B14368D0
:10B8A000984708E002F02AFF05E0012674E701202E
:10B8B00002F024FFB1E730461FB0BDE8F08F00BFB3
:10B8C000041702209CD70120141702200017022021
:10B8D000801702201C0100201017022030170220C0
:10B8E000B8D70120024B1B68012283F8542070470F
:10B8F0001C010020034B1B68002283F8542002F037
:10B9000061BD00BF1C01002010B5044640682368DB
:10B91000E168172B0FD006DC0E2B0ED0142B14D1A0
:10B92000FEF7BEFE11E0222B0CD0282B0DD1BDE876
:10B930001040FFF7BEBBE06010BD2146BDE81040DF
:10B9400005F0ACBF6FF0704300E00023E36010BD72
:10B9500003680E2B10B5044602D00F2B09D020E04F
:10B96000C3685A68012A21D11868BDE8104003F065
:10B970005BBC0F4A436811688B4206D05268934201
:10B9800014BF4FF0FF33012300E00023094A52F8AF
:10B9900023006FF07043984203D003F0D5FB04F00E
:10B9A00063FA2046BDE81040FFF7AEBF10BD00BFF0
:10B9B000F81602202417022030B52B4B187885B0DA
:10B9C0001D4600284DD1294B1860294B1860294B82
:10B9D0001B685864284B1880284B04461880204662
:10B9E00004F01EF9C0B14FF0FF3202238DE80C00C5
:10B9F000002043F6FF72224B029303901346014648
:10BA0000FFF798FB1F4B43F824001F4B6FF0704269
:10BA100043F82420FFF74DFB0134022CDFD11B48F3
:10BA200005F086FF1A4805F083FF1A4805F080FFED
:10BA3000194805F07DFF194805F07AFF184805F010
:10BA400077FF104B1868FFF755FBFFF74BFF0123FB
:10BA50002B701448144B036005B0BDE8304004F06F
:10BA600013BA05B030BD00BFC4D70120141702209F
:10BA7000B8D701201C01002010170220F016022068
:10BA800051B90008F8160220241702206418022079
:10BA900054180220441802206C1802205C1802205E
:10BAA0004C180220BCD701207DA700082DE9F04FDB
:10BAB00087B0044604F008FE06AFB0F80080868820
:10BAC000B0F80290B0F806B047F8040D0FFA88F805
:10BAD00036B2C8EB0606D0F824A0013638460FFA75
:10BAE00089F90FFA8BF504F0FDFDC9EB0505002E71
:10BAF00005F101054DDD002D4BDDBAF1000F4AD0F7
:10BB0000504604F0E1FD06AB868843F8080DC58871
:10BB100036B2184604F0E6FD464502D12DB24D4539
:10BB200032D0504641464A4600F086F82CE0836AFF
:10BB300043F480338362384604F0D4FD404600F07D
:10BB400093FF0746504603F003FB404600F0B4F86D
:10BB50002D4B05FB06F219782C4D2D4E920002F06C
:10BB600021FD2046D5F800803460FEF7CCFC28602B
:10BB70002046FFF75DFD0020C5F80080306003F02F
:10BB8000E7FA384600F070FF204604F093FD406A63
:10BB900037E0002035E0FEF777FD844212D102F055
:10BBA000A3F8824602F0A8F8564502DC854209DD7A
:10BBB00000E056468542A8BF0546314620462A4643
:10BBC00005F014FE134B01934FF0010A124B029340
:10BBD0004046494632462B46CDF800A000F04EFEC6
:10BBE0008046204604F070FD0590C0F82480B8F12E
:10BBF000000F9CD1384604F075FD2046FFF718FD74
:10BC0000404607B0BDE8F08F040100204C17022029
:10BC10003C17022020CD0108F8F7010838B5054689
:10BC200005242846FFF742FF10B9013CF9D138BD81
:10BC3000BDE8384006F092BB37B50D46144618B93A
:10BC4000114B1B68186EE8B104F03EFDA4B2ADB212
:10BC5000C4808580009002F0B5FB009B586970B1EC
:10BC600004F032FD009B01901A895B898280C380B9
:10BC700012B10BB10580448001A804F033FD684681
:10BC800004F030FD03B030BD1C01002013B520B915
:10BC9000084B1B68186E044648B104F015FD02AB52
:10BCA000B0F90A4043F8040D184604F01BFD204685
:10BCB00002B010BD1C01002013B550B104F004FD0A
:10BCC000044602A840F8044D04F00CFD04F11800ED
:10BCD000FFE702B010BD00002DE9F04F1E4689B00D
:10BCE0004E4B04921A680391547C4D4A1257012A14
:10BCF00005469B46204606DD01F0E0FF074620464C
:10BD000001F0DFFF05E001F0DFFF0746204601F00C
:10BD1000DEFF044625B306A807A903F0FDFA069B3B
:10BD2000B5F900A0B5F90420B5F902801F44079BBE
:10BD30002AEAEA7A013F9742D4BFCAEB0707CAEB67
:10BD400002071C44B5F9062028EAE878013C944231
:10BD5000D4BFC8EB0404C8EB02040137013401E08E
:10BD6000A846AA4606B96642002F52DD002C50DDD7
:10BD7000129B0093504641463A46334600F038FE47
:10BD8000054620B90498039B9847012042E0FFF73D
:10BD90007DFFA042064606D0DBF80030986C10B15B
:10BDA000322105F041FC284600F05EFE7342059307
:10BDB000A1460027B14503DA2846494606F0CEFBE6
:10BDC00047B12846514607EB0802FFF735FF2846E2
:10BDD00006F0DAFB039B04989847124B1B680BB1E3
:10BDE00000209847284600F0B7FE3744059BA7423D
:10BDF0009944DFDB284600F0D9FD002000F034FE36
:10BE0000A64206D0DBF80030986C10B1332105F063
:10BE10000BFC002009B0BDE8F08F00BF1C01002022
:10BE200044170220C8D701200248012918BF00206A
:10BE3000704700BF20CD01080248162918BF002016
:10BE4000704700BF6D21010808290CBF2020002089
:10BE5000704708B50068C3681B6A984708BD37B5C6
:10BE600080680C4604F030FC034602A89988DA8802
:10BE70001D8940F8043D5B892180628029441A4471
:10BE80000139013AA180E28004F02CFC03B030BDFE
:10BE90000E4B1B6873B50546186E0E4604F014FC75
:10BEA000034602A8B3F9064040F8043D03F1180127
:10BEB000361BDC68B3F9043004FB0614ED1A04F0F9
:10BEC00011FC04EB8504204602B070BD1C0100206B
:10BED00008B508461146FFF7DBFF006808BD000003
:10BEE000154B1B6873B5186E15460E4604F0ECFB37
:10BEF000294600903046FFF7CBFF009B1B681B696B
:10BF000004469B68984723685840009B2060586906
:10BF100060B104F0D9FB02AC836844F8040D1B68DF
:10BF200031462A469847204604F0DCFB684604F078
:10BF3000D9FB02B070BD00BF1C01002073B51C46C8
:10BF4000104B1B68186E0E46154604F0BDFB2946C3
:10BF500000903046FFF79CFF009B0460586960B179
:10BF600004F0B2FB02AC836844F8040D1B68314650
:10BF70002A469847204604F0B5FB684604F0B2FB19
:10BF800002B070BD1C0100202DE9F7432C4D1E4668
:10BF90002B68186E0F46144604F096FB009040691B
:10BFA000A94608B104F090FB019021463846FFF7FE
:10BFB0006FFFD9F80020009BD16B127CD3F80C8066
:10BFC000D1F80090D20705461FD51B681B699B68F6
:10BFD00098478046019828B182683946D2F800C057
:10BFE0002246E0472B6883EA08032B60009B01345C
:10BFF000DB68B4421D44EDDD684604F073FB019B31
:10C00000D3B101A804F06EFB16E0019B63B1019867
:10C01000836822461B68394601349847B442C5F804
:10C0200000904544F3DDE7E7341B0134013CC5F8DB
:10C0300000904544FAD1DFE703B0BDE8F08300BFCC
:10C040001C0100202DE9F04FDFF8ACB01446DBF8FE
:10C05000002085B0106E0F461D4604F035FB2146CA
:10C0600002903846FFF714FF029ADBF80030D2F84E
:10C070000C90DB6B06465069D3F800A0ED1B013530
:10C0800038B304F021FB0E9A0DF11008131B48F889
:10C09000040D01330093394622462B4606F048FA38
:10C0A000404604F01FFB14E0DBF800301B7CDB078C
:10C0B00013D5029B1B681B699B68984732462B4629
:10C0C0001168013B81EA000142F8041BF8D14E449B
:10C0D00001340E9B9C42E7DD08E0002DF7DD2B4686
:10C0E0003246013B42F804ABFBD1F0E702A804F072
:10C0F000F9FA05B0BDE8F08F1C01002007B50092E9
:10C10000FFF7A0FF03B05DF804FB00002DE9F04F3E
:10C110009D4C9A46236891B08046186E07920E4651
:10C12000DDF874B01F9D002800F0878304F0CCFA7E
:10C130000E90406908B104F0C7FA0F9010A850F8AB
:10C14000083DDB680A9304F0CDFA1E9F0F98374430
:10C15000049750B123681B7C9C0706D41A9F009754
:10C160000499079A534606F0E3F904980799FFF7F4
:10C170008FFE1B9F172F064664DD4FEA8A0706973E
:10C180004FF000091A9F0F98B94557DA30B183680C
:10C19000079A5C6804994A445346A047D8F810307F
:10C1A000D86828B130465946069A0CF049FD3EE061
:10C1B0005B689847000E0590354657465C463B46FF
:10C1C00022464FF0000C52F8041B0598090E8142DC
:10C1D000059808BF0CF1010C814203F1FF3314D024
:10C1E000BCF1000F14D04FEA8C03284621461A46B2
:10C1F0000393CDF808C00CF023FD039BDDF808C0C5
:10C200001D441C44CCEB07070FE0002BDBD1E7E714
:10C210002068020EFF2A05D0D2432968D2B202F06C
:10C22000C5FA286004350434013F002FC7D11C9F94
:10C23000BB440A9F09F101093E44A3E7002840F0EE
:10C24000F982FAE21B9F102F37D1061F00251A9F93
:10C250000F9CBD4280F2A080079F2F443CB1A36891
:10C260000499D3F804C020463A465346E047ABF160
:10C27000020306930596D1460499D8F81030069A21
:10C280005B6832F8020F06925144C9EB0101039139
:10C290009847059B039943F8040F059324B1A368BD
:10C2A00020461B683A469847B9F10109E4D11C9F22
:10C2B000BB440A9F01353E44C9E71B9F082F00F18C
:10C2C00004066DD1079F07991A9A0F9C7B1A934217
:10C2D000A6F1040060DA2C4B1B681B7C6DB313F0D5
:10C2E000030305D0022B51D1B146DDF810801CE0CC
:10C2F0001BF8032055F8222040F823200133534532
:10C30000F6D143E055F8233049F8043C2CB1A3683A
:10C3100020461B6841463A469847049B08F10108AD
:10C320005344434509F1040930D00498C0EB0B0392
:10C3300013F80830002BF0D0E4E713F0030305D026
:10C34000022B23D1B146DDF8108015E05946524644
:10C350000CF076FC1AE049F8043C2CB1A3682046A6
:10C360001B6841463A469847049B08F1010853442C
:10C37000434509F1040909D00499C1EB0B0313F8F3
:10C380000830002BF0D0E6E71C0100201C9A0A9B25
:10C39000934401371E4496E7002C40F04B824CE258
:10C3A0001E9FB24B09967F000C971E9FBF000D97F2
:10C3B000079F0597002D08BF1D46099F07983C1F42
:10C3C000059F3B1A1A9FBB4280F232821B9F022FAD
:10C3D00000F0AD80042F00F04F81012F40F01E824D
:10C3E000DFF89092D9F80030186E04F06DF99BF8E0
:10C3F00000309F4A1E99D65CD9F800300E901B7C05
:10C40000DDF83CC003F00303022B5746C1F10808D6
:10C4100046FA01F620D0032B61D0012B5FD05A469B
:10C42000474538BFB846C8EB07074346214606F0E4
:10C430000100013B55F8200041F8040B4FEA560675
:10C44000F5D104EB8804002F6DD012F8013F884924
:10C450004FF00808CE5CE3E76B68DDF810900B93B3
:10C46000CDF820B0474538BFB846C8EB0707BCF148
:10C47000000F26D01EB904EB8804C14425E0F00764
:10C480000CD5DCF80830059A1B68CDF808C060466A
:10C49000494698470B9BDDF808C02360B8F10108B6
:10C4A00009F1010904F104040FD07608E2E7F1076D
:10C4B00044BF0B9B2360B8F1010804F1040404D0CD
:10C4C0007608002EF3D104EB880467B30898684A15
:10C4D00010F8013F0890D65C4FF00808C2E70368E7
:10C4E0001B699B6898475946474538BFB846C8EB13
:10C4F0000707231DC646F20704D553F8042C424013
:10C5000043F8042CBEF1010E4FEA560603F1040372
:10C51000F1D104EB880437B111F8013F544A4FF0D0
:10C520000808D65CE0E70EA804F0DCF876E11E9F70
:10C530000C9BDDF83CC0C7F104069BF800709F40DF
:10C540004C4B1B681B7C03F00303012BF6B2FFB2BC
:10C5500066D008D3022B40F061810498CDF820B05A
:10C56000D04606903EE05A4653469E42C8BFDEB2D1
:10C570009B1B314620464FEA971C013955F82CC0C9
:10C5800040F804CBBF0011F0FF01FFB2F3D1013E30
:10C59000F6B2013604EB8604002B00F03F8112F85E
:10C5A000017F0426E1E7069917F0C00F494422D124
:10C5B00009F101095FFA89F2BF009642FFB2F2D198
:10C5C000069F013EF6B27B1C721C9E1904EB82048E
:10C5D0000696B8F1000F00F02181089B13F8017F47
:10C5E000089304264645C8BF5FFA88F6C6EB0808DC
:10C5F0004FF00009D7E7BA0955F8222044F829205E
:10C60000BCF1000FD4D0DCF8082012680B92604611
:10C61000CDF808C0059A0B9B9847DDF808C0C7E71E
:10C62000584653469E42C8BFDEB29B1B221DB446ED
:10C6300017F0C00F05D052F8041C81F0FF0142F83A
:10C64000041C0CF1FF3CBF001CF0FF0CFFB202F118
:10C650000402EDD1013EF6B2013604EB8604002B54
:10C6600000F0DC8010F8017F0426DBE7E0CC010855
:10C6700060F601081C010020714A9BF80030126826
:10C680000D98127C0F9F02F003028340012ADEB254
:10C6900000F09C8002D3022A35D0BFE01E9F5FB11C
:10C6A00036090BF1010255F8263023609BF8016032
:10C6B000099C0AF1FF3301E053465A46012B1ADD6B
:10C6C000581004F1080103F0010302EB00084FEADF
:10C6D000161C06F00F0655F82C7041F8087C55F82A
:10C6E000266041F8046C12F8016F424501F108011F
:10C6F000EDD104EBC004002B00F09080360955F812
:10C70000263023608AE01E98C0B113F0F00F0AD0E3
:10C71000360955F8263023602FB1BB6804991B6891
:10C72000059A384698470499099C9BF8016001F1E5
:10C7300001080AF1FF3C0BF1010911E0D446D9468A
:10C74000DDF810800CE016F0F00F0DD116F00F069A
:10C750001BD119F8016F083408F10208ACF1020C82
:10C76000BCF1010FEFDC21E0330955F823302360E1
:10C77000002FEBD0BB68059A1B68CDF808C038467F
:10C7800041469847DDF808C0E0E755F82630636079
:10C79000002FDED0BB68059A1B68CDF808C038466C
:10C7A00008F101019847DDF808C0D2E7BCF1000F9D
:10C7B00034D0360932D055F82630236077B3BB68C1
:10C7C000059A1B6838464146984727E01E9FC7F1E7
:10C7D0000203DBB25F4652469342C8BFD3B2D21ABD
:10C7E000201D9C4616F0C00F05D050F8041C81F0A7
:10C7F000FF0140F8041C0CF1FF3C36011CF0FF0C5B
:10C80000F6B200F10400EDD1013BDBB2013304EBE1
:10C8100083041AB117F8016F0223DDE7059B1C9F03
:10C820000133BB4405930A9F099B3B440993C4E52C
:10C830000F9B13B10FA803F055FF11B0BDE8F08FA7
:10C840001C0100202DE9F3410E469046074603F0F7
:10C850003BFF036802ACDB6844F8040D5B6A002010
:10C86000162198470546204603F03CFF1DB1384687
:10C8700031464246A84702B0BDE8F0812DE9F04FAD
:10C880003E4E87B01D463368109F5B7C83468A46C8
:10C89000904611981299002203F0D4F9044600281A
:10C8A00033D003699B68984701F0CBFA08FB00F688
:10C8B0000390073604F0D0F817F001094FEAD606C6
:10C8C00004D1042390FBF3F000EB4000002D09DCC1
:10C8D0001EB11838B0FBF6F000E030466D42A842B9
:10C8E000B8BF0546B9F1000F09D1CDF80090584600
:10C8F000514642462B4605F0DBFD074600E0002787
:10C90000002D04DC204603F09BF9002032E006FBFA
:10C9100005F01830B9F1000F02D004F029F901E058
:10C9200004F0A4F9814640B9204603F089F9002FAC
:10C93000EBD0384603F002FF1BE003F0C5FE0346D0
:10C9400006A8039A40F8043D1A611C60A3F804B0DD
:10C95000A3F806A0A3F808805D81DE605F6103F0A4
:10C96000C1FE064A129B23611368C4F808905B7CE1
:10C97000A361484607B0BDE8F08F00BF1C0100204E
:10C9800037B5054670B103F09FFE036802AC1B6922
:10C9900044F8040D9B68984701F053FA0546204679
:10C9A00003F0A0FE284603B030BD000037B50446B2
:10C9B000D0B10E4B1B681B6E834201D102F0F0FB1D
:10C9C000204603F081FE0190406908B105F09CFD0E
:10C9D00002AD55F8043D186803F032F9284603F01B
:10C9E00081FE204603F0AAFE03B030BD1C010020EA
:10C9F0002DE9FF479A46194B0C9D1B680746587C4A
:10CA0000174B53F8204088469146E3681B68042B77
:10CA100006D02468002CF8D103F002F9044630B1A6
:10CA2000E3682046DB6A01219847064608B90020E2
:10CA300010E02469A3689847013004BF45F0010560
:10CA4000084C02948DE86000384641464A465346F9
:10CA5000FFF714FF04B0BDE8F08700BF1C01002001
:10CA600074170220F8F70108114BF7B51A6804464D
:10CA7000166E1F4610B902F093FB16E00EB102F0DD
:10CA80008FFBFEF737FF204603F01EFE02AD3B682A
:10CA900045F8040D1C66006803F010F9284603F001
:10CAA00021FE01F079F801F08DFC304603B0F0BDB5
:10CAB0001C0100202DE9F0430C4685B015460646C2
:10CAC000002841D0002002F01DFB214B1B680746C7
:10CAD0003046D3F8608003F0F7FD03680190986951
:10CAE00002F048FB1B4B9C42019B04BFB3F904407E
:10CAF000B3F906501A895B89ADF80840013A013B49
:10CB000022442B448146ADF80C20ADF80E30ADF830
:10CB10000A50FEF7E7FE01A803F0E4FD02A8FEF7C5
:10CB2000FFFC48B9484602F025FB4046FFF79CFF52
:10CB3000384602F0E7FA07E0304621462A4604F07C
:10CB400083FFFEF72BFCECE705B0BDE8F08300BFE8
:10CB50001C01002001F0FFFF01490A46FFF7AABFB0
:10CB600001F0FFFFF8B504460E46D0F88C302A21BC
:10CB700015469847E16AD4F8903031442046C1F315
:10CB80000F219847E16AD4F89030B7B23944204673
:10CB9000C9B29847E16AD4F8903031442046C1F3D5
:10CBA0000F219847E16AD4F8903039442046C9B241
:10CBB0009847D4F88C3020462B219847216BD4F825
:10CBC000903029442046C1F30F219847216BD4F8B7
:10CBD0009030AEB231442046C9B29847216BD4F8A8
:10CBE000903029442046C1F30F219847216BD4F897
:10CBF000903031442046C9B29847D4F88C30204652
:10CC00002C219847F8BD2DE9F041044688461F467F
:10CC10002A21D0F88C30069D16469847E16AD4F850
:10CC2000903041442046C1F30F219847E16AD4F87F
:10CC3000903041442046C9B29847E16AD4F8903018
:10CC400039442046C1F30F219847E16AD4F8903067
:10CC500039442046C9B29847D4F88C3020462B215D
:10CC60009847216BD4F8903031442046C1F30F210E
:10CC70009847216BD4F8903031442046C9B2984788
:10CC8000216BD4F8903029442046C1F30F219847F6
:10CC9000216BD4F8903029442046C9B29847D4F883
:10CCA0008C3020462C219847BDE8F08113B50D4A01
:10CCB0000446516810686B4603C3D4F88C30204694
:10CCC00036219847636BA18C02AA134421F0E0013E
:10CCD00013F8083C19432046D4F8903089B298479D
:10CCE00002B010BDE4F5010813B50446D0F80C31CC
:10CCF0002E209847216AD4F8283168460331984796
:10CD0000226A00AB13441DF8022059789878D208A3
:10CD10008908D20242EA411242EAD00002B010BDB4
:10CD20001FB50446D0F82C312E209847216AD4F83C
:10CD30004831684602319847236A00A901EB430253
:10CD40003DF81300528802F47C41C2F3C40242EA67
:10CD5000511200F0F80042EA002004B010BD38B5CE
:10CD600004460D46D0F80C31080A9847D4F80C3127
:10CD7000E8B2984738BD08B5D0F82C310846984736
:10CD800008BD08B5D0F81031C8B2984708BD08B53D
:10CD9000D0F830310846984708BD0000082902D075
:10CDA000102905D07047064BC0F88C30054B03E0C6
:10CDB000054BC0F88C30054BC0F89030704700BF71
:10CDC0005FCD000883CD000877CD00088FCD000827
:10CDD000F0B585B084680A9F0097BD1A581A0135CE
:10CDE00000FB0555D4F8A8700B9E2046B847D4F830
:10CDF0000C312E209847D4F82831216A02A8984790
:10CE0000D4F8283102A8032198479DF808309DF8EE
:10CE10000920DB089208DB0243EA42139DF80A204E
:10CE2000013D43EAD20326F8023BE9D105B0F0BD4B
:10CE3000F0B587B084680C9F0097BD1A581A013569
:10CE400000FB0555D4F8A8700D9E2046B847D4F8CD
:10CE50002C312E209847D4F84831216A02A89847EF
:10CE6000D4F8483102A802219847BDF80A3003F4EB
:10CE70007C42C3F3C40343EA5213BDF8082002F016
:10CE8000F80243EA0223013D26F8023BE8D107B04D
:10CE9000F0BD000010B5044600F0A6FDA368124ADC
:10CEA000C3F8AC20114AC3F8A820114AC3F8B02037
:10CEB000104AC3F8B8200022C3F8BC20C3F8CC2025
:10CEC0000D4A0E491268C3F8C420DA8C0968C3F809
:10CED000B41022F003020A49DA840A4AC3F8C810DF
:10CEE000C3F8942010BD00BF65CB000807CC000834
:10CEF000ADCC0008E9CC00080C010020080100209E
:10CF0000D1CD00089DCD000808B5D0F8B4309847C1
:10CF100008BD08B5D0F8303188B2984708BD000088
:10CF20002DE9F04F3D4F846882463868007C10F050
:10CF3000010F85B00E4615469846C1EB030945D052
:10CF40004FEA490B0E98854265DCD4F8C4C0E76E01
:10CF5000BCF1000F01D1B44607E08DE8A0005046B7
:10CF600031462A464346E04711E0C4450EDCD4F87A
:10CF7000EC30CDF80CC0614650462A469847DDF8A3
:10CF80000CC027F8020B0CF1010CEEE7E76EBB1E9C
:10CF900009F1010C5F44BB4205D0A26A59884A409E
:10CFA00023F8022FF7E700952A46D4F8A870CDF8A9
:10CFB0000CC0204631464346B847DDF80CC0D4F8D3
:10CFC0003831E06E614698470135BBE70E98009016
:10CFD000851AD4F8A8602046B0473B68A76EDB6B83
:10CFE00009F10109D3F8008005FB0995012395B1EA
:10CFF000FA2D34BF2E46FA262BB138461FFA88F197
:10D00000324601F0A1FAD4F8383138463146984713
:10D01000AD1B0023EBE705B0BDE8F08F1C0100203D
:10D020002DE9F04F8DB08568179F05937B1E012B6E
:10D03000099008910A920B9503D9042F01D0082F6B
:10D0400006D18F4B1B681B7C03F00303022B10D00F
:10D050000A9A169F1A9D0899059B3A442944013A59
:10D060000B9D00920B44D5F8A8400A9A2846013B34
:10D07000A047DDF828B00A9F169DC7EB0B03AB4213
:10D0800080F25182179F7B1E0F2B00F24582DFE852
:10D0900013F01000B7004302400143024302430271
:10D0A000D7014302430243024302430243024302C5
:10D0B0003D02734B099D1B68AC681B9D1B7C2F6850
:10D0C0006D680795DDF820A01A9D03F00303022B7D
:10D0D000AA441BD0032B6ED0012B6CD0059EDDF82B
:10D0E000648098F80010D4F8303180222A4111422F
:10D0F00016BF0799B8B288B201359847082D04BF0A
:10D1000008F101080025013EEBD105E2199D0695C5
:10D11000D4F86C90DDF86880CDF80CA00025564658
:10D120002B46069F4FF0800C3A784CFA08FC12EA26
:10D130000C0C0BD013B9D4F86C900396079FA9F888
:10D140000070013509F10209012317E0012B14D108
:10D15000CDF800B0CDF810C020460399D4F8A870DF
:10D160005A46731EB847D4F83831E06E29469847BE
:10D17000DDF810C06546634600E0634608F101082B
:10D18000B8F1080F06F1010604D1069F0137069792
:10D190004FF00008059A5244B242C2D1059F7B1E4F
:10D1A0005344002D00F0B881CDF800B0D4F8A86049
:10D1B000039920463DE1DDF814801A9E199DDDF8A3
:10D1C00014902A7880233341D1441A42C8EB0909CC
:10D1D0000DD0D4F8EC30099849465A469847A36ACE
:10D1E000D4F8F0704340494609985A46B84701368A
:10D1F000082E04BF01350026B8F10108DFD18BE10C
:10D20000099D1B9FAC68002F00F086811C4B199D67
:10D210001B6895F800A01B7C13F0030311D0022BB0
:10D2200040F07A811A9DDDF82090E76E0397A944BB
:10D23000A846199D07950025CDF818904E462B4617
:10D2400040E01A9D059E199FC5F103035B00C3F1E1
:10D250000602C02141FA02F202EA0A02DA401B99F0
:10D26000D4F8303131F8220001359847042D03D12C
:10D2700097F801A000250137013EE5D14CE100BF40
:10D280001C01002013B9E76E039706961B9F57F801
:10D290002C30039F3B80023701350397012308F1AF
:10D2A0000108B8F1040F06F1010606D1079F97F8AF
:10D2B00001A0013707974FF00008059A4A44B2428F
:10D2C00000F0AC80C8F103025200C2F106014FF039
:10D2D000C00C4CFA01FC0CEA0A0C3CFA02FCD1D15D
:10D2E000012B14D1CDF800B0CDF810C0204606991E
:10D2F000D4F8A8705A46731EB847D4F83831E06E97
:10D3000029469847DDF810C065466346C7E763467F
:10D31000C5E7099D1B9FAC68002F00F0FD80834B83
:10D32000199D1B6895F800A01B7C13F0030311D016
:10D33000022B40F0F1801A9DDDF82090E76E0397F4
:10D34000A944A846199D07950025CDF818904E468A
:10D350002B463CE01A9D059E199FC5F101039B00D9
:10D36000C3F10402F02141FA02F202EA0A02DA40B1
:10D370001B99D4F8303131F8220001359847022D3D
:10D3800003D197F801A000250137013EE5D1C3E0A4
:10D3900013B9E76E039706961B9F57F82C30039F2F
:10D3A0003B80023701350397012308F10108B8F1EA
:10D3B000020F06F1010606D1079F97F801A0013779
:10D3C00007974FF00008059A4A44B24226D0C8F1A8
:10D3D00001029200C2F104014FF0F00C4CFA01FC82
:10D3E0000CEA0A0C3CFA02FCD2D1012B14D1CDF884
:10D3F00000B0CDF810C020460699D4F8A8705A465F
:10D40000731EB847D4F83831E06E29469847DDF8E6
:10D4100010C065466346C8E76346C6E7059F7B1EA6
:10D420004B44002D78D0CDF800B0D4F8A860069910
:10D4300020465A46B047D4F83831E06E29466AE0B3
:10D44000099D1B9FAC68002F66D0384B1B681B7C66
:10D4500013F0030309D0022B5ED1DDF82090D4F83D
:10D460006C8000264F46334622E0199D199B059F8C
:10D470003B445B1B002B4FDD15F8012B1B9FD4F8A1
:10D48000303137F822009847F0E713B9D4F86C80B0
:10D49000B9461B9D55F82A30A8F80030013608F12E
:10D4A00002080123089A059D01372A44BA421CD07C
:10D4B000199D08982A1A12F807A0BAF1000FE4D1B2
:10D4C000012B10D1CDF800B0204649465A467B1EAC
:10D4D000D4F8A850A847D4F83831E06E31469847C0
:10D4E00056465346DEE75346DCE7089F6B1E3B4437
:10D4F00096B1CDF800B020464946D4F8A8505A4617
:10D50000A847D4F83831E06E314604E00B9D1998F5
:10D51000D5F8383105999847199F189D2F441997C8
:10D520000BF1010BA7E50DB0BDE8F08F1C01002049
:10D5300010B5044600F058FAA468104BC4F8E43063
:10D540000F4BC4F8E8300F4BC4F8EC300E4BC4F866
:10D55000F0300E4BC4F8A0300D4BC4F8A430D4F812
:10D56000C430C4F8FC302046D4F8943010219847D9
:10D570001023A363074B636410BD00BF21D00008D4
:10D5800021CF000837D90008A7D8000809CF000824
:10D5900013CF000884F80108084670470068401A55
:10D5A00001387047084670470068401A01387047D4
:10D5B000104670474068801A01387047104670471F
:10D5C0004068801A0138704710467047104670470F
:10D5D0004068801A013870474068801A01387047E7
:10D5E00008467047084670470068401A013870477F
:10D5F0000068401A0138704710B58468D4F8F040CC
:10D60000A04710BD08B58368D3F8EC30984708BD33
:10D61000F7B504460F4616468568FFF7F3FF0190FD
:10D62000DDF804E0AB6A2046394632468EEA030351
:10D63000FFF7E2FF03B0F0BD13B584680092D4F8A1
:10D64000E840A04702B010BD13B584680093D4F839
:10D65000E8400B46A04702B010BD37B5069C856870
:10D660000094D5F8E840A04703B030BD30B587B08E
:10D6700085680A9C00940B9C01940C9C02940D9C60
:10D6800003940E9C04940F9C0594D5F8E440A047A5
:10D6900007B030BD7047000073B5079E84680C4D1D
:10D6A00076B1286888B906980090D4F8A86020461A
:10D6B000B047D4F8A8302B60064BC4F8A83004E07B
:10D6C0002B6813B1C4F8A8302E6002B070BD00BF43
:10D6D000CCD7012095D6000808B5026CD0F8D4301C
:10D6E0009069984708BD08B5026CD0F8D8309069A9
:10D6F000984708BD2DE9F7430A9D846800951746B1
:10D700002046D4F8A86099468846ED1BB047216CA6
:10D71000D4F8DC3088690B99C8EB09086A1C08FB4F
:10D720000222984703B0BDE8F0832DE9F7430A9D34
:10D730008468009517462046D4F8A8609946884624
:10D74000ED1BB047216CD4F8E03088690B99C8EB29
:10D7500009086A1C08FB0222984703B0BDE8F08361
:10D760000139172924D8DFE801F0102323232323CC
:10D770002323230C250E1523232323232323231FB5
:10D780001A210D4870470D48704703689B68D3F80D
:10D79000FC00704703689B68D3F8F4007047036887
:10D7A0009B68D3F8F80070470548704705487047F4
:10D7B000002070470448704717DB0008B9DA0008FA
:10D7C0001DDA000899D6000803DB000801398068DB
:10D7D0000D2923D8DFE801F0090B0D0F22222211B9
:10D7E00007252513181D0020704700687047406802
:10D7F000704780687047C0687047806B704788B119
:10D80000406B00F00100704760B1406BC0F3400016
:10D81000704738B1406BC0F3800070474FF0FF3065
:10D82000704701207047836801290CBF586C0020A5
:10D830007047836800220A804A801A685B68013A50
:10D84000013B8A80CB807047F0B5104D2E460746CD
:10D850000FCE91B06C460FC496E80F00203584E8D7
:10D860000F000FCD08AC0FC495E80F0084E80F003F
:10D870007B6B10AA02EB830353F8402CC7F80021FE
:10D8800053F8203CC7F8043111B0F0BDECF50108A5
:10D8900007B580698DE8060003216A46F2F776FF36
:10D8A00003B05DF804FB2DE9F74384689846E38CE8
:10D8B0009B078946174632D5D4F800312046984751
:10D8C000D4F8045106463A4620464946A8472369FB
:10D8D000A2699E42ACBF002301239642D4BF1A46E0
:10D8E00043F0010263699842ACBF134642F0010362
:10D8F000054613B9E36998420ADD62682368013A74
:10D9000000920021D4F8A87020460A46013BB8478F
:10D91000D4F8AC70204631462A46B84703E0D4F824
:10D92000AC502046A847D4F8A4302046414698473A
:10D9300003B0BDE8F083F7B58468E38C9B070F461E
:10D94000164645D5D4F8003120469847D4F804311E
:10D9500032460546394620469847D4F89830064660
:10D960001BB120460121002298472369A2699D42EC
:10D97000ACBF002301239542D4BF1A4643F00102F5
:10D9800063699E42ACBF134642F0010313B9E369D9
:10D990009E420ADD62682368013A00920021D4F8B1
:10D9A000A87020460A46013BB8472946D4F8AC3057
:10D9B000204632469847D4F8A03020469847D4F8FD
:10D9C000983005466BB1204600210122984708E0B7
:10D9D000D4F8AC3020469847D4F8A0302046984779
:10D9E0000546284603B0F0BD38B58568044695B9AC
:10D9F0004FF4BA7002F0C0FF4FF4BA72A06029462B
:10DA000000F0D0FDA3680222DA8401221A62024AE1
:10DA10001C64C3F8082138BD49D8000870B5064613
:10DA20000D461446FFF7E0FFB368002B3BD0262DD0
:10DA300002D0272D16D070BD9A6B102A02D0122A60
:10DA400008D070BD184AC3F8D440C3F8B820C3F852
:10DA5000B42070BD154AC3F8D840C3F8BC20C3F841
:10DA6000C02070BD9A6B102A02D0122A0ED070BD51
:10DA70003CB10F4AC3F8DC40C3F8C820C3F8C42047
:10DA800070BDC3F8C840C3F8C44070BD3CB1094A7A
:10DA9000C3F8E040C3F8CC20C3F8D02070BDC3F871
:10DAA000CC40C3F8D04070BDD9D60008E7D60008F6
:10DAB000F5D600082BD7000838B50546FFF794FFC8
:10DAC000AC684FF4FA7002F057FFA36BA0660733FF
:10DAD000D8102368584302F04FFF01210022E0666E
:10DAE000A869F2F753FED4F8083105462046984756
:10DAF0002046D4F8B0309847002DD4BF0020012034
:10DB000038BD70B504460D461646FFF76DFFA36895
:10DB100083E8600070BD70B504460D461646FFF7F9
:10DB200063FFA3689D60DE6070BD38B505460C4696
:10DB3000FFF75AFFAB682268DA6262681A63A2686C
:10DB40005A63520707D593E806001A605960DA68ED
:10DB50009968D9609A60A2899A84226912B122EAEE
:10DB6000E2721A6238BD2DE9F04104461F4616469E
:10DB70008846FFF739FFA5684146682205F586709B
:10DB80000BF05EF82046B0472046B84723699B68F3
:10DB90009847A862BDE8F08110B5074C2368186B60
:10DBA00000F06AFC00F088FC2368586B00F064FC0D
:10DBB000BDE8104000F09CBC1C01002037B5094CAA
:10DBC00023685A7C084B054653F82200C268694610
:10DBD000126B9047206829466A46083000F096FD8F
:10DBE00003B030BD1C0100207417022037B50D466C
:10DBF000144602F015F8019008B901200CE0C36842
:10DC00000A215B6A01A8984703460028F5D00198CD
:10DC1000294622469847002003B030BD37B50D464F
:10DC2000144601F0FDFF019008B901200CE0C36823
:10DC30000B215B6A01A8984703460028F5D001989C
:10DC4000294622469847002003B030BD37B50D461F
:10DC5000144601F0E5FF019008B901200CE0C3680B
:10DC600010215B6A01A8984703460028F5D0019867
:10DC7000294622469847002003B030BD012810B540
:10DC80000C4608DC01F0CCFF20B1C36821469B6A3A
:10DC9000984710BD10BD002010BD38B50446214680
:10DCA0000120FFF7EBFF214605460020FFF7E6FFC6
:10DCB000A842B8BF284620EAE07038BD0121FFF72E
:10DCC000DDBF0221FFF7DABF0321FFF7D7BF042131
:10DCD000FFF7D4BF0821FFF7D1BF0921FFF7CEBF5F
:10DCE0000E21FFF7CBBF0000024B1B68587CFFF7EB
:10DCF000E5BF00BF1C010020024B1B68587CFFF7EA
:10DD0000E0BF00BF1C010020024B1B68587CFFF7DE
:10DD1000E4BF00BF1C010020024B1B68587CFFF7CA
:10DD2000DFBF00BF1C01002008B5044B53F82000E2
:10DD3000C36808219B6A984708BD00BF741702207A
:10DD400008B501F06DFF20B1C3680221DB6A984776
:10DD500008BD08BD024B1B68587CFFF7F1BF00BF30
:10DD60001C010020024B53F820301B695868704793
:10DD700074170220024B53F820301B691868704753
:10DD8000741702200120FFF788BF0220FFF785BF2C
:10DD90000320FFF782BF0000024B1860024B19609E
:10DDA000704700BFD4D70120D0D70120014B18689D
:10DDB000704700BFD4D70120014B1868704700BFDF
:10DDC000D0D7012000283BD030F0010329D030F01B
:10DDD000030328D030F0070327D030F00F0326D0FC
:10DDE00030F01F0325D030F0FF0324D020F4FF7360
:10DDF00023F001030BB320F47F6323F00F03E3B19F
:10DE000020F4FF4323F07F03BBB1030C1B04A3B139
:10DE1000830C9B049BB110F07F4F0CBF1820202077
:10DE2000704701207047022070470320704704208C
:10DE30007047052070470820704710207047122057
:10DE4000704708B5FFF7BEFF01280FD0831E062BD1
:10DE500009D9A0F10903072B07D91138102834BFBD
:10DE60002020002008BD082008BD102008BD0000AB
:10DE700070B5084B1B681A7C80EA0201490705D57A
:10DE80009C6BD96B26680D6825600E60187410466F
:10DE900070BD00BF1C01002008B5024B1B689B68C9
:10DEA000984708BD1001002038B5144B1B680A467E
:10DEB000B3F90A108A4204461EDBB3F90E108A42F7
:10DEC0001ADCB3F90810884216DBB3F90C1088424B
:10DED00012DC197C587C11F0010F094951F820001F
:10DEE00004D0C3682146DB69984738BDC168DB6B45
:10DEF0008D691B682146A84738BD00BF1C01002062
:10DF00007417022038B5104B1C68B4F90A309942D6
:10DF10000D4617DBB4F90E30994213DCB4F9081042
:10DF2000B4F90C308842A8BF01469A42B8BF1346E4
:10DF30008B4207DB607C054A52F82000C268946877
:10DF40002A46A04738BD00BF1C01002074170220DC
:10DF500038B5104B1C68B4F9083005469D42104690
:10DF600017DBB4F90C309D4213DCB4F90A20B4F984
:10DF70000E309142A8BF0A469842B8BF034693426A
:10DF800007DB607C044951F82000C168CC68294651
:10DF9000A04738BD1C0100207417022073B50E463F
:10DFA00012490C68B4F90810B4F90C508842A8BFA3
:10DFB0000146AA42B8BF15468D4214DBB4F90A20C7
:10DFC000B4F90E009642A8BF32468342A8BF03466A
:10DFD000934208DB647C064850F82400C468009330
:10DFE00024692B46A04702B070BD00BF1C01002071
:10DFF000741702202DE9F04FDFF8ACC18FB0DCF8C8
:10E0000000C009900E4615469B461C9CDDF87880A2
:10E01000BCF1000F0DD0189D199E009501961A9F16
:10E020001B9D1D9E0297039504940596DCF8004005
:10E0300053E0189F199847EA0003012B4FD1584B22
:10E040001868B0F90A20511A002908DDC1EB0B034A
:10E05000002B40F3A2801B9F07FB014401E05B46BD
:10E0600032465E44B0F90E10013E761A002E03DDF2
:10E070009B1B002B40F391800999B0F90C60294457
:10E080000139891B099E0029C8BFC1EB0505C8EBF2
:10E090000601B0F90860B1420CDAC1EB060C08EBDE
:10E0A0000C078E1B2CF0070C354404EBE70461448D
:10E0B00007F00708002D70DD467C3A481A9F50F89B
:10E0C0002600C668019703941B9F1D9C009302972E
:10E0D000CDF81080059474682B46A0475DE01A9F28
:10E0E000C7F108070C976746DC4556DA2C4B1998A0
:10E0F0001B683044B3F90A200A90411E91420B91EB
:10E1000045DBB3F90E309E4241DC4FF00008DDF8EC
:10E1100024900894C246AA4539DAB8F1000F05D117
:10E12000089A1778013208924FF008080C981A994B
:10E130001B4A47FA00F3C1EB08088F4013F0FF01B8
:10E14000FFB203D11068007C80071BD41268D26B29
:10E1500010680D901D9810B150F8213000E0DBB22E
:10E16000189913604A1E4A440B9BCDF81CC04846C0
:10E170003146FFF713FF0A4B0D9A1B68DDF81CC0F0
:10E18000DB6B1A60189B0AF1010A9944C3E71B9ED6
:10E190000CF1010C34440A9EA6E70FB0BDE8F08FE5
:10E1A0001C01002074170220481702202DE9F04FAF
:10E1B000DFF80CC291B0DCF8009007920546884663
:10E1C0009B461C9E1E9CB9F1000F0CD01A9D1B9FF4
:10E1D000009501971D9D1F9F029603950494059736
:10E1E000D9F8004081E01A9F1B9847EA0003012BF1
:10E1F0007DD1714B1868B0F90A20531A002B08DD45
:10E20000C3EB0B01002940F3D4801D9F07FB03449F
:10E2100001E059464246D844B0F90E3008F1FF38C3
:10E22000C3EB0808B8F1000F04DDC8EB01010029B9
:10E2300040F3BF80079BB0F90CC02B44013BCCEBF3
:10E240000303002B02DD079FFF1A0797B0F908C0F0
:10E25000654533DA079FC5EB0C03FF1A082E0797B5
:10E2600027D00DDC022E14D0042E1AD0012E26D178
:10E2700023F0070C04EBE304654403F007031EE0FE
:10E28000182E18D0202E16D0102E18D104EB4304CF
:10E2900013E023F0030C04EBA304654403F0030331
:10E2A0000DE023F0010C04EB6304654403F001036B
:10E2B00005E01C4401E004EB830465460023079F4E
:10E2C000002F76DD90F811E03C481D9F50F82E009D
:10E2D000D0F80CE003948DE842001F9C0493029751
:10E2E0000594DEF80440079B2946A04761E0C6F18B
:10E2F00008070E97CDF828900A9F5F4559DA2E4BF4
:10E300001B9F1B684744B3F90A200C97013F9742B3
:10E310000D9746DBB3F90E30984542DC4FF0000A0A
:10E320000B94AC465746079887423ADABAF1000F89
:10E3300006D10B9890F8009001300B904FF0080A2E
:10E340000E991D4A49FA01F313F0FF0109FA06F983
:10E350005FFA89F9C6EB0A0A03D11068007C8007CE
:10E360001BD41268D26B10680F901F9810B150F830
:10E37000213000E0DBB21A9913604A1E6244604605
:10E380000D9BCDF820C04146FFF708FE0A4B0F9ABF
:10E390001B68DDF820C0DB6B1A601A9B01379C44B8
:10E3A000C1E70A9FDDF8308001370A971D9F3C4482
:10E3B000A2E711B0BDE8F08F1C0100207417022005
:10E3C0004817022008B5054B1968054B4A7C53F8DD
:10E3D0002200C36808311B6B984708BD1C01002050
:10E3E0007417022037B5FFF7EDFF04F02DFF044648
:10E3F00000283DD10546284601F012FC019048B1A5
:10E40000C3680C215B6A01A89847034670B3019862
:10E41000984704430135022DEDD14CBB04F030FF89
:10E420000124204601F0FCFB0190D0B1204600F011
:10E43000A1FE0420FFF730FD43F6FF7200200146E5
:10E440001346FFF7ABFD0020FFF726FD02A80E21C3
:10E4500050F8043DDB685B6A9847034608B10198B1
:10E46000984714F1FF34DCD2002002E0012000E0E4
:10E47000204603B030BD000008B5054B1B685A7C30
:10E48000044B53F822301B691B68984708BD00BF36
:10E490001C0100207417022008B5054B1B685A7C2C
:10E4A000044B53F822301B695B68984708BD00BFD6
:10E4B0001C01002074170220044B1B681A7C5207B1
:10E4C0004CBF9B6BDB6B1860704700BF1C010020CA
:10E4D00008B5064B1B68196B814206D01863FFF71D
:10E4E000CBFFBDE80840FFF7E7BF08BD1C010020D7
:10E4F000044B1B681A7C52074CBFDB6B9B6B18608C
:10E50000704700BF1C01002008B5064B1B68596B03
:10E51000814206D05863FFF7AFFFBDE80840FFF720
:10E52000E7BF08BD1C01002008B5024B1B685B68F3
:10E53000984708BD1001002008B5024B1B681B68F6
:10E54000984708BD1001002070B5840702D50180EE
:10E55000013A023055082B4605B3032D01EB014467
:10E5600002DC06461D4612E003462E46043E032EFC
:10E570001C605C609C60DC6003F11003F6DC043D11
:10E58000AB085E1C00EB0610A5EB8303E9E71DB1A9
:10E5900046F8044B013DFAE700EB8300D30748BF80
:10E5A000018070BD70B52AB1830703D000F8011B4C
:10E5B000013AF8E7930801D1024417E04FF0013423
:10E5C00002F003024C43032B054606DD0460446061
:10E5D0008460C460043B1030F5E71E461BB145F86B
:10E5E000044B013BFAE700EB8600E5E7904202D0DE
:10E5F00000F8011BFAE770BD0B8892B21344038048
:10E600008B889B1A83804B8813444380CB889A1A4B
:10E61000C28070470128F7B504460D4665DC344BCF
:10E620001B6803B19847012D04D0022D21D0002D85
:10E630005BD135E02F4E56F82470B7B9204601F073
:10E64000EFFA0190002850D0C3680D215B6A01A841
:10E6500098470346002848D001982946984756F81D
:10E660002430013346F8243018E0013746F824708E
:10E670003BE0204601F0D4FA0190002835D0C36871
:10E680000D215B6A01A89847044600282DD01A4B3B
:10E690001B6803B1984701980221A047002025E09C
:10E6A000144D55F82430012B01D0012015E02046EF
:10E6B00001F0B6FA01900028F7D0C3680D215B6A1B
:10E6C00001A8984706460028EFD00B4B1B6803B102
:10E6D000984701980021B047002055F82430002BBE
:10E6E00018BF013B45F8243000E0012003B0F0BD25
:10E6F000E4D70120DCD70120D8D70120024B1B68CA
:10E700000146587CFFF786BF1C01002070B5B2F9A6
:10E710000030B1F90040B1F90250B1F90460B1F92B
:10E7200006109C42B8BF1C46B2F902309D42A8BFF9
:10E730002B46B2F90450B2F90620AE42B8BF3546B6
:10E74000A4B2ADB29142B8BF0A460480858024B21B
:10E750002DB29BB292B2A5424380C28006DB10B2BA
:10E760001BB29842B4BF0020012070BD002070BDD4
:10E770000B8810B5B0F900401AB29442B8BF0380BC
:10E780004B88B0F902401AB29442B8BF43808B88DC
:10E79000B0F904401AB29442C8BF8380CB88B0F964
:10E7A00006101AB29142C8BFC38010BD01F07F436A
:10E7B000B3F17F4FF0B527D0D343DBB2CDB2C6B2B1
:10E7C0005D4302FB065501F47F4600F47F445E433F
:10E7D00002FB046601F47F0400F47F075C43090E2A
:10E7E000000E02FB07444B43360A02FB0032240AA8
:10E7F000C5F3072306F47F401843120404F47F0393
:10E80000184302F07F421043F0BD000070B50A4C7F
:10E810000A4D20680A4E01F043FF286801F040FFCE
:10E82000306801F03DFF074A00231360064A336059
:10E830002B602360136070BDECD70120E8D7012066
:10E84000F0D70120F4D7012004D801202DE9F843A6
:10E850001C46284B17461A680646884632B90122DC
:10E8600025481A60254B036001F00EFB244D2B68F0
:10E8700033B9244B1B682B6013B9FFF789FA286062
:10E880000CB12B68236096B11F4B1A68994600247F
:10E890004AB92868800002F06FF8D0F10104C9F885
:10E8A000000038BF0024D9F80030336000E034465F
:10E8B000B8F1000F0DD0154E33683BB928688000C1
:10E8C00002F05AF80028306008BF01243368C8F805
:10E8D000003067B10E4E33683BB92868800002F003
:10E8E0004BF80028306008BF012433683B602046A5
:10E8F000BDE8F88304D80120FCD701200DE800080A
:10E90000F4D701207C170220ECD70120E8D70120A2
:10E91000F0D701202DE9F04F93B000241D9E0B90FD
:10E920000C9190461F4634600FA810A9224611ABE7
:10E93000FFF78CFF0546002840F0C380634C119A16
:10E940002368587C624B53F8203007939742A8BF46
:10E9500017461A690D920A97FFF7E6F9236808909F
:10E96000587CFFF7FFF95B4B0490984205D05A4B57
:10E97000C31A18BF0123069300E0069500250A9CE0
:10E98000AB4643461C9A53F8040B05939047030E7D
:10E990008146099300F08580BBF1000F3FD14B4BBE
:10E9A0000B9F1B680A9AB3F90830DDF82CC00C994C
:10E9B0002F44BB42C8BFC7EB030B0BEB050AC8BF14
:10E9C0001F460F9B4FEA8A0A534494440093079BC7
:10E9D00001930CF1FF3238460B46CDF80CC004F021
:10E9E000F9FB089A0F98DDF80CC0172A06DC504492
:10E9F000CBEB04010D9B04F093FC01E0069B13B9E3
:10EA00004FF0010B0BE0C7EB0C078244DAF8000073
:10EA1000049A9047013F4AF8040BF7D1F0E72F4BD7
:10EA20000F99D3F800C0109F4FEA850ABCF1000F80
:10EA300024D007EB0A025144109223460F9140461E
:10EA4000E0470F9D109A002358F8031001F07F4013
:10EA5000B0F17F4FE85801D1D05005E000F07F4081
:10EA6000B0F17F4F08BFD150013C03F10403EBD15B
:10EA70003368109743F00103336020E0099BFF2BBC
:10EA800004D151F80A3047F80A3011E0099B51F8D7
:10EA90000A10DA434846D2B2FFF788FE47F80A0068
:10EAA00002E0109B43F82500336843F00103336014
:10EAB000013C05F1010502D0DDF8148061E71098F2
:10EAC00000E0204613B0BDE8F08F00BF1C0100201D
:10EAD000741702201F0E01081D0E0108F8D701202F
:10EAE0001FB508B103AA00E0024601A802A900234D
:10EAF000FFF7ACFE05B05DF804FB000008B5024B63
:10EB00001B6803B1984708BD08D80120B5EEC00ABC
:10EB1000F1EE10FADFED0D7A48BFB1EE400A30EEAB
:10EB2000270A0020B5EE400AF1EE10FA0CD0F2EE02
:10EB3000047A20EE270A0130FCEEC07AC0B217EE4C
:10EB4000903A002BF3D07047704700BF5F70893058
:10EB5000B5EEC00AF1EE10FA08B5F6EE007A0AD565
:10EB600070EE677A17EE900A08F028FC41EC100B63
:10EB700007F0B6FB09E070EE277A17EE900A08F06E
:10EB80001DFC41EC100B07F02BFC51EC100B08F0B6
:10EB9000F5FC00EE100A08BD0E4B53F8213007EECD
:10EBA000903AF8EE677A70B520EE270A05460C46D3
:10EBB0001646FFF7CDFFBDEEC00A294610EE100A3B
:10EBC00022461EB1BDE8704000F0AEB8BDE870400E
:10EBD00000F09DB8B8F7010838B5B5EE400AF1EE7F
:10EBE00010FA2DED028B0446B0EE408A0D4652D04D
:10EBF000B5EEC00AF1EE10FA24DBF7EE008AB4EEAF
:10EC0000E80AF1EE10FA1DD5FFF780FFA04202DC02
:10EC100078EE287A46E0F6EE007AB4EEE78AF1EE76
:10EC200010FA09DBDFED367A002C18BFF0EE687AB7
:10EC300008BFB0EE688A35E044B3F0EE687A9FED25
:10EC4000308A2FE0B5EEC08AF1EE10FA28D5FFEE3B
:10EC5000008AB4EEE88AF1EE10FA21DDB0EE480A3F
:10EC6000FFF754FFA04204DCF7EE007A78EE677AF3
:10EC700018E0FEEE007AB4EEE78AF1EE10FA03D85F
:10EC80004CB9B0EE688A0BE044B104E0DFED1C7AC9
:10EC9000B0EE678A06E0F7EE007A03E09FED188A8F
:10ECA000F0EE487A174B53F8243000EE103AB8EEE5
:10ECB000400A27EE800AFFF74BFFBDEEC00A10EEB8
:10ECC000100A01F061FF012DC4EB000020EAE070A2
:10ECD00005D1B5EEC08AF1EE10FAC8BF0130B0EE32
:10ECE000480ABDEC028B002C0CBF2346631C184461
:10ECF00021462A46C0B2BDE83840FFF74DBF00BFED
:10ED000000000000B8F701080021FFF765BF1FB53C
:10ED100004AB01AC43F8104D6B4601F059FF20469F
:10ED200000F0FAFE04B010BDF0B585B004AC0D469D
:10ED300001AE6946174644F8106D01F03DFF00280A
:10ED4000C4BF05F1FF35EDB229463A466B4601F0E6
:10ED50003FFF304600F0E0FE05B0F0BD034A00235F
:10ED60001360034A1360034A136070470CD80120F4
:10ED700010D801201CD801202DE9F043194B1F6841
:10ED800085B000259846D8F80030164C33B300F013
:10ED900091F90646206801F097FC034604A85969DA
:10EDA00040F8103D891B002913DC2168039101966E
:10EDB00019695E68029168462660D3F8009001F0F8
:10EDC00091FC01A8C8474EB12368BB4205D001257C
:10EDD000D9E7684601F086FC00E00025284605B02A
:10EDE000BDE8F08310D80120F0B5254C85B005466C
:10EDF00001F06AFC2368019013B92560436039E093
:10EE0000184601F061FC04AB466943F8100D6846F2
:10EE100001F068FC019B5A69921B002A03DC2268FE
:10EE20005A60256026E02668304601F04DFC04ACAF
:10EE3000466844F8080DBEB1304601F045FC04AB0D
:10EE4000476943F8040D184601F04CFC019A5369D8
:10EE5000DB1B002B029B02DC56605D6007E0204656
:10EE60005E6801F03FFCDFE7019B5E604560204685
:10EE700001F038FC01A801F035FC05B0F0BD00BF81
:10EE800010D8012037B50546F0B101F01DFC0F4B3D
:10EE900000901C68AC4204D142681A6011E001F095
:10EEA00021FC74B1204601F00FFC034602A85C6807
:10EEB00040F8043DAC42F2D1009A52685A6001F029
:10EEC00011FC684601F00EFC03B030BD10D80120E3
:10EED000002337B50360094B1C68054654B1204632
:10EEE00001F0F2FB02AB026943F8040D2A601846F8
:10EEF00001F0F8FB204603B030BD00BF0CD8012064
:10EF0000002373B50B600E46044690B101F0DCFBA4
:10EF100002AD846845F8040D44B1284601F0E2FBD7
:10EF2000204601F0D1FB036901903360284601F0CF
:10EF3000D9FB204602B070BD2DE9F74381461C2065
:10EF40000E4690461F4601F091FE0446002831D03F
:10EF50001A4B1B4A1A6001F0B7FB009016B900F07B
:10EF6000A9F8064602A850F8085D68466E61C5F823
:10EF70000090C5F81080AF8101F0B4FB2046FFF788
:10EF800033FF104B1A6832B901220F481A600F4B39
:10EF9000036000F079FF204601F096FB0C4A0190D7
:10EFA000136813B91460836001E08360146001A8E2
:10EFB00001F098FB204603B0BDE8F083581702200B
:10EFC00079ED00081CD8012014D801205DED00085F
:10EFD0000CD8012073B5044658B3174D2E688642ED
:10EFE0000BD101F071FB02AB826843F8040D2A607B
:10EFF000184616E0684601F075FB304601F064FBE8
:10F00000866802ADA64245F8080DF3D1204601F00E
:10F010005BFB009B826801909A6001A801F062FB93
:10F02000684601F05FFB2046FFF72CFF204601F009
:10F0300085FB02B070BD00BF0CD8012013B50C4693
:10F0400040B101F041FB02AB846143F8040D184666
:10F0500001F048FB02B010BD13B5044698B101F0B1
:10F0600033FB019000F026F802AB53F8042D9169B0
:10F0700008445061184601F035FB2046FFF702FFB7
:10F080002046FFF7B1FE02B010BD13B50C4668B1C3
:10F0900001F01AFB02AB828943F8040D14421846B2
:10F0A0000CBF0024012401F01DFB00E001242046D8
:10F0B00002B010BD05F016BB034B1B68B3F92A2044
:10F0C00058851046704700BF1C010020034B1B6889
:10F0D000B3F92C2098851046704700BF1C01002012
:10F0E000024B1B689A7E9876104670471C010020E0
:10F0F000034B1B68D96900B1D8610846704700BF4F
:10F100001C010020FEF7C8BE08B5002000F01CF866
:10F110006FF07F4000F01AF8012000F07DF8002029
:10F12000FFF7D4FF0020FFF7C7FF0020FFF7EAFF3B
:10F13000044B1868FFF7DCFF0020BDE80840FFF72C
:10F14000CFBF00BF20010020FFF7EEB9FFF7F4B9F1
:10F1500010B5074B1C7820B101221A704FF0FF3018
:10F1600002E018706FF07F4004F0C8F8204610BD30
:10F170006517022070B5084D2B68012804465E7C97
:10F1800008D800F04DFD28B12B685C7400F008F839
:10F19000024B1C60304670BD1C0100201817022075
:10F1A00008B503F003FFFEF7F7FCBDE80840FCF7E5
:10F1B00099BB000008B5034B7022196809F040FDA7
:10F1C00008BD00BF1C01002008B5034B014670229A
:10F1D000186809F035FD08BD1C010020B0F90220B7
:10F1E000B1F906309A4214DCB1F90220B0F90630C8
:10F1F0009A420EDCB0F90020B1F904309A4208DCE2
:10F20000B0F90430B1F900209A42CCBF00200120AF
:10F210007047002070470000024B1B681A7E18766A
:10F22000104670471C010020024B1A6802B9186092
:10F23000FFF764BC20D801200A4A0B49136809680B
:10F240008B4210B50BD0094CA34293E8030014BFC6
:10F250000833503B136002F02FFB012010BD00204B
:10F2600010BD00BF180100201401002074D8012037
:10F2700068B1038889B20B440380838819444388AA
:10F28000818092B213444380C3881A44C28070477D
:10F2900010B538B309B30AB3B1F90040B2F9003080
:10F2A0009C42B8BF23460380B1F90240B2F9023054
:10F2B0009C42B8BF23464380B1F90440B2F9043000
:10F2C000B1F906109C42A8BF23468380B2F90630EC
:10F2D0009942A8BF0B46C38010BD11460B6803605E
:10F2E0004B68436010BD0000054B1B68002B18BF26
:10F2F0000020044B0129B8BF01211954704700BFF9
:10F300007CD8012044170220024B1B685884998442
:10F31000002070471C010020044BB3F9003003604B
:10F32000034BB3F900300B60704700BF5C1702203D
:10F3300050170220014B1B68987E70471C0100206B
:10F3400003F0E4BF0A4B10B51C681CB1A047041CB5
:10F3500018BF0124FCF718FA064B1B68002818BFD9
:10F3600001241BB19847002818BF0124204610BD76
:10F37000581702207017022010B50024FFF7E2FF93
:10F3800008B10124FAE7204610BD00000F4B73B509
:10F390001B68DE6C1C6D06440D19B3B2144468463C
:10F3A000ADF80030ADF80430ADF80250ADF80640CD
:10F3B000FCF7B6F838B1304629462246FEF7C8FDBC
:10F3C000FBF7ECFFF6E702B070BD00BF1C010020A8
:10F3D0001E4B1B689B7E013B032B32D8DFE803F0FA
:10F3E000020D1A221A4B06300340002B03DA013BB0
:10F3F00063F00F0301330B2B08E0164B0340002B87
:10F4000003DA013B63F003030133012BCCBF00207F
:10F4100001207047142390FBF3F203FB12000B282A
:10F4200009DC10E0182390FBF3F203FB12000B2819
:10F4300009DD20F00400103801288CBF00200120D5
:10F440007047002070470120704700BF1C0100205A
:10F450000F00008003000080C0F30B00B0F5006FC8
:10F46000C6BFA0F5006001210021B0F5806FC8BFC4
:10F47000C0F5006000F03F0310B582110B4CC3F1E2
:10F4800040039BB234F81200402B00FB03F008D07D
:10F49000102A06D00132C3F1400334F8122003FBD6
:10F4A00002002030800901B1404210BD6CF7010814
:10F4B00000F58060FFF7D0BF2DE9F74FDDF8308011
:10F4C000171A5C1A54EA070C05460E46D8F800B025
:10F4D00004D103B0BDE8F04F04F000BB87EAE77049
:10F4E000A0EBE77084EAE471A1EBE471884204DBED
:10F4F00021463C460F46002106E011461A460B46BF
:10F50000294635460E460121009184EAE471A1EBBB
:10F51000E4718C4208D01E462B46644215467F4259
:10F520001A464FF0FF3A01E04FF0010A002FDFF8D2
:10F5300048913ED1009BD3B1D9F800309B7E8BB966
:10F540003046294603B0BDE8F04FFEF701BDFFF796
:10F550003FFF30B9D9F800305B6E30465B687919EF
:10F5600098470137A74207EB0B00F0DD1DE0D9F803
:10F570000030997E11B1DDF800A012E05B6E2846E4
:10F580001B683146984774E0FFF722FF38B9D9F875
:10F5900000305B6E0AEB05005B68314698470AF164
:10F5A000010AA2450AEB0B00EEDD0138C8F80000A5
:10F5B0005FE0D9F800104FF00202897E94FBF2F26E
:10F5C000B8BF5242D9B99346A846C5EB0803A34237
:10F5D0004FDC009B9BFBF4F131442BB9D9F8003090
:10F5E0005B6E40465B6805E0D9F800305B6E5B6897
:10F5F00008464146984708F10108BB44E5E7BAF1DF
:10F60000FF3F04BF04EB0B01C8F800100192AB46AA
:10F61000C5EB0B01A142D8F800001EDC5044C8F82D
:10F620000000FFF7D5FE80B9DDF804C0D9F800006E
:10F63000009B406E9CFBF4F1314413B9436858467B
:10F6400002E04368084659469847DDF804C0BC44C8
:10F650000BF1010BCDF804C0DAE7BAF1FF3F04BFAC
:10F660002418C8F80040D8F80020CAEB0203C8F8F4
:10F67000003003B0BDE8F08F1C0100202DE9F04FF1
:10F68000674D2C6894F818B0BBF1010F87B0814624
:10F69000884617461E46AA4604D1109C0094FFF7E0
:10F6A0000BFFBAE0841ACD1A54EA050300F0B580C6
:10F6B000002CBABF644201230023002DBCBF6D4261
:10F6C00043F00203A5420BF1FF3B04DD224643F069
:10F6D00004032C461546022294FBF2F202EB852528
:10F6E00095FBF4F4A1114F4AC4F38304C4F110054F
:10F6F00032F91100102D05FB00F004D0013132F970
:10F70000112004FB02001022083090FBF2F0590790
:10F7100048BFC0F58060DA0748BFC0F500609B07AE
:10F7200048BFC0F5805000F580652846FFF7C0FE51
:10F7300000FB0BF42846FFF78FFE002C00FB0BF0BC
:10F7400004DAC4F500739B125B4202E004F5007317
:10F750009B12002806DAC0F5007B4FEAAB2BCBF1F9
:10F76000000B03E000F5007B4FEAAB2B002B03DD21
:10F77000581C40105B1005E0022293FBF2F0013BA5
:10F7800093FBF2F3BBF1000F05DD0BF10102521008
:10F790004FEA6B0B06E002219BFBF1F20BF1FF3B02
:10F7A0009BFBF1FB80B21FFA89F4011992B2ADF80C
:10F7B00008101FFA8BFB1FFA88F15518CBEB0101DB
:10F7C0009BB2ADF80E10B9B2E41ACB1AADF81030F6
:10F7D000B3B20144CBEB030B13440022ADF8141079
:10F7E000ADF8163002A813460421ADF80A50ADF862
:10F7F0000C40ADF812B004F08FF8DAF800305B7E00
:10F800001BB94846414604F069F9DAF800305B7EDE
:10F810001BB93846314604F061F907B0BDE8F08FF6
:10F820001C0100208EF7010830B585B004AC00251E
:10F8300044F8045D0094FFF721FF05B030BD0000DF
:10F840002DE9F8431E460C4B1C6881460020E56CF0
:10F85000246D88461746FBF763FE50B109EB05009F
:10F8600008EB04017A193319FFF7DEFFFBF796FD69
:10F87000F3E7BDE8F88300BF1C010020F7B5104F87
:10F880003B681D6DDC6C05440E19ABB21444684630
:10F89000ADF80060ADF80440ADF80230ADF80630C8
:10F8A000FBF73EFE48B13B685B6E30461B6829465D
:10F8B00022469847FBF772FDF4E703B0F0BD00BFA6
:10F8C0001C0100202DE9F04F9846814B8BB08A46F1
:10F8D0001968069000209146149F159ECD6C0C6D02
:10F8E000FBF71EFE002800F0EF800AF100430698A7
:10F8F000013B00EB43030793169B002B14BF6FF0F3
:10F9000001030223A9444444099327B9FBF746FDA8
:10F910000028FAD1D8E0002EF8D0BAF1000FF5DDBA
:10F920007B1C04D1012E14BF022301230AE0012F06
:10F9300004D1012E14BF0323002303E0012E14BFC2
:10F94000052304230593624B1B685B69EBB1B3F994
:10F950000080B3F90200B3F90420B3F906B00490B3
:10F9600008F1FF38C14509EB0A03B8BFC9EB080825
:10F9700003F1FF33B4BF28EAE8784FF00008934260
:10F980000ADDC9EB0202013207E04FF0FF3B5246AD
:10F99000CDF810B0984600E05246169B1BB9069B66
:10F9A00003EB480300E0079B90450393AEDA4A441B
:10F9B00008920022C84401230292039809990588FD
:10F9C00008442DB247F6FF718D4203900DD1029885
:10F9D00000286FD1002B6FD1114608F1FF30019242
:10F9E000FEF762FA0123019A67E00598411EDBB138
:10F9F000042917D8DFE801F00305070B0F00621B8D
:10FA00000EE0651B00E02544B5FBF6F208E0254456
:10FA100007FB05F204E0254407FB05F2B2FBF6F212
:10FA200000234AE02A19FBE7042912D8DFE801F095
:10FA30000305070B0E00651B0CE0651B00E0254469
:10FA4000B5FBF6F506E025447D4303E025447D4300
:10FA5000F6E7254404998A4201DA8D4225DB5A45AE
:10FA600001DD5D4521DC05EB020C0221AA429CFB75
:10FA7000F1FC08F1FF300BDC114662468DE80810FE
:10FA8000FEF766FADDF804C0404661462A4609E002
:10FA900061468DE80810FEF75BFADDF804C04046C9
:10FAA00029466246FEF754FA009B029A01320292FE
:10FAB0002A4602E0002302930123089808F1010876
:10FAC00080457FF47AAF21E70BB0BDE8F08F00BF2F
:10FAD0001C010020F8B50B4B1B680546B3F92C0040
:10FAE00040F002000F461646FFF7F0FA394604468A
:10FAF0003246284600F008F82046BDE8F840FFF7F7
:10FB0000E5BA00BF1C010020024B1B6859849A848F
:10FB100000F002B81C0100202DE9F74F0446002830
:10FB200079D03E4D00F0B4FC2B688046B3F82290AB
:10FB300000F096FC2B689A8C87B2D21B9A842378AB
:10FB4000002B5DD047F6FF71204600F0D7FB06463C
:10FB50003146204600F000FC2B689A8D02F003022B
:10FB6000012A05D0022A14BF002290FBF2F200E025
:10FB70000246598C8A1A92B291B259841FFA80FABD
:10FB80009B8CADF800100AF1FF310A44ADF8023049
:10FB90001FFA88FB013B5B44ADF804202046314648
:10FBA0006A46ADF8063000F007FC2B68BDF802206D
:10FBB0009A842046314603F029FE235C0A2B04EB8D
:10FBC000000201D00D2B12D12B68998D01F0030199
:10FBD000013901298ABF198CA3F822905984117820
:10FBE0000A290BD1998C8B44A3F824B006E00B4B67
:10FBF000BDF800001B688244A3F822A0137843B923
:10FC00002B689A8C17449A8D9F8422F003029A8560
:10FC100001E0541C93E703B0BDE8F08F1C01002005
:10FC2000012809DC054B53F8200020B1C3681B688C
:10FC30001BB10068F9E77047002070477417022075
:10FC400000F02EBD012BF8B506460D4617461C46A2
:10FC500001DD0020F8BD1C2000F08EFE0028F8D049
:10FC60000DB1056109E0094B53F8241029B10B6867
:10FC70000BB11946FBE70B690361002383608461C4
:10FC80008782C66003604360F8BD00BF741702201E
:10FC9000094B826953F82210814204BF016843F87E
:10FCA000221043680BB102681A60026802B1536007
:10FCB00000230360436070477417022070B538B3A7
:10FCC0008269012A24DC194951F822300D4613B902
:10FCD00041F822001AE0596809B10B46FBE7C168F8
:10FCE0000E68D9680C68B44203DD1B68002BF8D19C
:10FCF0000EE002D1818A012911D0596899B10860BA
:10FD000041605860984208BF00230360002070BD26
:10FD1000012070BDCB681B68A3420B46EDDB196860
:10FD20000029F7D1E9E745F82200EAE77417022035
:10FD300038B51D46FFF786FF044648B1FFF7BEFF02
:10FD4000E3681B6823B9034B16351B6843F825404D
:10FD5000204638BD1C01002010B5074B0748002481
:10FD6000214670221C60FEF71DFC21460448082233
:10FD7000BDE81040FEF716BCFCD8012084D8012055
:10FD80007417022038B5194D2B681A1DDA6303F178
:10FD900008029B631B6442615A7C154B044653F86E
:10FDA0002200C36804F108011B6B9847114B63667E
:10FDB000114B1B68E3612B680833636101232376D1
:10FDC000FAF762FC032384F868306FF07043236312
:10FDD0006363A0640020FEF7A7FB6FF07F40FEF78F
:10FDE000ABFB064B064A1A6038BD00BF1C01002061
:10FDF00074170220B0F70108200100206C170220C0
:10FE00009C1802082DE9F347074604209A460E463F
:10FE10009146FEF741F8134B1C68E56C246D2F44A6
:10FE2000264480464D4454446846ADF80070ADF811
:10FE30000450ADF80260ADF80640FBF771FB28B93D
:10FE40004046FEF729F802B0BDE8F0873846314653
:10FE50002A462346FEF7A2F8FBF7A0FA0028F5D1C0
:10FE6000EEE700BF1C01002010B500200146FFF79F
:10FE70004BFA044843F6FF7201461346BDE81040B2
:10FE8000FFF7C0BF01C0FFFF80B483B000AF786050
:10FE9000054B1A687B685A60034B7A681A600C3706
:10FEA000BD465DF8047B704780D8012008B5084B3B
:10FEB0001A6862B901221A60F0F7F6FBF0F71EFC2F
:10FEC0000448054B0360BDE80840FFF7DDBF08BDEF
:10FED000FCD80120F4D8012059FD000890B583B06A
:10FEE00000AF204B1F4A126822F001021A601E4B1D
:10FEF00001221A601D4B1E4A1A601C4B1A681D4BCA
:10FF00009A4200D0FEE7FFF7D1FF1B4B2E221A705A
:10FF100004F0EAFB1948FFF735FFFEF763FA786053
:10FF2000FDF744FF0346002B04D0FDF745FF0346D1
:10FF3000002B09D1FDF726FF0446FDF726FF0346F7
:10FF400020461946FDF728FF0020002103F070FC31
:10FF5000FBF732FD0A4B01221A707B6818460C37FA
:10FF6000BD4690BD002000E0083002400030024055
:10FF7000C2A507F4CDB5E8B54617022084D8012004
:10FF80006417022038B103888B4202D843888B4221
:10FF900001D28068F6E770472DE9F04F384C2368AE
:10FFA000B3F92A90DB69054689B0D8692946FFF77D
:10FFB000E9FF002861D0B0F800804768C8EB050869
:10FFC00007EBC806484696F802B0FDF765FF2568BE
:10FFD00017F83820D5F81CE0B5F924109EF81AC09F
:10FFE0009EF8183006938246B5F92200CDF800C07D
:10FFF0009EF81BE0CDF804E04FF0010ECDF80CB0F8
:020000040801F1
:10000000CDF808E073680493AD6B069B0595FEF789
:10001000CDF82368DA6992F819B0117E8B4520D9A2
:10002000B9F1020FD57E1CD0079103F04DFC81463B
:1000300003F043FCFFF78AF8246817F83870E26988
:10004000B4F92430B4F92200D27E079907FB0202EA
:1000500001FB05310BFB0533FDF7A0FF4846FFF719
:1000600075F85046FDF718FF054B1B68DA69598C87
:10007000907E727800FB02125A8409B0BDE8F08FBE
:100080001C0100200D4B70B51B68DD6906460C464F
:10009000E8693146FFF776FF70B103884268F61AC7
:1000A00002EBC6035878AB7E10FB03F024B112F8C4
:1000B000362012FB03F3236070BD00BF1C0100203B
:1000C00001230B80704708B5C069FFF75BFF003064
:1000D00018BF012008BD0000524B2DE9F04F1B68EE
:1000E000D9695F8CCC699D8CA28990428BB008D372
:1000F000E689864205D3D4F80090821A4FF0FF3B80
:1001000015E0A268D4F80490002A00F081801688D7
:10011000B0427DD3B2F802C0844579D35268801BC7
:1001200080B202EB800632F92020B6F902B0501CF2
:100130006ED091F81880A17CB3F82AA0267C069294
:1001400018FB01F107910FFA8AF108460891FDF7B3
:10015000A3FE344909900B68069AD969887E0090FD
:10016000C97E019101210291A17C0391079901FBB4
:10017000029204929B6B05933FB22DB238462946FA
:1001800032464346FEF712F8BBF1FF3F1BD04AF060
:10019000020000B2FDF780FE224A1368DA69917E00
:1001A0000091D27E0192012102910799A27C0392D3
:1001B00001FB0B9204929B6B05933846294632460D
:1001C0004346FDF7F3FFDFF85C80D8F80030DB69C9
:1001D0005A7E1B7E9A4217D9089A022A14D08AF0B6
:1001E000040000B2FDF758FED8F80030DB6993F840
:1001F00018E0D97E9A7E5B7E38460EFB015106FBE5
:1002000002722B44FDF7CAFE099BD8B2FDF744FEEB
:10021000044B617C1B685A8C0A445A840BB0BDE8BD
:10022000F08F00BF1C010020044B1B68DB69DB69F9
:1002300009B11A7C0A60587C704700BF1C0100207D
:1002400002230B807047C3699A898A4202D8DA89EF
:100250008A420FD2986880B1038899420CD34288B1
:100260008A4209D3C91A426832F82100C043C0F358
:10027000C030704701207047002070477047000071
:1002800037B5154602AB1A4A43F8081D01901268AB
:10029000184C6946904723680190586958B9012065
:1002A000FEF72CFA2368DB695B69BBB19B68019898
:1002B0000099984717E02946FEF790FF0028EED1F5
:1002C00014E001A803F08EFA2368DB691B68054679
:1002D0009847094B1B680BB128469847009B013B88
:1002E000002B0093EDDA0020FEF708FA03B030BDD2
:1002F000240100201C0100206017022037B50D46A4
:100300000190044698B10B4B1B68DB695B690BB12C
:100310005B680BB9002408E0984709E001A803F0E6
:1003200061FA20B10A2802D00134AC42F6DB204643
:1003300003B030BD1C01002013B502A9002441F810
:10034000044D00F0B7F8019B8342CCBFC0EB030023
:10035000204602B010BD000037B5154A019002AB2F
:10036000126843F8081D694690470190F0B1114B9F
:100370001B68DB695B690BB11B6813B900252C4650
:1003800002E00099984711E0009B013B002B00938D
:1003900007DB01A803F026FA054600F081F80444C3
:1003A000F2E72846FFF7C8FF2044FFE703B030BD5F
:1003B000240100201C010020274B1B6873B5054653
:1003C0000C4663B10020FBF7ABF8002841D028466B
:1003D00021466A46FFF754FFFAF7E0FFF5E7106899
:1003E00051681E4E6B4603C33368BDF80010B3F866
:1003F0004C20B3F850301144ADF80010BDF8021095
:100400001944ADF80210BDF804100A44ADF80420F8
:10041000BDF8062068461344ADF80630FBF780F8B7
:10042000336840B9598CDA6C8A1A5A84998C1A6DDF
:100430008A1A9A840DE0BDF800205A84BDF8022083
:100440009A84284621466A46FFF71AFFFAF7A6FF64
:10045000E6E702B070BD00BF481702201C01002073
:100460000A4B1B689A8D02F00C02082A07D00C2A4E
:1004700005D0042A07D1DB69187E01387047DB6993
:10048000187E400870470020704700BF1C01002004
:10049000024B1B68DB69587E704700BF1C010020BF
:1004A00008B5034B1B68DB6900215B68984708BDF2
:1004B0001C01002008B5034B1B68DB695B6898478B
:1004C00008BD00BF1C010020074B5A68596A013261
:1004D00010B55A605A6B02EBC0046160002102F84B
:1004E0003010586210BD00BF8417022038B50B4D84
:1004F000002405F140002146802285F82840FEF7BF
:1005000051F828462146C022FEF74CF821460448FF
:100510000C22BDE83840FEF745B800BF8417022022
:1005200000D9012010B542680F230D4901EBC30427
:10053000246CA24203D213F1FF33F6D210BD0F2B6D
:100540000CD80C68A21A0A608268C06802B15060B8
:1005500008B1026010BD01EBC3035A6410BD00BFB7
:1005600084170220F8B5264EF3685A1EB36B054671
:100570001344081898420C4605D84B591BB94368D8
:100580001D44FFF7CFFFB36B9C420AD954F8047C9B
:10059000E71B3B682BB97B6838461D44FFF7C2FF59
:1005A0003C460F2306EBC302126C954203D213F1B3
:1005B000FF33F7D222E00F2B20D8083306EBC3021B
:1005C00061195268A260002084E82100246141F88A
:1005D000045C04F1080102B1516006EBC303E06062
:1005E0005960336896F82910054A2B44336029B9BD
:1005F000D168CB1A9168994238BF93602846F8BDFC
:1006000084170220254B2DE9F74FDA689C6B013ADD
:10061000824602EB04099B4694E82800002B33D164
:1006200004EB0508C8452FD254F805C0D8F804607B
:10063000BCF1000F28D0DBF83430184F13F83C30F1
:10064000012B21D1FB6A20468DE80810FFF76AFFD5
:10065000D8F800107A6B02EBC10220465460414684
:10066000324608F041FA9DE808109C4502D17B6BA8
:100670005B1B7B632846A119FFF774FFBAF1000FDB
:1006800001D0824505D935462C444C45C4D30120C0
:1006900000E0002003B0BDE8F08F00BF8417022007
:1006A00028B1034AD36B036003B15860D06370472D
:1006B0008417022028B1034B5B6B03EBC00040683A
:1006C0000830704784170220054BD9690131D96180
:1006D0005B6B13F83010013103F83010FFF7EABFFD
:1006E0008417022030B50268094B52F8081C5A6B77
:1006F00012F83140012C03D9DD690DB1013DDD61F6
:10070000013C02F8314000230360184630BD00BFB1
:1007100084170220024B21F00301186059607047D2
:1007200000D9012030B1044B5B6B03EBC000436880
:1007300058680C38704700BF8417022010B5044673
:1007400080B1094B5B6B03EBC00213F83030012B17
:1007500008D151684868FFF705FF2046BDE8104002
:10076000FFF7B2BE10BD00BF841702202DE9F04193
:10077000224CE36A3BB9224B9D685B680835B3FBAA
:10078000F5F5023503E023691D1D05EBD305E800EF
:1007900000F078F9804660B3616B2269E76A01EB8B
:1007A000C003D2005E680836304608F049FA226974
:1007B000666306EBC201C4F82C8004311346681E40
:1007C000834201F1080103D2013341F8083CF6E706
:1007D00006EBC30300265E60636862629B1A2B44CB
:1007E0006360256138463FB1FFF7A8FF3046BDE89A
:1007F000F0810120BDE8F081BDE8F081841702207E
:1008000000D90120F8B5584E96F82810002940F07C
:10081000AA80564D6A68012386F82830B2F5205F19
:1008200028BF4FF420522B6894080020A0420CD01F
:1008300047184FF0FF0EB7FBFEFECEEB0E2ECEEBB1
:10084000070743F820700130F0E70020A04216D0DF
:1008500047184FF0FF0EB7FBFEFECEEB0E2ECEEB91
:10086000070E53F82070774507D0AA683F4B002A3F
:1008700055D15A6892089A6051E00130E6E701319B
:100880000229D2D1540800210020A0420CD04718E0
:100890004FF0FF0EB7FBFEFECEEB0E2ECEEB0707A2
:1008A00023F810700130F0E70020A0420FD0471865
:1008B0004FF0FF0EB7FBFEFECEEB0E2ECEEB070782
:1008C00033F810C0BFB2BC45CFD10130EDE70131E4
:1008D0000229D9D100210020904207D04418FF27D7
:1008E000B4FBF7F73C441C540130F5E7002090427C
:1008F0000BD04418FF27B4FBF7F73C441F5C04F00F
:10090000FF04A742B1D10130F1E701310229E2D160
:1009100000219142A9D0002058540131F9E7144830
:10092000144B0360FFF7B0FA5A23336200231021FF
:1009300006EBC30299400133102B0B4C1164F6D126
:1009400068682968A16302232361A0F114030B44A2
:1009500001256363E0605D6065626560FFF702FE2C
:10096000FFF704FF2563F8BD8417022000D901209A
:100970000CD90120ED0401082DE9F0410546264E71
:100980000335FFF73FFF25F00305336CF26B0435A9
:100990009D4238BF1D4614462CB154F8043CAB426E
:1009A0002CD02468F8E7F368B26B02EB030858F820
:1009B000047CC7EB08073B6833B12046FFF722FEF3
:1009C00058F8047CC7EB08073B6813BB7B68AB4255
:1009D0001FDB38461C1DFFF7A5FDF36878685B1B1D
:1009E000F3607369641B2B44401B3C44736102D069
:1009F0003946FFF7B7FD44F8045C0AE023680BB101
:100A000061685960616801B10B60A24201D123683D
:100A1000F3632046BDE8F0818417022008B5FFF794
:100A2000F1FE00220B4B1344D3F8BC3013B19B688A
:100A300000200BE0083A12F1800FF3D1F8E75A6872
:100A40009B68904238BF104613B19B68002BF6D1CB
:100A50000C3808BD8417022008B5FFF7DFFFB0F59A
:100A6000800F4FF06403064A04D990FBF3F0136A39
:100A7000584308BD126A5043B0FBF3F008BD00BFF5
:100A8000841702202DE9F843384D0446FFF7BAFEDB
:100A90002F6C2B68BC4224BFE71C27F003070C37E0
:100AA0009F42324C3ED8236B62689A420FD96B68E2
:100AB0006E6A013B6B606B6B4FEAC60903EB090280
:100AC00052686A62012203F8362056B92AE0013BD7
:100AD0002363FFF74BFE236B013323630028E6D02B
:100AE00020E00F2305EBC302126C97420CD213F1E6
:100AF000FF33F7D208E094682CB16268974214D9AA
:100B0000A268002AF7D101330F2B03D805EBC302EB
:100B1000526CF6E73846FFF775FD0028E1D0304605
:100B2000FFF7D2FC0020BDE8F883D4F804802B6CDA
:100B3000C7EB08020C3320469A4238BF4746FFF7FE
:100B4000F1FC6B6B4B44E1195C60B8454FF000035E
:100B500084E8C000A360246141F8047C03DDC7EB96
:100B60000800FFF7FFFC3046BDE8F8838417022039
:100B700008B1FFF787BF704710B504460068FFF75C
:100B8000DDFD0023236010BD10B580EAE071A1EB0C
:100B9000E0710022531C0A2B06D0064C54F8234067
:100BA000A14201D31A46F5E70028B8BF931C1846A6
:100BB00010BD00BFB8F70108002807DD0B685A1CFC
:100BC0000A602B221A700B6800221A70704700000E
:100BD000B0F1004FF0B51C6809D1601C18600139F4
:100BE0002D202070C9B26FF0004001260CE00028D3
:100BF00006DA651C1D602D2525704042012400E0A9
:100C00000024091BC9B200260AB30139C9B21EE08B
:100C10004D1E9142EDB205D11C68671C1F60114F3B
:100C20003F782770104C54F8257090FBF7F4E4B22D
:100C30000A2C0ED807FB14007DB10A2C18BF2946D8
:100C40001D6808BF01246F1C30341F602C70002900
:100C5000DED11B6800221A70F0BD002EEDD00134E9
:100C6000E4B2EAE746170220B8F7010873B5054673
:100C7000FFF77EFF064658B1FFF726FD02AC0021C4
:100C800044F8040D2A46FDF78DFC2046FFF72AFDA7
:100C9000304602B070BD00002DE9F7431E4CD4F879
:100CA00000E0DEF84C40DEF85060051914449EF870
:100CB0001820013A92B28F191E44AB1AADF80030D9
:100CC0001319ADF804306846BB1A3244ADF802304F
:100CD000ADF80620FAF724FCD0B128463946224662
:100CE000FDF710F907F1010928463146224606F1C1
:100CF000FF38FDF707F9284649464246FDF728F92F
:100D0000204649464246FDF723F9FAF747FBE3E759
:100D100003B0BDE8F08300BF1C010020C0F3C42174
:100D2000064B00F01F02C0F345109A5C5B5C03EBBE
:100D30000243034A105C03EB002070477C16020854
:100D40003C160208C0F30741064BC2B2C0F30720AD
:100D50009A5C5B5C03EBC223034A105C03EB40101C
:100D6000704700BF9C1702089C1602084FF6FF70E0
:100D700070470000F8B50F4F3F6806460D46144611
:100D80009C460FB1B847F8BD56F8042B0A49D3B2B8
:100D9000013CC85CC2F30743C2F30722CB5C07499E
:100DA0008A5C03EBC02303EB42132B806544EBD139
:100DB000F8BD00BF18D901209C1702089C16020834
:100DC000F8B5134E3668844614461D460EB1B0473A
:100DD000F8BD501E02F18042013A03FB00C001EB56
:100DE000820102880B4B02F01F06D70A9E5DDB5D75
:100DF000C2F3451203EB0643074EB25C013C03EB22
:100E0000022341F80439C5EB0000EAD1F8BD00BF68
:100E100014D901207C1602083C160208704770475E
:100E200070474FF0FF30704710B550F8044B0C601E
:100E3000013A1944F9D110BD10B5046841F8044BCA
:100E4000013A1844F9D110BD10B59CB0044668466B
:100E5000FEF7B0F9094B1868FDF76EFBB4F9000016
:100E6000B4F90210B4F90420B4F90630FFF714FF06
:100E70006846FEF7A9F91CB010BD00BF1CD90120BF
:100E800010B59CB004466846FEF794F9094B186803
:100E9000FDF752FBB4F90000B4F90210B4F90420D4
:100EA000B4F90630FFF7F8FE6846FEF78DF91CB07E
:100EB00010BD00BF1CD9012007B56846F9F702FC38
:100EC0006846FFF7C1FF03B05DF804FB07B568464D
:100ED000F9F7F8FB6846FFF7D3FF03B05DF804FBB2
:100EE00013B5044640B1FFF7EFFB02AB046D43F8C6
:100EF000040D1846FFF7F6FB204602B010BD1FB5E3
:100F000001F00803002B40F28A3440F28A5208BFF5
:100F100022460CBFFF23FE238DE80500002002912E
:100F2000039302460346014600F0AEF8062104464C
:100F3000F9F707FA204604B010BD07B5FFF7C4FB68
:100F40000190406E00F0D4FB02A8002250F8043D4E
:100F50005A66DA65FFF7C6FB03B05DF804FB438E03
:100F60001B0710B512D5B0F90420B0F9003008887D
:100F70004C880C80D31A8A88CC888C8001339BB231
:100F8000C043D24318441344C8804B8010BD10B5F1
:100F9000044600F0B6FCFAF78CF82046F9F7ABFAF5
:100FA0002521BDE81040F9F74FB90000F0B589B030
:100FB0000E9E109C119DFAB9F3B9304606A9F9F7B7
:100FC00017FB14F0080F2C4BBDF91C70BDF91EE087
:100FD00009D0BDF91A10B3F90020781CC1EB0E033B
:100FE000801A013308E0BDF91800B3F900300EF1A2
:100FF00001013A1AC91A013200960F9E01961F4E3E
:101000000296129E3C360396FAF794F8064600289C
:101010002FD0FFF759FB04F00802E30648BF42F067
:101020001002A5F1FE0348BF92B2012B88BF42F027
:10103000100229460590F8F741F8114B08AF0FCB85
:1010400057F80C4D04F1340585E80F006423E36480
:101050000C4D0A236365002323652B6863643846BF
:10106000FFF740FB2B6830465B6898473046FFF738
:101070008EFF304609B0F0BD3C0100202B11010865
:10108000280100203801002010B586B0089C00948B
:10109000099C01940A9C02940B9C039400240494E0
:1010A000FFF784FF06B010BD37B50C46054600B308
:1010B000FFF70AFB002C0190C16C426D05DB8A1A18
:1010C00022EAE272944202DC00E000242246016D32
:1010D00091420BD002652846F9F7EBFF01A8FFF714
:1010E00001FB28460521F9F72CF902E001A8FFF7DA
:1010F000F9FA03B030BD73B50D46064660B1FFF78F
:10110000E3FA024602A8146D40F8042DFFF7EAFA4C
:1011100030466119FFF7C8FF02B070BD4FF0FF31D4
:10112000FFF7E9BF0121FFF7E6BF2DE9F04F446863
:1011300080468FB020464146F7F7C8FF002800F0F0
:10114000C081D8F80030232B00F082810BDC0E2BFD
:1011500000F02A810F2B12D00B2B40F0AF812046DC
:10116000FFF715FFAAE140F21312934200F07F81CE
:10117000B3F5107F12D0242B40F0A08143E120462C
:10118000FFF7A2FA0590002800F09B81436C05A8A8
:101190001D68FFF7A7FA2046A84792E1D8F80C701F
:1011A000002F00F08B813B7A2046002B00F0D68088
:1011B000FFF78AFA05A9836C0390066D20469847CD
:1011C000039BB3F832A05D6DDA6C1AF0080FC5EB23
:1011D000020903D097E806003A6079609A6D3F688B
:1011E000032A14D12046FFF7A8FE0D9B0C9902207C
:1011F00093FBF0F3FF1A069BFB1A581E00FB09F045
:1012000002F049F9039B0646186603A87EE006989B
:1012100087420BDC022A39D05B6E13B12046FFF700
:101220008CFE039B0222013E9A652FE007998F42B4
:1012300002DA761B6D422FE008998F4212DC0C997E
:1012400000290BDD0D9B022293FBF2F3FF1A3F1ADC
:10125000013F07FB09F002F01EF90646039B03223B
:101260009A6516E009998F4201DA2E4414E00A9932
:101270008F420EDC012A0ED05B6E13B12046FFF7C1
:101280005CFE039B012501369D6505E04FF0FF35AF
:1012900002E0002500E01546DDF80CB00C99DBF803
:1012A0005C30DDF834E0069A71B102209EFBF0F06C
:1012B000381A801A013800FB09F0019302F0EBF8AC
:1012C000019BCBF8600009E0DBF85820012A04BF3D
:1012D000DBF84C1001F1FF31CBF8601003A801934B
:1012E000FFF700FA019BA5B1BBB94FF4C87240F2F9
:1012F000D241204600F034FA07462046FFF7E4F9D1
:1013000002460EA840F8282D5766D565FFF7EAF982
:1013100003E013B12046FFF710FE2046012100F044
:10132000A3FA20463146FFF7BFFE1AF4807F40F053
:10133000C5802046FFF7C8F90EAB856A43F8280D33
:101340001846FFF7CFF94FF480712046F7F78AFE71
:10135000A90740F1B3802046012174E0FFF7B4F9FA
:10136000458E039003A8FFF7BDF9EA0540F1A6807A
:1013700020464FF48071F7F78BFE2046FFF7A4F963
:10138000C36D059013B12046FFF7D7FD0EA80022CC
:1013900050F8243D9D6A9A65FFF7A4F9AB0740F128
:1013A0008D80204602214EE02046FFF78DF90EABDE
:1013B000456D43F8240D1846FFF794F9D8F80C2032
:1013C00013685268002A79DD103B122B76D8DFE8CB
:1013D00003F0161612127575757575757575757538
:1013E0007575750A0D002046294601E020466942C0
:1013F000FFF781FE62E02046FFF794FE5EE02046A4
:10140000FFF78CFE5AE02046D8F80C60FFF75CF935
:101410000EAD034645F8240DDA6C3068B168904291
:10142000726805D15E6D8E4202D11E6D96420DD05E
:10143000D86459651A652046F9F73BFE2846FFF740
:1014400051F920460521F8F77CFF37E0284633E0C4
:101450002046FFF739F9059000282FD0D8F80C3036
:10146000C26C1A60426D9A60026D5A6023E0204699
:10147000FFF72AF9C16D059011B12046FFF73BFE39
:10148000059BDA6D196D002A1A6E05DD9142B4BF15
:101490000021012106DD04E09142CCBF00210121A1
:1014A00000DA1A6519B12046FFF747FD03E0586ED0
:1014B000322100F085F905A8FFF714F94046FAF744
:1014C00023FA0FB0BDE8F08F0388994213B50C469C
:1014D0000ED2406850B1FFF7F7F802AB50F8244045
:1014E00043F8040D1846FFF7FDF802E0044600E05B
:1014F0000024204602B010BD13B5044640B1FFF7EA
:10150000E3F802AB048843F8040D1846FFF7EAF845
:10151000204602B010BD2DE9F743054600283DD016
:101520004AB10846114602F04FFBD0F101040746CC
:1015300038BF002401E0144617462846FFF7C4F8D8
:1015400002AEB0F8008046F8080DD0F80490684666
:10155000FFF7C8F824BB08F101014846890002F0F2
:1015600081F9814618B93846FFF7E8F818E0FFF727
:10157000ABF802AB43F8040D40F828701846FFF7AB
:10158000B1F82846FFF7A0F8038800900133C0F8AF
:10159000049003806846FFF7A5F802E0044600E0E7
:1015A0000124204603B0BDE8F08337B5054618B3E3
:1015B000FFF78AF800904068C0B1FFF785F8002473
:1015C0000190009B1B889C4206DA019800EB840086
:1015D000FFF7D2FA0134F4E701A8FFF783F8009887
:1015E0000430FFF7C9FA009B00221A806846FFF713
:1015F00079F82846FFF7A2F803B030BD73B50E4660
:10160000054658B1FFF760F802AC314644F8040DC6
:10161000FFF75AFF05462046FFF764F8284602B058
:1016200070BD0820FFF722BB30B585B004461022FC
:101630000D466846002107F070FA2046FFF73AF899
:1016400003691BB1019400956846984705B030BD09
:1016500070B50D4C2368132B06460D4612DCFFF7C0
:1016600029F803696E6043B122682846013222607E
:1016700098472368013B236070BD2846BDE8704051
:10168000FAF742B970BD00BF20D9012038B5054630
:1016900000F00FF8044654B1AC4207D02046FFF7E3
:1016A00009F8036AAB4202D01C46F4E70024204646
:1016B00038BD08B5F8F71FFF18B1FEF7FBFFC0698A
:1016C00008BD08BD1FB5044600216846102207F07A
:1016D00024FA606850B1FEF7EDFF40F21313406842
:1016E0000093694663680393F9F78CFC04B010BD5E
:1016F00037B5054668B1FEF7E7FF02AC44F8040DC4
:101700000068FDF767FC2046FEF7ECFF2846FFF770
:1017100015F803B030BD73B5054601A8FDF7D8FB39
:101720000446DCB120460121FDF7AFFC019B83B1EB
:1017300078B11846FEF7BEFF4368AB4209D1204698
:1017400001A9019EFDF7DCFB04463046FFF7D0FF00
:10175000E7E7204601A9FDF7D3FBE1E702B070BD42
:101760002DE9F34180460C200F461646FFF77EFA1E
:101770000446F0B1FDF79EFC2246811901230F4873
:10178000FDF7DAFB0546204685B1FEF79DFF0346CF
:1017900002A8C3F8048040F8043D9F601D60FEF776
:1017A000A1FF28463146FDF749FC02E0FEF7C6FFDF
:1017B0002C46204602B0BDE8F08100BFC5160108E6
:1017C00013B50C4680B1FEF77FFF01901CB1006895
:1017D0002146FDF733FC02AC54F8043D1868FDF7D0
:1017E0003BFC2046FEF77EFF02B010BD2DE9E7412D
:1017F0000E4690460746D0B1FEF766FF034602A8A4
:10180000B3F90410B3F90020B3F9065040F8043DD1
:10181000B3F902308A1AED1AD243ED431644454417
:10182000FEF760FF384631462A46F8F70FFD03B051
:10183000BDE8E08130B50A4D0A4C2B6854F823000E
:1018400085B050B104A9182341F8103D6946FFF74F
:10185000FFFE2B68002244F8232005B030BD00BFF6
:101860001817022034170220F8B5094B094A04461C
:1018700018680F4652F82010A14215461E4601D0A6
:10188000FFF7D8FF336845F82340034B1F70F8BDBE
:1018900018170220341702201C17022038B50546FD
:1018A0000C4641B1F8F727FE28B1A5602146BDE8F6
:1018B0003840FFF7CDBE38BD7FB50A4A03461068F1
:1018C000094A52F8200048B100930E230191029377
:1018D00002A900AB0593FFF7BBFE012007B05DF83E
:1018E00004FB00BF181702200817022010B50C4691
:1018F00030B129B1FEF7DEFE034603CB2060616004
:1019000010BD38B50546F8F77FFEFF28044603D022
:10191000FE2808BFFF2400E0FE242846F8F7EBFD70
:101920002146BDE83840F8F7ABBE02F00ABD000022
:10193000024B1A6802601860704700BF2C17022023
:101940002DE9F043044687B0002839D0FEF7BCFEED
:101950000346019003C804AD85E8030001A81E6A90
:10196000D3F82890FEF7BEFE2046FFF78FFE07460D
:1019700030B32046F8F7BFFD19F0020F804604D0BF
:10198000284641463246F9F725FB2046FEF79CFEE5
:1019900001904046FEF798FE03903846FEF794FE0D
:1019A000039B019AD96906620290116201A8DC6169
:1019B000FEF798FE03A8FEF795FE02A8FEF792FE3A
:1019C00007B0BDE8F0832DE9F84FDDF828B0DDF869
:1019D0002CA005460E4690461F461446894635F80B
:1019E000020BD847D047013C49F8040BF7D11F2F11
:1019F00006D8304641463A46BDE8F84F01F058BD9A
:101A0000BDE8F88F2DE9F84FDDF828B0DDF82CA0FF
:101A100005460E4690461F468946044614F8010BBB
:101A2000D847D0472B1B434449F8040B002BF5D172
:101A30001F2F06D8304641463A46BDE8F84F01F020
:101A400037BDBDE8F88F00002DE9F04F9DB0064688
:101A50000F910D92002800F08683FEF735FE1CAB37
:101A6000446943F81C0D1846FEF73CFE3046FAF771
:101A700087FF0828014602DD002C00F0C381012207
:101A80004FF0000830461B920B92CDF86880FEF7AD
:101A90001BFE0368DFF80CA61B69B0F90A105B682F
:101AA0000E930DF1700BDAF800304BF8140D046949
:101AB0004569D0F80C90B0F90870587C1291FCF789
:101AC00033F9DAF800301090587CFCF74BF90346F4
:101AD00058460993FEF706FE082C51460B9A099BBF
:101AE00004D9102C8CBF0422022205E0012C03D162
:101AF00011940DF1680800E011920E98984200F0E0
:101B0000E2800B68587CFCF735F91390B800FFF7BA
:101B10002FF80C90002800F026833046FAF7CCF816
:101B20000646002D00F0BE802846FEF7CDFDDDF80C
:101B300034B018904FF0000A129A924580F2AE80AD
:101B4000189800231993836819A95B69524698472E
:101B5000B84205462FD10C98FEF7B6FD082C014679
:101B6000169009D90E9A139B0092019330463A467B
:101B7000109BFFF728FF08E00E98139A009001923F
:101B800030463A46109BFFF73DFF01231098029024
:101B90001CAD002200930193039255F8182D049276
:101BA0000F98CDF8148059463A46FCF7FFFA2846BC
:101BB000FEF798FD60E0012C5CD1002D5CD01998F7
:101BC0000F99CDF80C90082290FBF2F232440123D9
:101BD000049200F0070200930844019302930692D6
:101BE00059462A46CDF81480FCF704FA199B189838
:101BF0001D44836819955B6919A9524698470546A3
